:100000002428002051A20000A1A20000DDA00000D1
:10001000DDA00000DDA00000DDA00000DDA00000EC
:10002000DDA00000DDA00000DDA00000D59C0000E8
:10003000DDA00000DDA00000919C0000DDA000001C
:1000400015A200007B94000015A2000015A200007C
:1000500015A2000015A2000015A2000015A20000C4
:1000600015A2000015A2000015A2000015A20000B4
:1000700015A2000015A2000015A2000015A20000A4
:1000800015A2000015A2000015A2000015A2000094
:1000900015A2000015A2000015A2000015A2000084
:1000A00015A2000015A2000015A2000015A2000074
:1000B00015A2000015A2000015A2000015A2000064
:1000C00015A2000015A2000015A2000015A2000054
:1000D00015A2000015A2000015A2000000000000FB
:1000E0002D0C0000000000004DA0000000000000EA
:1000F0004DA00000000000004DA000000000000026
:100100004DA00000000000004DA0000048030020AA
:10011000A9090000000000004DA000000000000040
:100120004DA00000000000004DA0000000000000F5
:100130004DA00000000000003D9400000000000001
:100140004DA00000000000007794000000000000B7
:100150004DA00000000000004DA0000000000000C5
:100160004DA0000000000000850700000000000016
:100170004DA00000000000004DA0000000000000A5
:100180004DA00000000000004DA000000000000095
:100190004DA00000000000004DA000000000000085
:1001A00071940000000000004DA00000000000005D
:1001B0004DA00000000000004DA000000000000065
:1001C0004DA00000000000004DA000000000000055
:1001D0004DA00000000000004DA000000000000045
:1001E0004DA00000000000004DA000000000000035
:1001F0004DA00000000000004DA000000000000025
:100200004DA00000000000004DA000000000000014
:100210004DA0000053B94AB9002908BF00281CBFEF
:100220004FF0FF314FF0FF3000F08EB9ADF1080C08
:100230006DE904CE00F01AF8DDF804E0DDE90223F0
:1002400004B07047430803F05533C01A830803F025
:10025000333300F03330184400EB101000F00F304F
:1002600000EB002000EB0040000E70472DE9F04746
:100270008C460D460446089E002B51D18A421746F3
:100280006DD9B2FA82FEBEF1000F0BD0CEF1200C78
:1002900001FA0EF520FA0CFC02FA0EF74CEA050CF6
:1002A00000FA0EF44FEA174A250CBCFBFAF81FFAC5
:1002B00087F90AFB18CC45EA0C4508FB09F3AB4269
:1002C0000AD9ED1908F1FF3280F02381AB4240F2E8
:1002D0002081A8F102083D44ED1AA4B2B5FBFAF062
:1002E0000AFB105544EA054400FB09F9A14509D968
:1002F000E41900F1FF3380F00A81A14540F2078143
:1003000002383C44A4EB090440EA08400021002ED6
:1003100061D024FA0EF4002334607360BDE8F087E6
:100320008B4207D9002E54D0002186E821000846D0
:10033000BDE8F087B3FA83F1002940F08E80AB422C
:1003400002D3824200F2FA80841A65EB0305012091
:10035000AC46002E3FD086E81010BDE8F08712B9F9
:100360000127B7FBF2F7B7FA87FEBEF1000F34D1D1
:10037000EB1B3A0C1FFA87FC0121B3FBF2F8250CAA
:1003800002FB183345EA03450CFB08F3AB4207D9DF
:10039000ED1908F1FF3002D2AB4200F2D180804665
:1003A000ED1AA3B2B5FBF2F002FB105543EA054487
:1003B0000CFB00FCA44507D9E41900F1FF3302D27D
:1003C000A44500F2B8801846A4EB0C0440EA0840AB
:1003D0009DE731463046BDE8F087CEF1200405FAAE
:1003E0000EF307FA0EF720FA04F83A0C25FA04F493
:1003F00048EA0308B4FBF2F14FEA184502FB114446
:100400001FFA87FC45EA044501FB0CF3AB4200FAF6
:100410000EF409D9ED1901F1FF3080F08A80AB426A
:1004200040F2878002393D44EB1A1FFA88F5B3FB8E
:10043000F2F002FB103345EA034500FB0CF3AB423C
:1004400007D9ED1900F1FF386FD2AB426DD90238F0
:100450003D44EB1A40EA01418FE7C1F1200722FA3F
:1004600007F88B4005FA01F448EA030320FA07FE77
:100470004FEA134CFD404EEA040EB5FBFCF94FEA7F
:100480001E440CFB19551FFA83F844EA054509FB85
:1004900008F4AC4202FA01F200FA01FA08D9ED18A8
:1004A00009F1FF3043D2AC4241D9A9F102091D4400
:1004B0002D1B1FFA8EFEB5FBFCF00CFB10554EEA0F
:1004C000054400FB08F8A04507D9E41800F1FF3502
:1004D00029D2A04527D902381C4440EA0940A4EBA0
:1004E0000804A0FB02894C45C6464D4615D312D0E0
:1004F00056B1BAEB0E0364EB050404FA07F7CB40E0
:100500001F43CC40376074600021BDE8F087184677
:10051000F8E69046E0E6C245EAD2B8EB020E69EB97
:1005200003050138E4E72846D7E7404691E78146CE
:10053000BEE7014678E702383C4445E7084608E74D
:10054000A8F102083D442BE7704700BF10B50446F0
:1005500086B028B10146104800F02AFE06B010BD52
:100560000E4800F025FEA0230394ADF80E30F023D2
:100570000494ADF81030012300930949094B059408
:10058000032203A801F0A0FD014608B10648E3E7F5
:10059000064800F00DFEE1E708B6000028B60000AE
:1005A000F0B500008CB600003FB6000065B6000054
:1005B00008B5074800F0FCFD064801F00BFD0146B8
:1005C00020B10548BDE8084000F0F2BD08BD00BFFD
:1005D00075B600004D05000008B600000A2838B5C1
:1005E0000446074D04D1286843680D215B6898478D
:1005F00028684368E1B25B689847204638BD00BF71
:10060000B8030020014800F0A3BC00BFDD050000D6
:1006100008B5044809F092FE034B1860FFF7F2FF9B
:10062000002008BDA0B60000B803002003689B6846
:100630001B68D3F8082132B10020C3F80801D3F8B1
:1006400018350B7070474FF0FF30704703689B6898
:100650001B68C3F81C15D3F81C21002AFBD000220C
:10066000C3F81C210846704703689B681B68D3F8D1
:10067000240118B1D3F88004C3F8800400F00F00FF
:1006800070470000F8B503689B68054618481C6869
:1006900009F054FE436806461F680D2240F201131C
:1006A0000021B84773681F68002319460F2230469F
:1006B000B8470D23C4F80C350F23C4F81435AB68C4
:1006C0004FF4E1321A602B689B681B684FF0EB72A5
:1006D000C3F824250423C4F8003500200123C4F8FE
:1006E0001C01C4F80801A3602360024B6B60F8BDD5
:1006F000B1B60000D8B60000084BC3F84005D3F8E7
:100700000435C01A20F07F40054B0238984282BF62
:10071000044B4FF40032C3F8002170470010014031
:10072000FDFF7F0000E100E010B5124B124CD3F842
:1007300004052268801A20F07F40B0F5A37F11D90C
:100740000E49096840F24713B0FBF3F0884228BF16
:10075000084603FB002323F07F432360084B186007
:100760000AF086FC2068BDE8104000F24710FFF751
:10077000C3BF00BF00100140C0030020BC03002025
:10078000FC020020024B0022C3F84021FFF7CCBF3F
:100790000010014046F23543984228BF1846054BE9
:1007A0001860054B1B6840F2471202FB0030FFF750
:1007B000A3BF00BFBC030020C003002008B5074B47
:1007C0000022C3F84021064B4FF40032C3F88021C9
:1007D000FFF7AAFF034B01221A6008BD0010014079
:1007E00000E100E0BC03002070B5184809F0A6FD48
:1007F00048B34368164D1B6801219847154B0024E8
:100800001C60154B01261E6040F24713C5F80845D1
:10081000C5F840354FF48033C5F84433C5F8043388
:100820000E4BC5F840414FF40032C3F880213146E9
:100830002246112009F0F2FB112009F0C5FBAE6041
:1008400020462E6070BD4FF0FF3070BDB8B600007E
:1008500000100140C0030020BC03002000E100E0C4
:1008600003689B689A68836810B5DC68002024FAE6
:1008700000F3DB0707D500F5A27352F82330C3F36A
:1008800004238B4204D001300828F0D16FF012000D
:1008900010BD00688068006841B9D0F8101521FAD1
:1008A00002F202F001021A6000207047D0F8102511
:1008B000F9E700688068006849B9012191401BB1DF
:1008C000C0F8081500207047C0F80C15FAE7C0F80A
:1008D0000435F7E710B583683AB11A680A605A68B8
:1008E000196002B95960002010BD18680028FAD0BC
:1008F00081420ED15C68086832B9A142186000D10B
:10090000586000230B60EEE7A142106008BF5A60F8
:10091000F7E702460068E9E7F8B514460268876819
:1009200092680D469668A1B92146FFF799FF002805
:1009300011DBBA68012303FA04F4144300F1400206
:1009400003FA00F0BC6046F82250C6F804032846BB
:10095000F8BD6FF02200F8BDF8B51446026886684D
:1009600092680D46976889B92146FFF779FF0028FC
:100970000EDBB268012303FA04F403FA00F022EA62
:100980000404B460C7F808032846F8BD6FF02200DD
:10099000F8BD08B500220121062009F03FFB062022
:1009A00009F012FB002008BDF8B5036806469B68F5
:1009B000B4689868002213461546012700EB8201AF
:1009C000D1F800E1BEF1000F08D0C1F80051D1F814
:1009D0001015C1F3042107FA01F10B430132082A73
:1009E000ECD1A56806201D4009F0FCFA246824B962
:1009F0000620BDE8F84009F0E7BAA3681D42F5D02B
:100A000063682A46214630469847EFE72DE9F843C8
:100A1000144602688768926880469568166819B11E
:100A20006FF02200BDE8F88303F44071B1F5807FD8
:100A3000C3F30132C3F381394FD0B1F5007F0CBF4E
:100A40000420002013F0010FDFF8B8C04FEA820243
:100A500004F5E07E4AD00C2841D10121A140C6F81E
:100A600008154A445CF8222042F00302024313F0C6
:100A7000020046F82E2043D09906D1D55A063AD422
:100A800013F0040F14BF4FF480364FF40036F868AB
:100A9000FFF7D8FB082831D021464046FFF7E0FE9B
:100AA0000028FB6808DADA4392FAA2F0002AB0FACA
:100AB00080F008BF4FF0FF302402012204F4F85404
:100AC000824044F0010400F5A27013433443FB60FC
:100AD00045F820400020BDE8F8830C20B2E7042848
:100AE00002BF0121A140C6F80C15BAE702EB0901CB
:100AF0005CF82120BAE74FF44036C8E76FF00400F5
:100B0000BDE8F883E4B6000010B54FF02003EFF322
:100B1000118283F31188114C237823B982F3118851
:100B20006FF0440010BD013BDBB223701BB182F3B8
:100B30001188002010BD0A4B1878012128B12170BE
:100B400082F311886FF00A0010BD197082F31188CA
:100B50004FF080425160187010BD00BFD5030020D7
:100B6000D403002008B500221046012109F056FAEE
:100B7000002009F029FA002008BD0000F8B54FF068
:100B80002002EFF3118382F31188254A1078441C68
:100B9000147060B183F311884FF08043D3F80C34A4
:100BA00013F4803F14BF00206FF04300F8BD1D4DCB
:100BB0002F782FB1107083F311886FF00A00F8BD01
:100BC00001262E7083F311884FF0804419B3384604
:100BD00009F008FAC4F80071D4F80433C4F80463C7
:100BE0002660D4F8002192B10022C4F800210E4AF8
:100BF00013F0010F4FF0010308BFC4F808330020C1
:100C0000C2F8803109F0E0F900232B70C4E720BF5F
:100C100040BF20BFE5E7C4F800112660F4E700BF3D
:100C2000D5030020D403002000E100E0F8B54FF028
:100C300080430546D3F808E1D3F80423D3F80C44E5
:100C4000D3F80071D3F80401D3F80C11D3F8106174
:100C500002F00102BEF1000F03D04FF0000EC3F806
:100C600008E127B14FF080430027C3F800713AB183
:100C7000E30341BF4FF080430122C3F808231A6108
:100C800020B14FF080430022C3F8042149B14FF056
:100C900080440021C4F80C112846FFF735FF0123DA
:100CA000636176B14FF0804300210124C3F8101135
:100CB0002846C3F80443FFF761FF10B9014BC3F89E
:100CC0000041F8BD00E100E0F8B54FF08044074670
:100CD000D4F8186416F480360D4648D1304609F031
:100CE00081F9C4F804610222D4F80433C4F804235F
:100CF0000122C4F81855A260D4F804219AB39B07C6
:100D000058BF02234FF000021A4EC4F8042158BF06
:100D1000C4F808330124C6F88041002009F054F9D2
:100D20004FF0804300211822C3F80823C3F80C11A8
:100D3000C3F8101115F003010CD11020C3F83805C9
:100D4000C3F804233846C3F80443FFF717FF08B974
:100D5000C6F800414FF08043D3F8180480F4803087
:100D6000C0F30040F8BD20BF40BF20BFC4E7002053
:100D7000F8BD00BF00E100E00139034611F8012F82
:100D80000AB91A70704703F8012BF7E701380139E7
:100D900010F8013F11F8012F934202D1002BF7D137
:100DA0001A46981A704770B582B1013A0C4603464C
:100DB00003D11A782078101A70BD1E782578AE42BB
:100DC00000F1010001F10101EFD0F2E7104670BD22
:100DD00081EA000313F0030F70B503460BD0013B0B
:100DE0000A4491421BD170BD002AFCD011F8014B7E
:100DF00003F8014B013A9C07F6D11E1F0D46541B08
:100E00000C44032C06D822F003042144234402F0AE
:100E10000302E4E755F8044B46F8044FEFE711F8F6
:100E2000014B03F8014FDCE770B5C9B203469C07DC
:100E300011D141EA012444EA04441E46951B1D4495
:100E4000032D0ED822F00304234402F003021A44B7
:100E5000934209D170BD002AFCD003F8011B013A6E
:100E6000E5E746F8044BE9E703F8011BF0E700204B
:100E7000704700000B6801330B60014B1B6818477B
:100E80001C0000202DE9F04F85B09B460E9CDFF83A
:100E900090A0012CB8BF0124012B0CBF30232023CC
:100EA0001546804689460194029301260A270022AE
:100EB0000AF101040AB9AA451FD2B5FBF4F049466C
:100EC0003030C04701360122013F012FB5FBF4F15C
:100ED0004FF00A0304FB1155BAFBF3FAE8D1494677
:100EE00005F13000C047BBF1030F03D1019B9C1BF0
:100EF000002C0FDC05B0BDE8F08F019BBB42E3DBAB
:100F0000BBF1020FE0D84946029803920136C04770
:100F1000039AD9E749462020C047013CE8E700BFD3
:100F2000FFC99A3B0A688B6830B512B14C68A3427E
:100F300002DB01338B6030BD651EAB420BBF8C60A2
:100F40005C1C00218C600CBFD154D05430BD00001B
:100F5000014B1860704700BF1C0000202DE9F04FC6
:100F600089B04FF0000A06460F4604921C464FF027
:100F7000FF39D0465546049B187810B909B0BDE832
:100F8000F08F45B9252800F0F8803946B047049B1A
:100F900001330493EFE7642855D018D839280AD8CC
:100FA000312844D22D2830D0302831D0252807D1FF
:100FB0003946B04763E058287DD0632800F0D780D9
:100FC00039462520B047049B39461878F1E7702848
:100FD00067D006D8692836D06C2831D06828D6D09A
:100FE000EEE775284DD00CD87328E9D104F1040B35
:100FF0002468013C14F8010F002840F0B5805C46DD
:101000003DE0782857D07A28E9E74FF00308BEE79B
:10101000B9F1000F0EDAB8F1000F00F0B480A0F1C2
:101020003009B8F1000F08BF4FF00208AFE7B9F17F
:10103000000FF4DB0A2303FB0909A9F13009F0E7EB
:101040000AF1010AA3E7BAF1010FC5BF073424F082
:10105000070325681D68D4BF043403F10804002D7C
:1010600005DA39462D20B0476D4209F1FF39CDF838
:10107000009043462A4639463046FFF703FF0025D5
:1010800085E7BAF1010FC5BF073424F007032268D2
:101090001A68CDF80090CCBF03F10804043443462D
:1010A000E9E739463020B04739467820B0474FF05D
:1010B00008094FF00108BAF1010FC7BF073424F047
:1010C000070323680593C2BF03F108041B68059357
:1010D0004FF008024FF00003D8BF04340393079386
:1010E00093460BF1FF3B059B4FEA8B0023FA00F080
:1010F00010F00F0009D1079B13B9BBF1000F22D1EB
:101100004FF0300E07E0069AEBE709288CBF4FF04E
:10111000570E4FF0300E394670440692B047039B8D
:10112000079501330393BBF1000FECD1B8F1030F26
:101130002CD1039BC3EB4905002DA0DD39462020AF
:10114000B047013DF8E7531E91450693EBDBB8F13C
:10115000010F03D139463020B047E4E7B8F1020F60
:10116000E1D139462020F7E73946B04742E7206809
:10117000251D3946B0472C4681E7AA46A8464FF0C0
:10118000FF39012503E74FF0010800E75D46FEE661
:1011900013B502AC002344F8043D02460B46034855
:1011A0002146FFF7DBFE019802B010BD750E00006E
:1011B0000FB407B504A951F8040B0191FFF7E8FF3C
:1011C00003B05DF804EB04B0704700000CB430B518
:1011D00085B008AB044653F8042B0190029100251A
:1011E00001A9074800930395FFF7B8FE0398029BF7
:1011F0009842B8BF255405B0BDE8304002B07047F2
:10120000250F00007047000070B54FF02003EFF38A
:10121000118583F31188144C144E237803EBC31209
:10122000013303F003033244237085F3118840290E
:1012300028BF40210E4D0138134602EB4106B34250
:1012400004D1002302F81130104670BD44782409FF
:1012500002332C5D03F8024C10F8014F04F00F0428
:101260002C5D03F8014CEAE7D6030020D7030020E9
:1012700064B70000438A1844173020F00300704719
:1012800070B50B4D06460FCD8AB06C460FC40FCD1E
:101290000FC495E80300092E84E803009BBF0AAB46
:1012A00003EB8606034856F8280C0AB070BD00BF51
:1012B000B0B500009DBD000000B5BFF35B8F50E8E6
:1012C000003F43EA010240E8002EBEF1000FF6D1D4
:1012D000BFF35B8F18465DF804FB00B5BFF35B8F6F
:1012E00050E8003F03EA010240E8002EBEF1000F83
:1012F000F6D1BFF35B8F18465DF804FB7FB505465A
:1013000010460E461446FFF7B5FF4388AB420BD09C
:101310000E4A02930E4B0392009301950D4B0E4A19
:101320000E490F48FFF744FF2046FFF7A3FF43682D
:101330004BB146702046FFF79DFF406804B0BDE802
:10134000704009F033BE04B070BD00BFB8BA0000F1
:10135000BDBA000075B700006BBA000072BA000099
:1013600075BA0000074BBFF35B8F420903EB8203A2
:1013700000F01F00DB6EBFF35B8F43FA00F000F05C
:101380000100704720000020F8B505460E460F48C2
:101390004FF0FF3108F018FB0021044608F068FB0D
:1013A0002046FFF767FF002202702046FFF762FF2A
:1013B00045802046FFF75EFF0321426004F10C00E8
:1013C00008F082FB867005802046F8BDF4000020FE
:1013D00070B5154686B00C4619B9FFF7D5FF04461F
:1013E00048B301AE01220021304609F0D7FD204666
:1013F000FFF740FF4660204608F062FB21460F4899
:1014000008F03BFB42F21071304609F013FE204613
:10141000FFF730FF407830B1204608F03BFB6FF01B
:10142000040006B070BD0DB12C60FAE7204608F04C
:1014300031FB2846F5E76FF03600F2E7CC000020DC
:1014400070B5154D062205F108010646FFF7ABFC05
:101450000446D8B1062142F20500FFF795FF044685
:10146000B0B1062231460C3008F034FB2146002290
:1014700042F20500FFF7ACFF044638B906223146B8
:1014800005F10800FFF7A4FC0123EB71204670BDB5
:101490006FF03604FAE700BF2000002007B50621F0
:1014A000684603F0FDF840B99DF80530684603F042
:1014B0003F038DF80530FFF7C3FF03B05DF804FB71
:1014C00037B50720FFF74EFF70B3022142F20C0040
:1014D000FFF75AFF044650B302210C3008F0F4FA2B
:1014E000022205460021FFF79FFC002321466B7076
:1014F0002B7001AA42F20C00FFF76AFF044680B984
:10150000019BDB681C784CB96FF080010948FFF73C
:10151000E4FE6FF400710748FFF7DFFE019808F062
:10152000B9FA204603B030BD6FF04404F9E76FF01C
:101530003604F6E78C0000202DE9F8430C46202104
:1015400007469046FFF720FF064600283CD02021A2
:101550000C3008F0B9FA202200210546FFF764FCA0
:101560004FF00009C14506D1314638460022BDE89A
:10157000F843FFF72DBF62782B78D11802311F296D
:1015800004F1080406DD304608F084FA6FF0150017
:10159000BDE8F883E918501C4870981CC0B20133AC
:1015A000287055FA83F314F8081C5970013054F868
:1015B000041C2844FFF70CFC2B7814F8072C134468
:1015C0002B7009F10109CDE76FF03600BDE8F88313
:1015D00008B50820FFF7C6FE38B90720FFF7C2FE9E
:1015E00018B1BDE80840FFF76BBF002008BD01231C
:1015F00010B50621044600F8013B03F051F818B974
:10160000A37963F03F03A37110BD00002DE9F04101
:1016100094B00DAF3A46002140F60340FFF7D8FEE4
:10162000044600287FD10D9BDB681B786BB9B54A57
:101630001360B54BBFF35B8F012253E8001F43E8F3
:1016400000200028F9D1BFF35B8F0D9808F022FA33
:101650003A46002141F20300FFF7BAFE0446002893
:1016600061D10D9BA94ED9680822013106F11600FF
:10167000FFF7AEFB0D9808F00DFA21463A4641F20D
:101680000100FFF7A5FE3546044600284BD10D9812
:10169000C3685A78B273D9789A7842EA01223282C2
:1016A0001A79F273197ADA7942EA012272825A7946
:1016B0009B7942EA0323B38208F0ECF921463A46CB
:1016C00041F20900FFF784FE044660BB0D9BD96818
:1016D00006220131701CFFF77BFB0D98347008F077
:1016E000D9F921463A4641F20200FFF771FE04465D
:1016F000C8B90D9BD9684022013106F11E00FFF7E1
:1017000067FB0D9808F0C6F9B37E58060FD4804BDE
:101710000193804B0093804A804B81498148FFF7B9
:1017200047FD6FF01204204614B0BDE8F081214659
:101730003A4642F20300FFF74BFE04460028F2D17E
:101740000D9BD9680822013106F17000FFF740FBBC
:101750000D9808F09FF9B37E990640F1868095F8C0
:101760003A301A0700F19D80082142F20100FFF78C
:101770000BFE044600287FD008210C3008F0A4F9A5
:1017800095F8403003F00603062B14BF02234FF4F4
:10179000C173002203701B0A43708270C270027111
:1017A00042718271C271214642F20100FFF710FEC0
:1017B00004460028B7D1082140F60140FFF7E4FDB8
:1017C0000646002858D008210C3008F07DF9802307
:1017D00043700223C3702023047084700471447129
:1017E0008471C3712246314640F60140FFF7F0FD97
:1017F0000446002897D107900722CDF81F0007A9BB
:101800004248FFF7D0FA00285FD1474A1368904654
:10181000002B40F08F804FF08053D3F8A42001328A
:1018200007D1D3F8A8304FF6FF729BB2934200F075
:10183000AA804FF08052D2F8A030DB0740F1A3809D
:1018400001232B70D2F8A4306B70C3F307211B0C5B
:10185000EB701B0AA9702B71D2F8A8306B71C3F31F
:10186000072363F03F03AB716DE0022140F66D404A
:10187000FFF78AFD064610B96FF0360453E70221E0
:101880000C3008F021F901234470037022463146E0
:1018900040F66D40FFF79CFD044600283FF45FAF23
:1018A00041E73A46002142F21C00FFF791FD044651
:1018B00000287FF438AF0D98C36853F8012F5B6898
:1018C000EB67AA6708F0E6F84EE7184B18689A88A5
:1018D00009909B79ADF8282009A907220B488DF8BB
:1018E0002A30FFF760FA00288FD02B780BAE002B40
:1018F00079D0012B00F0B9800D4A07213046FFF75F
:1019000065FC74E0280600208C00002020000020E8
:10191000B8BA000000BB0000C5BA0000C4B70000A0
:1019200072BA0000CCBA000004150020D8B500003F
:10193000BCBB000000211E684D4A07230846B04783
:1019400007287FF468AF2B78012B04D1AB7903F023
:10195000C003C02B3CD0474B0193474B0093474AF1
:10196000474B48494848FFF723FC6FF01506414BA9
:101970000193414B0093414A444B42494448FFF78D
:1019800017FC3446CFE63A48FFF731FE06460028FA
:10199000EDD1D8F8003093B1D3F80480344A07234E
:1019A0000146C0470728CED0324B0193324B0093FB
:1019B000324A334B33493748FFF7FAFBC3E72D4B25
:1019C0000193354B0093354A2D4B2E493448F3E7AC
:1019D0003448FFF735FD06460028C8D104213248B7
:1019E000FFF76AFC81E731493046FFF7C5F9AB796B
:1019F00005966A780492AA780392EA7802922A7984
:101A000001922B4E6A7900921B212A4A3846FFF731
:101A1000DDFB8DE8C000284B284A1A490296284869
:101A2000FFF7C6FBAF7B3846FFF72AFC0596AB8A6B
:101A300004932B8A0393029701901F4B1F4A11496D
:101A400000962048FFF7B4FBEF7B3846FFF718FC01
:101A500004966B8A0393019002970096164B174ADF
:101A600008491948FFF7A4FB5DE61849BCE700BF29
:101A700020000020B8BA000000BB0000C5BA00007A
:101A8000CCB7000072BA00006DBB0000EAB70000DE
:101A90008FBC000008BB0000BDBA00006BBA00009C
:101AA00037BB0000210000208C000020AEBB0000EE
:101AB00027B60000C3BB0000DCB70000E6BB000097
:101AC000EDBB00000ABC000058BC0000B5BB000024
:101AD000064B4FF0FF3041F6FF71C3E90001044BA4
:101AE0001F200021C3E90001704700BF4001002012
:101AF0004801002010B5FFF789FD044630B90221E6
:101B00000648FFF7D9FB2046FFF762FD044B1B6830
:101B10001BB12046BDE81040184710BD8C000020C6
:101B200024060020024BD3F8C030DB68184700BF02
:101B3000200000202DE9FF413E4C3F4D04F1AC0850
:101B40006B683D486FF310334FF0FF3201216B603B
:101B500008F05AFE002853D16B68C3F30433022BFC
:101B60000DD0082B0ED053B1344A0193344B02925E
:101B70000093344A344B35493548FFF719FB09F0D7
:101B800073F9DDE72E79002EF9D13146404607F092
:101B900056FF0746002843D04FF0FF312D4809F08B
:101BA00049FAD4F89430D3B9384607F089FFC4F81D
:101BB00094003846FFF7B6FF0028E0D01F4B029391
:101BC000254B01900093254A254B20492548FFF7D6
:101BD000EFFA204809F0EAF900239B68FFDE174B73
:101BE00001931D4B00931D4A1D4B18491E48FFF7DA
:101BF000DFFAD4F8940007F04DFFC4F89460D3E7FF
:101C00000E4B0193144B0093144A184B0F4918487C
:101C1000FFF7CEFA404080F311884FF0040002DF56
:101C2000064B01930C4B00930C4A0D4B074911488E
:101C3000EEE700BF20000020E8000020B8BA000056
:101C4000BDBA00006BBA0000A7B7000072BA00006E
:101C5000BEBC0000A000002000BB0000C5BA000010
:101C60009EB7000067B80000EFBC0000B6B70000E8
:101C70001ABD000044BD00002DE9F04F83685B8B66
:101C8000032B89B004460FD86C4B01936C4B009327
:101C90006C4A6D4B6D496E48FFF78AFA204607F093
:101CA000F9FE6FF0150032E0FFF7E4FA0678012E36
:101CB0006BD1E7683B780E3B012B72D85F4B0193E9
:101CC0005F4B00935F4A634B60496348FFF770FACC
:101CD000404080F311884FF0040002DFE7685F485E
:101CE0006FF01001FFF7F9FA3B7843B9791C4022F5
:101CF0005B48FFF76DF831465848FFF7DDFA594B5E
:101D00001D687E1C35B9204607F0C4FE002009B0CE
:101D1000BDE8F08F3A782B68002A0CBF30460020CF
:101D200098476D68EEE7504DE0682A68002AEAD0CF
:101D3000037823B90130904700232B60E3E70020AC
:101D4000F9E7258AE0682946FFF75EFA3B4B0493E2
:101D5000464B03900093464A464B3C494648029501
:101D60000196FFF725FACEE7258AE0682946FFF7B6
:101D70004BFA324B04933D4B03900093029501972D
:101D8000344B3B4A31493D48EBE72C4B02932C4BFB
:101D9000009301962C4B2B4A2C493948FFF708FA3F
:101DA0007CE704F10C050221284607F0A4FE3F78E9
:101DB0003E2FD9D1E7683146284607F09CFE3E7891
:101DC000082E8BD0092EAED0022EBAD1284607F0AD
:101DD0009AFE2C4F069004F1140A069B002B92D019
:101DE00009212846D4F80C8007F085FE3B68D3B162
:101DF00098F8083043442846597A079107F08BFE3B
:101E000098F808300799B4F810B02382814640460C
:101E10002B4610F8012B3E6849B2B0471AFA89F3F5
:101E2000E360A4F810B098F808102846013107F0D4
:101E300062FE069B5E1EF3B20693CEE7B8BA0000C0
:101E400000BB0000C5BA0000F3B7000072BA000082
:101E500099B8000094B700004DB900008C00002034
:101E6000E005002020060020DC050020BDBA0000AF
:101E70006BBA000082B70000C2B80000F7B80000DB
:101E800029B90000280600202DE9F7430446C6685A
:101E9000FFF7F0F90378012B0FD0394B0193394B41
:101EA0000093394A394B3A493A48FFF781F94040A3
:101EB00080F311884FF0040002DF238A012B08D839
:101EC0002F4B01932F4B00932F4A304B3049324810
:101ED000EBE733780E3B012B48D804F10C050221C7
:101EE000284607F008FE33782C4F0E2B0DD00F2B11
:101EF00027D0204607F0CEFD214B0193214B0093C4
:101F0000214A224B22492648CFE7E368032128468D
:101F1000B3F801801E7807F0EEFDA368BB4205D13F
:101F2000E368224619784046FFF7E8F916B11D48E4
:101F300009F03CF8204607F0ADFD002003B0BDE8F5
:101F4000F083E66804212846B6F8029096F80180EE
:101F500007F0D1FDA368BB4204D122463178484640
:101F6000FFF7CCF9B8F1000FE4D0E0E7044B0193A0
:101F7000044B0093044A054B05490B4895E700BF05
:101F8000B8BA000000BB0000C5BA0000FBB70000F3
:101F900072BA00008CB90000D0B90000F400002033
:101FA0000ABA0000A00000202DBA0000084AD2F8AA
:101FB000C0303BB9816841B1C16831B1C2F8C000DD
:101FC000184670476FF0440070476FF01500704777
:101FD0002000002070B52F4DD5F8C03086B00646E1
:101FE00073B92D4B01932D4B00932D4A2D4B2E4948
:101FF0002E48FFF7DDF86FF01204204606B070BDE2
:10200000012105F16C00FFF757F910F001003ED1F6
:10201000274B28491E606FF0080305900490039336
:10202000029001900090244B24484FF46B7209F009
:10203000ADF9D5F8C0309B689847044658B1164BA7
:102040000293164B01900093154A164B16491C48F3
:10205000FFF7AEF8D1E76EB9FFF7D8FA04460028CB
:10206000CBD1022105F16C00FFF726F92046FFF7DE
:10207000AFFAC2E7012105F16800FFF71DF9C307B8
:10208000BBD405F160010F4808F04EFDB5E76FF0D5
:102090004404B2E720000020B8BA000000BB0000F2
:1020A000C5BA000008B8000072BA000012B80000FB
:1020B0002406002064160020351B00002C0600209A
:1020C0003BB80000E81500202DE9F0419846037860
:1020D00013F0010F0546144643880AD14D4A927BFE
:1020E000082A06D89F2B04D86FF015042046BDE8B7
:1020F000F081A8888342F7D81F2BF5D9B0F5804F1F
:10210000F2D80520FFF72EF910B16FF04404EDE787
:10211000224642F20800FFF70FFA04460028E5D1F4
:10212000B8F1000F0CD12B78DA0709D40F2142F255
:102130000600FFF729F9074660B96FF03604D5E7C6
:10214000069A414642F20900FFF7F6F904460028D4
:10215000ECD0CBE70F210C3007F0B6FC0F2206467F
:102160000021FEF761FE6B883380AB887380072304
:1021700073732B78DB0732D50220FFF7F3F810B129
:102180002548FFF75DF9234B1B78737100233371EA
:102190000022394642F20600FFF71AF904460028E9
:1021A000A4D1012142F20A00FFF7EEF8054600280B
:1021B000C3D001210C3007F096FC2246294642F29A
:1021C0000A00FFF705F9044600288FD120211348A3
:1021D000FFF772F840211148FFF76EF886E7A8680C
:1021E00060B1437913F0C00F7FF47EAFFFF728F999
:1021F000044630B1384607F04DFC77E7FFF74EF95B
:10220000F6E701237371B8F1000F01D00223BEE796
:102210000323BCE720000020210000208C000020C8
:1022200038B50546064807F0CFFB044630B100211B
:1022300007F01EFC2046FFF71DF80570204638BD4C
:102240001801002010B501464FF02003EFF3118074
:1022500083F311880C4B0022D3F89440C3F89420E8
:1022600080F3118824B90120BDE81040FFF7D8BFE2
:102270002046FEF7FFFF012303701146204622820D
:1022800007F0F6FB204610BD2000002038B50C30CA
:102290000D460221144607F017FC0570447038BD46
:1022A00038B505464FF0FF30FFF7CCFF0422044657
:1022B0000F21FFF7EBFF042104F10C0007F004FCF1
:1022C00001234370024B05701B884380204638BDB4
:1022D0009406002038B504464FF0FF300D46FFF756
:1022E000B1FFEA1C2060D2B20E21FFF7CFFF2068B9
:1022F00003210C3007F0E8FB01230370054B1B881A
:10230000A0F80130206829460C30BDE8384007F0BD
:10231000DBBB00BF9406002070B5044615460132B1
:102320000E460C34D2B23E21FFF7B0FF0121204609
:1023300007F0CAFB067029462046BDE8704007F04A
:10234000C3BB00000E4B70B51546D3E90023002334
:1023500002F08002134304460E4610D004220821E6
:102360002846FFF793FF042105F10C0007F0ACFBB2
:10237000B4FA84F35B090470A0F80160C37070BD07
:102380004001002070B504461846134B1646D3E9A9
:102390000023002203F0005313430D461BD00F4BC4
:1023A000D3E90023002302F00802134313D00B22C9
:1023B0000421FFF7B1FF08220470A0F80160033088
:1023C00024B9291DBDE87040FEF702BD0021BDE81B
:1023D0007040FEF729BD70BD40010020480100207B
:1023E000034600685968704770B5018A8AB00025B5
:1023F0000229044605950CD8BF4B0193BF4B0093AF
:10240000BF4AC04BC049C148FEF7D2FE28460AB0B9
:1024100070BDC368BE4E1A7858789B7842EA002295
:102420008B42328008D9B44B0193B44B0093B44A29
:10243000B44BB549B748E7E7032104F10C0007F0B6
:102440005AFB3388DAB29B0A013B072B09D8DFE835
:1024500003F004082140080808A3062A07D01D2A13
:1024600013D0012105A8FFF735FF012315E1E3682B
:102470009978188806F098FE002814BF0C200020D8
:10248000FFF70EFF05900598C1E7E368188806F08E
:1024900077FEF1E7012A15D0032AE2D19E4B4FF0D7
:1024A000FF3041F6FF71C3E900019C4B1F20002162
:1024B000C3E9000106F05AFC012105A8FFF70AFF55
:1024C0000023EAE0E068FFF78BFF934BC3E90001CC
:1024D000F2E7013A082AC4D801A353F822F000BF5A
:1024E0000525000029250000652500006324000063
:1024F00063240000632400006324000063240000C0
:1025000081250000092105A8FFF7E4FE0023092228
:1025100003708370C3704FF0FF33427002714371D8
:102520008371C3710372AEE7412105A8FFF7D2FEA4
:1025300000210446402200F8011BFEF775FC202311
:102540006370C023A3712823E37302232374F7234A
:10255000A376FF23E37623770F236377302384F872
:10256000223090E7092105A8FFF7B4FE00210446B8
:10257000082200F8011BFEF757FC6023637182E715
:10258000072105A8FFF7A6FE0146002301F8013B3D
:10259000184607F0ABF876E7013A1B2A3FF661AF21
:1025A00001A353F822F000BF1926000023260000E3
:1025B0003B260000632400005D2600004327000046
:1025C0005F2700006D2700007927000085270000A5
:1025D00063240000632400006324000063240000DF
:1025E00067260000792600007F2600009F26000055
:1025F00063240000632400006324000063240000BF
:10260000BD260000E32600006324000063240000D0
:102610006324000021270000E068FFF7E1FE3F4B44
:1026200054E7042105A8FFF755FE002303701B2281
:10263000837002234270C37025E7092105A8FFF7C4
:1026400049FE00250446082200F8015B2946FEF7F2
:10265000EBFB0F236370A570E57014E7E1680120C0
:1026600007F05CF828E7022105A8FFF733FE0023F6
:1026700003700823437006E706F0C0FB1CE7E3681D
:10268000591C187806F0C2FB0121044605A8FFF783
:1026900021FE002C0CBF002307230370F3E6E36840
:1026A000591C187806F0D6FB0446012105A8FFF74F
:1026B00011FE002C0CBF00230C23EEE7E06806AAF5
:1026C000002300F1100100F025FD112105A8FFF7FE
:1026D00001FE002300F8013B102206A9FEF778FB5B
:1026E000D1E6092105A8FFF7F5FD002300F8013B1D
:1026F000082101F0D5FFC6E6B8BA000000BB000013
:10270000C5BA0000AABD000072BA0000E8BD000012
:10271000940600200EBE0000400100204801002069
:10272000092105A8FFF7D6FDFF230022437083701F
:10273000C37003714371032302708371C27102720B
:10274000A1E6E468A57BA3796279217920880295C6
:10275000657B01950734009406F0ECFFACE602219E
:1027600005A8FFF7B7FD0023037083E7E368591C52
:10277000187807F069F89FE6E368591C187807F0A5
:10278000B1F899E6E368187807F0E8F88CE700BF3D
:10279000F0B50379012B87B004460E4669D0022BB1
:1027A00057D101228DF811208DF816300322954B58
:1027B0008DF81220FF228DF813208DF81520D3E913
:1027C0000023002203F000530025042113438DF859
:1027D00010508DF814103AD08B4BD3E9002300230E
:1027E00002F00202134332D0037A03F00F03012BED
:1027F0001EBF457A063DEDB205F10B02D2B20221B1
:102800003046FFF789FD01230370237A06AA03F0FF
:102810000F031344274613F8083C437017F8083F8A
:102820000646C3F38013837004F10A0106220330C5
:10283000FEF7CEFA0A3606F8015C2A4607F10801CF
:102840003046FEF7C5FA637A1C44A37A735507B085
:10285000F0BD6E4B01936E4B00936E4B6E4A6F4909
:102860006F48FEF7A5FC404080F311884FF004004C
:1028700002DFC37AC588033B122B00F2BD80DFE87C
:1028800003F00ABBBB31A7BB39BBBB4362BB66BB12
:10289000BBBBBB8787005B4BD3E90023002203F05F
:1028A00000531343D3D0584BD3E90023002302F045
:1028B00010021343CBD00C2205213046FFF72CFD2C
:1028C00004F10C010646082220F8025BFEF780FAAC
:1028D000022204F1140106F10A0007B0BDE8F0403D
:1028E000FEF776BA0A460020294607B0BDE8F04058
:1028F000FFF728BD0B462A4600F10801002007B06B
:10290000BDE8F040FFF73EBD3E4BD3E90023002376
:1029100002F4006213439AD007220C213046FFF7DD
:10292000B5FC072106F10C0007F0CEF80023037078
:10293000A0F80150237BC370B4F80D308380B4F845
:102940000F30837183E70A46007B2946CDE72D4B84
:10295000D3E90023002203F0005313433FF477AF81
:10296000294BD3E90023002302F0200213433FF454
:102970006EAF0A2206213046FFF7CEFC0580A38900
:102980004380E3898380238AC380638A03815EE76F
:102990001C4BD3E90023002203F0005313433FF400
:1029A00056AF194BD3E90023002302F04002134332
:1029B0003FF44DAF0A2207213046FFF7ADFC0580FA
:1029C000238A4380638A8380A389C380E389DDE708
:1029D000037B0E2B04D10B462A4600211A208EE7DA
:1029E0000A4A01930F4B029200930F4A0F4B0B4977
:1029F0000F48FEF7DDFB2AE7044B0193044B0093DD
:102A00000C4B2BE74001002048010020B8BA000021
:102A100000BB0000B9BD0000C5BA000072BA0000DA
:102A20000ABA0000BDBA00006BBA0000C8BD0000C1
:102A30003CBE0000D7BD00000379012B06D0023B4D
:102A4000DBB2042B0AD8074AD0567047037A03F04A
:102A50000303032B0CBF0220032070474FF0FF300D
:102A6000704700BFA5BD000008B50248FFF79EFAF9
:102A7000002008BD88BE00007FB5214D00264FF024
:102A8000FF31284608F09EF8044618B3FFF7D4FF3C
:102A90000228039421D801280EBF00214FF0FF31F6
:102AA0000120FFF7BDFB044618B101460398FFF76C
:102AB0006FFE039B0021D88806F094FC04A850F810
:102AC000043D1E6006F018FC24B1238A2046A3B101
:102AD000FFF7D2F808F0C8F9D1E70A4B01930A4B87
:102AE00000930A4A0A4B0B490B48FEF761FB404032
:102AF00080F311884FF0040002DF06F0CBFFE9E716
:102B0000A0030020B8BA000000BB0000C5BA000056
:102B100059BE000072BA00000ABA000037B50C4C6A
:102B20000C4D0DF1020101A806F052FB0028F8D16E
:102B3000019B33B106F084FB0199284607F0F4FFAE
:102B4000EFE74FF0FF31204608F074FAE9E700BFE5
:102B500078030020A00300201FB5038A044663B950
:102B6000154B0193154B0093154A164B1649174800
:102B7000FEF71EFB6FF015000FE0438A0344173386
:102B800023F003031B7853B9FFF72EFC08B1FFF7BE
:102B90007BF9204606F07EFF002004B010BD064AF7
:102BA0000193064B02920093054A064B06490848DA
:102BB000FEF7FEFADEE700BFB8BA000000BB000077
:102BC000C5BA000065BE000072BA0000C5BE0000B4
:102BD000E6BE000010B51A4886B006F0F9FC0446BF
:102BE00068B1184B0293184B01900093174A184B89
:102BF00018491948FEF7DCFA204606B010BDFEF76A
:102C000067FF6FF009030393059404940294019401
:102C10000094124B124913484FF43B7208F0B6FB74
:102C20006FF00803039305940494029401940094B4
:102C30000D4B0E490E4840F22C5208F0A7FBDBE783
:102C400078030020B8BA000000BB0000C5BA00003D
:102C500075BE000072BA000098BE00001D2B000077
:102C6000101A002070150020792A0000CC1D0020C9
:102C7000081500202DE9F047114FDFF84890042691
:102C8000013EF6B2FF2E19D033B24FEA830803EBB0
:102C900043031D0104244FF00C0A0AE01AFB0451FF
:102CA0000A1D04EB08003A44394409EBC00000F067
:102CB00080F9013CE4B2FF2CF0D1E1E7BDE8F087F8
:102CC0001807002098060020F0B4124B05460F4666
:102CD0000C26302472B1614306FB00142344597A58
:102CE000187A814204BF0131197228463946F0BC76
:102CF00006F0D2BB4C4306FB004423449C7ADA7AAC
:102D0000A24204D101329A72F0BC06F02BBCF0BC96
:102D1000704700BF18070020F8B505460E461C4650
:102D20008AB1012362782078801A10F0030729D035
:102D300003B3012F39D00132D2B222703146284676
:102D400006F010FC1CE006F0FBFB0028E9D0314641
:102D5000284606F0CDFB0028E3D030230C22734335
:102D600002FB0533124A1A44937AD27A9B1A18BF8F
:102D70000123D7E70232D2B22270E368A0689847F5
:102D80000020F8BD002BF8D00132D2B2227004230B
:102D9000302212FB06320C2313FB0523044A616820
:102DA0001A44204600F008F9C8E73846F8BD00BFCD
:102DB000180700202DE9F04F00EB400389B01B01FC
:102DC0004FF00008434E049305460424CDF80480D8
:102DD000013CE4B2FF2C0BD1019B002B76D0B8F163
:102DE000000F73D142462946284606F055FB6DE098
:102DF0000DF1200B00230C274BF8043D4FF0300958
:102E000007FB04F309FB053170185A4671584068F6
:102E1000029300F0D8F8049B17FB0437F31982469D
:102E20000393BAF1000F19D130220C236A4303FB3C
:102E300004223244917AD07A88421EBFD172012294
:102E4000019230226A4303FB042333441A7A597AED
:102E500091421CBF5A724FF00108B9E7079B1F78D7
:102E60005A78BF1A07F00307012F04D1013A5A70AC
:102E70009868DA689047079A13785278DBB29A1A02
:102E800002F00302012A05930DD0029B039909FB6E
:102E9000053030440022406800F09EF8079A059BF8
:102EA000C2F804A05370029B09FB0533F0185A4680
:102EB000F158406800F087F8012F8246B1D10CB973
:102EC0000028B1D02946284606F04CFB09B0BDE8E1
:102ED000F08F00BF18070020F7B51860C31D054626
:102EE00023F00303501E0E4680B214461A800021C0
:102EF000042206FB0050FDF797FF023CA4B24FF6F8
:102F0000FF77BC4201D103B0F0BD04FB06602B1873
:102F10000422801B0DEB02012844013C0193A4B262
:102F2000FDF756FFEDE773B50568064695B1EB1D55
:102F300023F0030304221C8829460DEB0200FDF751
:102F400047FF019B013CA4B21BB1DA1D22F0030232
:102F500014803360284602B070BD70B50C68064618
:102F60000D461CB1E31D23F003031C8804222946EF
:102F70003046FDF72DFFF21D22F00302631C138083
:102F80002E6070BD02FB01007047401A80B2B0FB9A
:102F9000F2F0704710B5114401384FF6FF73013A53
:102FA00092B29A4200D110BD11F8014D00F8014FC4
:102FB000F5E710600860704713681960136858607F
:102FC000116008467047814204D00AB14B68136013
:102FD000084670470021FBE70B68834206D00AB120
:102FE000586810601A680A601846704700231B680A
:102FF000FFDE10B5421E00200139C9B2FF2900D101
:1030000010BD12F8013F002BF6D05C1E01302340AA
:10301000C0B2F8E7054B0022C3F808254FF4403250
:10302000C3F84423C3F80423704700BF00B0004036
:10303000044A1378591C1170012013B9024A106018
:1030400018467047D807002000B0004007B50F4B66
:10305000187878B90E4B01930E4B00930E4A0F4B24
:103060000F491048FEF7A4F8404080F311884FF054
:10307000040002DF0138C0B21870012320B90A4AE7
:10308000536003B05DF804FB1846FAE7D807002048
:10309000B8BA000000BB0000C5BA00000ABF0000BB
:1030A00072BA000014BF000000B00040014BD3F81A
:1030B0000405704700B0004000F5A870014B43F8CC
:1030C0002010704700B00040114BF0B50124264697
:1030D00000251A465E60C3F80405C3F80051C3F822
:1030E00004511E60D3F8001131B9D3F8041119B995
:1030F000D3F804150029F5D15460D2F80411002941
:10310000E8D1D2F80475002FE4D0C2F80415F0BD60
:1031100000E0004070B58CB00E4615460146102206
:1031200068461C46FFF736FF10220DEB02003146C1
:10313000FFF730FF6846FFF7C7FF25B1102208A947
:103140002846FFF727FF24B1102208A92046FDF7E3
:103150003FFE0CB070BD0000024B1B6803B1184766
:10316000704700BFF0090020064B1860064B102284
:10317000C3F80423054B0222C3F88021012006F086
:1031800023BF00BFF00900200010004000E100E074
:1031900008B5012006F026FF034B0022C3F8FC2FE0
:1031A0000122C3F8FC2F08BD001000400228034B89
:1031B0000CBF04220322C3F8102570470010004002
:1031C000014BC3F80C05704700100040014BC3F8D9
:1031D0000805704700100040014BC3F854057047C4
:1031E000001000400A4A0023C2F82C350123C2F81F
:1031F0003035C378C2F82435437881781B0443EA1C
:103200000163017843EA0123C2F81C35704700BF0F
:1032100000100040C2F34203022B10B50CBF4FF068
:1032200080740024D307C0F108034FEA034300F081
:103230000F0003F4702340F48070074A48BF44F441
:103240008014034341F00071234341F44031C2F83C
:103250001435C2F8181510BD00100040014BC3F81A
:103260000405704700100040014BC3F80405704787
:1032700000100040014B01225A60704700100040CE
:10328000014B01221A60704700100040034B0022DE
:10329000C3F8002201221A61704700BF00100040ED
:1032A000064B0022C3F80021C3F80421C3F808210B
:1032B000C3F80C21C3F81021704700BF0010004074
:1032C000014BD3F80001704700100040014BD3F8C8
:1032D0000C01704700100040034BD3F85005B0FAC2
:1032E00080F04009704700BF00100040044B40F2DE
:1032F0000312C3F83425C3F83805C3F83C157047EA
:1033000000100040014BD3F800047047001000404B
:1033100000487047E808002000487047EC0800208B
:10332000024B0B22C3F80022704700BF0010004080
:10333000024B0722C3F80022704700BF0010004074
:10334000024B0322C3F80022704700BF0010004068
:10335000034AD2F8003243F48873C2F8003270474F
:1033600000100040014BD3F84805704700100040A2
:10337000024B0022C3F81C21704700BF0010004020
:10338000014BD3F81C0170470010004030B50024F9
:10339000A30003F1804303F580531568C3F800567A
:1033A00001349588C3F82056082C02F10602EFD1AB
:1033B000024B40EA0120C3F8400630BD0010004037
:1033C000034AD2F8403623F0FF03C2F84036704774
:1033D00000100040034B0022C3F81421C3F8182149
:1033E000704700BF00100040014BD3F81401704734
:1033F00000100040044BC3F86005D3F8002242F0EF
:103400004002C3F80022704700100040054B4FF403
:103410008022C3F8482303F5A033FF22C3F8082510
:10342000704700BF00B00040014BC3F8440570472F
:1034300000100040F0B5A2F57423234CA3F51073DF
:10344000A34288BF02F1E872204C214B88BF02F5ED
:10345000D4324FF0000688BF02F5A5724FF0010587
:10346000B2FBF3F24FF00403E560C4F80465C4F85E
:103470001035184B88BF01F1FF310227C4F80875D9
:10348000C4F84025C4F84061C3F848154FF48021C2
:10349000C3F84413C3F848610F4903F5A033C3F8D8
:1034A0001815A1F540510839C3F81C45C3F8047537
:1034B000C3F8101530B10949C3F814151046C3F804
:1034C0000455F0BD0649F7E7BFBDF07F008000401E
:1034D00040420F0000B0004048B1004000100040E2
:1034E00004100040024B01225A601A61704700BF6D
:1034F000008000400E4B0022C3F84805C3F8482165
:1035000003F5B8330B4AC3F8302502F5DE424432E6
:10351000C3F8342502F58072C3F83825A2F5E242DB
:10352000383AC3F83C253022C3F80425704700BF61
:1035300000800040041100400B4B0C4AC3F82025CA
:1035400002F5DE424032C3F82425A2F5DE423C3AC1
:10355000C3F8282502F5DE424032C3F82C250C22A0
:10356000C3F80425704700BF00F00140001100407F
:10357000034BD3F84405D3F84035C01A704700BF59
:1035800000800040064B074AC3F8482502F5DE429A
:103590003C32C3F84C258022C3F80425704700BF95
:1035A00000F001400C110040014BD3F84805704772
:1035B00000800040154B10B500220224C3F80025FE
:1035C000C3F80045124CC3F80445C3F80805114878
:1035D000C3F80C05C3F810150F49C3F81415C3F848
:1035E00000220E49C3F80021C3F80421C3F80821C2
:1035F0000B4AC2F8401501F55F41C2F8441540215D
:10360000C2F8041501221A6010BD00BF00F000408E
:1036100001000001EC080020DC070020041100403C
:1036200000F0014010B5104B00220224C3F8002521
:10363000C3F800454FF08074C3F80445C3F808058B
:10364000C3F80C1509480A49C3F81005C3F8141546
:103650000121C3F80012C3F80021C3F80421C3F804
:103660000821196010BD00BF00F00040EC080020E8
:10367000DC0700200C4B0222C3F80423D3F80421FA
:103680006AB10222C3F80823084A4FF40041C2F885
:103690008011D3F80801B0FA80F04009704720BFCC
:1036A00040BF20BFEAE700BF00F0004000E100E0BB
:1036B000014BD3F80004704700F0004010B50E4CE9
:1036C0000123C4F800350D4BC4F80405C4F80815EF
:1036D000D3F80435C4F810350023C4F8143540205D
:1036E000FFF788FE064B074AC3F840254022C3F87F
:1036F0004445C3F8042510BD00F000400010004010
:1037000000F0014028110040014BD3F8000470473D
:1037100000F00040074BD3F828213AB1064A0021B7
:10372000C2F80011C2F80411C2F808110022C3F84F
:10373000282170470010004000F00040074BD3F8EC
:10374000280148B103F56043D3F8000120B1D3F854
:103750000401003018BF0120704700BF0010004076
:10376000042907B50FD8114B0193114B0093114A4F
:10377000114B12491248FDF71BFD404080F31188A0
:103780004FF0040002DF0F4B033918600E4B01703D
:103790000122002181704170C3F80425C3F8001193
:1037A000C3F804231A6003B05DF804FBB8BA000044
:1037B00000BB0000C5BA00003FBF000072BA0000A5
:1037C00049BF0000F409002000D00040164B1A68E1
:1037D00030B50C188C42A4EB0100537806D10020C0
:1037E0000521013911F0FF0110D130BD95789D42BE
:1037F000F6D01344DB7804F8013D53781078013398
:10380000DBB2984208BF00235370E3E794789C42F0
:1038100003D1064B01221A6030BD01331478DBB2AC
:103820009C4208BF0023DCE7F409002000D00040E0
:10383000154AD2F8003170B523B3144B1968887853
:103840000D784C78431CDBB2AB4208BF0023A34287
:1038500005D1012353600023C2F8003170BD084434
:10386000D2F80865C6708B700133DBB29D4208BF89
:103870000023A3424FF0000108BF0123C2F800114A
:1038800008BF536070BD00BF00D00040F4090020A5
:10389000F0B5037E05681A460024FF2A01D10020F6
:1038A000F0BD02EBC2078A4205EB870615F82770C8
:1038B00004D0B3681C4413463A46EEE7934200D165
:1038C00007761BB203EBC3033278B06805F82320F8
:1038D0003378FF2B06D003EBC30305EB83039A6811
:1038E00002449A602044F0BD30B5551A15F4000F1B
:1038F0008468838A09D125F07F4222449A420FD9F5
:10390000D21A00238260838230BD8A1A22F07F425D
:10391000944201D9A21AF1E713441B1B9BB2002267
:103920009B1A9BB20022EDE701460120FFF7C4BBC2
:1039300001460020FFF7C0BB07B5032816D8DFE813
:1039400000F0020C112A012910D1154B0221002090
:1039500003B05DF804EBFFF7DFB9022906D1114B84
:103960000846F5E7012911D0022912D00E4B019328
:103970000E4B00930E4A0F4B0F491048FDF718FCF1
:10398000404080F311884FF0040002DF0C4B02210D
:10399000E6E70C4BE4E70229E8D10B4B0320D7E71D
:1039A000A0010020B0010020B8BA000000BB000058
:1039B000C5BA0000FBBF000072BA00000ABA0000DE
:1039C000C0010020D0010020E001002013B50C460A
:1039D000032816D8DFE800F0020C112D012910D1C0
:1039E000174B0021002002B0BDE81040FFF794B94A
:1039F000022906D1134B0121F4E7012911D0022934
:103A000013D0114B0193114B0093114A114B1249E2
:103A10001248FDF7CDFB404080F311884FF00400C1
:103A200002DF0F4B00212046DDE701210D4B084648
:103A3000D9E70229E5D10C4B01210320D3E700BFD0
:103A40005001002060010020B8BA000000BB000057
:103A5000C5BA0000E4BF000072BA00000ABA000054
:103A6000700100208001002090010020831E012BA6
:103A700007B50FD9094B0193094B0093094A0A4B2B
:103A80000A490B48FDF794FB404080F311884FF042
:103A9000040002DF03B05DF804FB00BFB8BA000009
:103AA00000BB0000C5BA0000C5BF000072BA00002C
:103AB0000ABA0000012807B512D015D3032810D088
:103AC0000A4B01930A4B00930A4A0B4B0B490C48D3
:103AD000FDF76EFB404080F311884FF0040002DFD9
:103AE000022003B05DF804FB0120FAE7B8BA000039
:103AF00000BB0000C5BA0000A6BF000072BA0000FB
:103B00000ABA00002DE9F047057F012304464377F8
:103B1000002D4AD1037EFF2B02D14577BDE8F08707
:103B2000FFF7C4FA6769267ED4F80080C71B27F028
:103B30007F47FF2E06D006EBC60608EB86018B6892
:103B4000BB4216D9A27AE37A934205D10133DBB2A4
:103B5000022B08BF0023E372E37A04EB8303012204
:103B6000DD60002363770221636A1046BDE8F047F9
:103B70001847FF1A1D448A784B7818F826609B1A5C
:103B8000DBB2012BD5D1D1F80C90013A8A70B9F192
:103B9000000FCED060698B8A4A8B2844C01A20F06F
:103BA0007F400B69096AC847C3E7BDE8F08700009A
:103BB0002DE9F04F427F91B08046002A40F0AD835E
:103BC000436907930121837A0177C07A984200F014
:103BD00088800B44DBB2022B08BF002388F80A3030
:103BE00008EB83030291D3F80CB0079B5B4423F0EE
:103BF0007F43C8F8143098F818300593D8F800308F
:103C00000493D8F804300C9398F8093003930023F8
:103C100008934FF0FF0A039B002B65D198F81830EA
:103C2000059A9B1A18BF01230693029BE3B1D8F8AB
:103C30000030DDF80C90049398F81860FF2E0CD03B
:103C400037B2049B07EBC70703EB8704A5685D4504
:103C500040F23881A5EB0B05A560069B029A0599F9
:103C6000B14218BF13460693D8F800300393D8F832
:103C700004300E9398F809300493049B002B40F015
:103C8000748198F81830059A9342089B40F03C8361
:103C900053B998F80940D8F80470013CE4B24FF0E9
:103CA0002C0BFF2C40F09182002388F81C30069BDF
:103CB0004BB198F81830FF2B40F0DB82FFF7C6F9C4
:103CC00008B9A8F81A0098F81D30002B00F02583D9
:103CD0000122D8F824301146022011B0BDE8F04F7F
:103CE00018470292934686E7039B03F1FF395FFA78
:103CF00089F30393039A0C9B03EBC2077B6806933B
:103D0000F9782C20BE788E4285D0069B3C7816FB35
:103D100000F29D18731CDBB29C4208BF0023BB70ED
:103D2000069B9A5C032AEDD9052A17D8697801EB1E
:103D3000C1030B930B98049B03EB80046378A0787A
:103D40001B1A13F0FF0309D0042A11D16A687AB94B
:103D5000AA686AB9EA6832F07F4209D100232B7061
:103D600001206B6A2862002BCAD0A96A9847C7E76E
:103D7000012B40F09D804046FFF78AFD2B78A06024
:103D8000042B064640F08680D8F814300993FFF7DC
:103D90008DF9099B0A90C31A23F07F435B449E422E
:103DA00002469CBFA28A961B62689BBF9B19A38296
:103DB000F31A00238AB1A98979B101F1FF3E1FFAF4
:103DC0008EFEA5F80CE09A422DD3DFF80C93B4F8E0
:103DD0001AC0E64549D8A4F818E0AA8809991344FE
:103DE000A360EA88A38A1344A3820A9A2046FFF7B5
:103DF0007BFD2A89E38A13449BB2E3826A8993425A
:103E00008CBF9B1A0023E382AB7B03B1E370049B5E
:103E10000B9A03F822A0637895F801A00133637030
:103E2000002028709DE7B4F81AC0E645CDD2216A7B
:103E3000A74EA8488E19864281BF01F1E87101F5AD
:103E4000D43101F5A5712162266AE1698CBF4FF07A
:103E500001094FF00009761A91440CF1FF3C2662EB
:103E6000A3EB0903A4F81AC0ADE7266AE1699948F3
:103E70000E449749711881428EBF002101214E44A2
:103E800011440CF1010C8CBF266226620B44A4F88D
:103E90001AC09CE7A37863706B7898F819209A424F
:103EA00001BFFF2388F819300023A8F81A30B7E7BC
:103EB0000221D8F824300122084698470123BE7019
:103EC0000893A8E6B8F81A309D4229BFFF235B1B70
:103ED00088F819300023A8F81A30E38AA9441BB1E6
:103EE00088F81960A8F81A300022049BA26013F821
:103EF000273088F81830D4F804E0BEF1000F30D035
:103F0000208BDFF8D0C1236AE1690B44704959184E
:103F100061459FBFA3F1E873A3F5D433A3F5A5735F
:103F2000236292BF029B23620023734410F1FF308F
:103F30001A44E8D2079BA260D8F8141003EB0902D8
:103F40002046FFF7D1FC238B63830023E370049B9F
:103F500003F827A0637801336370ABEB050BB2461F
:103F60006AE6A37863705646F7E7049B013BDBB231
:103F70000493049A0E9B03EBC20307935B780293AE
:103F8000BAF1FF0F00F083800FFA8AF303EBC3034B
:103F9000039AD14612F823A002EB83040025FF23E5
:103FA00023700FFA89F303EBC3039B000F930F9B5E
:103FB000D8F80020B8F81A0002EB030B98F8183074
:103FC000DBF8081009934FF0FF0EFF2B07D003EB2F
:103FD000C30C02EB8C07BE68B14200F29F80BBF8B5
:103FE00016600A9606EB010C1E46FF2E40F0A480D8
:103FF0000A9F2FB18142C0F0B880FF2E40F0898126
:104000000998CBF8081083428BF8003017BFBDF930
:1040100024B088F818900BEBCB0B02F82B90FF2BF9
:1040200006D003EBC30302EB83039A68511A99602D
:10403000A378013363700020BAE00299BDF808202C
:104040000131C9B22C2312FB03F30291079A07999D
:10405000526809780298814208BF0020D15C029022
:10406000032902EB030512D195F80190039909EB9E
:10407000C90401EB84046078A17888420DD0002146
:10408000D1546B6A012028620BB1A96A9847079B3B
:10409000029A9B789342D0D1EFE5EB6863602B697D
:1040A000E361AB8A2383EB8AE382AB69E360EB696C
:1040B0002361AB68A3600026A6826A68D8F8141052
:1040C0002046FFF711FC012326626683E37066E752
:1040D0005A2B17FF592B177FB6562EFE6168002901
:1040E00065D0236AE2698E4813448E4A9A18824248
:1040F0009DBFA3F1E873A3F5D433A3F5A5732362A1
:1041000098BF2362A3681944638B8CBF00220122ED
:1041100011440133A1606383564646E0FF8A891B40
:104120002FB138469E46099312F82C304DE786424F
:1041300034BF801B3846F6E737B207EBC7070D9749
:1041400002EB87070B97BF680C9767450BD20B9F55
:10415000FF8A002F7FF44CAF0C9EACEB060C0D9E3B
:1041600012F8266041E7FF2642E7F1453FF460AFD1
:10417000BEF1FF0FB2D0764637B2039B07EBC707FD
:1041800013EB870BAAD0E2789BF803309A42A5D9AB
:1041900031464046FFF77CFB9BF802308BF801303C
:1041A000039BCBF8080003F827A0B246FFE60120E6
:1041B000002D3FF4E5AE00232B706B6A2862002BC4
:1041C0003FF4DEAEA96A9847DAE607EBC4056B78E0
:1041D000EA789A4202D1013CE4B262E513FB0BF2A9
:1041E00069688B188A5C012A2FD0022A08D06B7864
:1041F0002A780133DBB29A4208BF00236B70E6E7EE
:10420000D3F804C09A689CF80010D3F80C90D8F842
:104210000000D8F814A0FF2902D0166856451DD01A
:1042200098F81810C2F800A00022FF2909D001EB6D
:10423000C10A00EB8A0EBEF81660DEF808E0A6B1EF
:1042400072448CF80010C9F8002000221A625A6AE1
:10425000002ACCD0996A186A9047C8E701EBC101DF
:10426000D9F8002010F82110DFE7724410F82A1066
:10427000DBE7059BFF2B07D1FEF718FF0446FEF78F
:10428000D7FE08B9C8F8144098F81830D8F80020BC
:1042900003EBC30302EB83030A269D68FEF706FFC8
:1042A000D8F81440031B23F07F430333AB422CBFE9
:1042B000E418641924F07F440746D8F828302046D3
:1042C0009847FEF7F3FEC01B20F07F40E41B03304D
:1042D00024F07F44A0427FF6F6AC013EDED1124BC3
:1042E0000193124B0093124A124B13491348FCF7E7
:1042F0005FFF404080F311884FF0040002DF9DF81B
:10430000103088F81C30D4E4002BF8D10123069338
:10431000BFE4B1457FF430AF8AE611B0BDE8F08F5D
:10432000592B177F5A2B17FFB8BA000000BB0000AB
:10433000C5BA00008CBF000072BA000012C00000B5
:10434000F0B5059F9DF8184018B1012828D001202C
:10435000F0BD1D4D1D4E2E621D4E6E621D4EAE6295
:10436000194D2C2606FB00FC05EB0C0E45F80C2025
:104370008EF8081007998EF80930CEF80470013BCA
:10438000DBB2FF2B14D1002CE1D12C2202FB005018
:1043900003764376448344618472C4722046F0BD40
:1043A000094D0D4EEE640D4E2E650D4E6E65D7E730
:1043B0001AB207EBC20ECEF8041017F83220A41A76
:1043C00002FB0611E4B2DAE7F8090020B53A000072
:1043D000CD390000313900006D3A00003939000054
:1043E00029390000054A2C2303FB0020436A1BB136
:1043F0000122114600201847704700BFF80900202D
:10440000F8B5224D2C2404FB00500FFA81FCD0F8A3
:1044100004E00EEBCC071EF83CE0FE78751CEDB214
:10442000AE4598BF002597F801E0AE452BD0D7F8F0
:1044300004E016FB04F60EEB06044FF0030C0EF836
:1044400006C06360069BA360079BE360089B236133
:10445000BDF82830E382BDF82430A3820B9BA36112
:104460000C9BE3610D9B636202260E9B6270A3624C
:104470002662FD70456A036A084698470022314665
:10448000A847206AF8BD0120F8BD00BFF809002048
:10449000F8B5214D2C2404FB00500FFA81FCD0F814
:1044A00004E00EEBCC071EF83CE0FE78751CEDB284
:1044B000AE4598BF002597F801E0AE452AD0D7F861
:1044C00004E016FB04F60EEB06044FF0040C0EF8A5
:1044D00006C0A380BDF81830E380BDF81C302381EE
:1044E000BDF820306381BDF82430A3819DF82830C9
:1044F000A3730B9B636202260C9B6270A36226620D
:10450000FD70456A036A0846984700223146A8476D
:10451000206AF8BD0120F8BDF8090020F8B5194C53
:104520002C2505FB00400FFA81FCD0F804E00EEBCF
:10453000CC071EF83CE0FE78741CE4B2A64598BF98
:10454000002497F801E0A64519D0D7F804E016FB3F
:1045500005F60EEB06054FF0050C0EF806C06B6273
:104560000226069B6A70AB622E62FC70446A036A84
:104570000846984700223146A047286AF8BD012026
:10458000F8BD00BFF80900202DE9F0411C4D2C2496
:1045900004FB00500FFA81FCD0F804E00EEBCC07CE
:1045A0001EF83CE0FE78751CEDB2AE4598BF0025C4
:1045B00097F801E0AE4520D0D7F804E016FB04F6EA
:1045C0000EEB06044FF002080EF80680A360069B6F
:1045D000E360079B6362FF26089B62606670A362CC
:1045E000C4F82080FD70456A036A08469847002297
:1045F0004146A847206ABDE8F0810120BDE8F0816E
:10460000F8090020F8B5194C2C2505FB00400FFADD
:1046100081FCD0F804E00EEBCC071EF83CE0FE78FD
:10462000741CE4B2A64598BF002497F801E0A645A3
:1046300019D0D7F804E016FB05F60EEB06054FF08F
:10464000010C0EF806C0FF266E7002266A62AB628D
:104650002E62FC70446A036A08469847002231467D
:10466000A047286AF8BD0120F8BD00BFF809002066
:10467000074A10B52C2303FB0020446A036A08464E
:104680009847234600220221BDE81040184700BF8A
:10469000F8090020FEF70ABD401A20F07F4070475D
:1046A00070B50C4D06460C460CB9002070BD4FF09D
:1046B000FF31284605F04EFF20463146FFF786F8C9
:1046C0000446284605F0AAFF002CEED020BF40BFCC
:1046D00020BFE9E78C03002020BF40BF20BF704708
:1046E0000860704718B90B6843F000430B607047CF
:1046F00018B90B6823F000430B60704770B502FBDC
:10470000011102789DF810500A44252192FBF1F422
:1047100001FB1424E1B2CA0801709A5C04F007049A
:10472000224112F0010209D1B1FBF5F005FB101096
:10473000C0B25D1E04339D4202D11146084670BDD1
:1047400015F8016F00241119082CC9B201D10A46CD
:10475000F1E716F0010F03D00028EFD00138C0B206
:1047600076080134EFE7000010B50E4A92F84632A1
:1047700092F845128B4238BF92F8444292F84512A3
:1047800038BF1B195B1ADBB298429FBFD2F8403288
:1047900092F8451253F82100012394BF03710020C1
:1047A00010BD00BFA00A002070B590F8581090F816
:1047B00059308B423FD190F8343013F0010511D0BD
:1047C00090F88C309B0738D590F88D30082B34D971
:1047D000B0F88E304FF6FF7293422ED1B0F8902091
:1047E0009A422AD1C48C828CA0F85E40848DA0F8B5
:1047F0005C20002354437D2201269D4202FB04F2EB
:104800004FF47A7492FBF4F2A0F8602090F88520BF
:1048100080F884600CBF3446022464F3020266F31D
:10482000C4020139C36780F8852080F8591080F8E8
:104830005A60184670BD012070BD022070BD000096
:104840002DE9F84F0C78944281460F4690463DD0B2
:104850001F4ED6F8743233F83430038000254FF001
:10486000020B06F51A7A22B2D6F87402B9F800E003
:1048700000EBC20130F83220964520D1486801286B
:1048800020F003030AD9F3B1021D1CD04279D2B142
:10489000027902F00302013A012A14D801221544D8
:1048A0004A60EDB213B15146FEF757FB013496F85A
:1048B0007822E4B2A24208BF00244445D3D13C7020
:1048C0002846BDE8F88FC1F804B0EBE70025F7E70C
:1048D000A00A002010B5094B93F81C22824204461E
:1048E00009D90246FC21D3F81402FEF74BFB10B1A4
:1048F000038CA34200D0002010BD00BFA00A0020FE
:104900002DE9F04186B0022305280546884602932A
:104910000CD0062824D029D9073880B2FFF7DAFF57
:10492000002800F0EC8090E8C00004E0754BD3F85C
:10493000C460D3F8C870734CA37B03F0FF00F3B1DD
:10494000714B0193714B0093714A724B72497348DA
:10495000FCF72EFC404080F311884FF0040002DF8A
:10496000684BD3F8AC61D3F8B071E4E7664B0193C0
:10497000664B0093674B664A67496948E8E702ABB4
:1049800000932A46674BA5730321FFF7C7FD022852
:1049900028D0029B002B40F0A380237B9D4203D0B4
:1049A000637B9D4240F0988006AB022243F80C2DB9
:1049B0000022009303215B4B1046FFF7AFFD022856
:1049C0001ED1012211460320FEF77EF9039B022B24
:1049D00016D14D4B01934D4B00934D4A524B4E49CE
:1049E0005248B5E7637B9D4204D101221146032062
:1049F000FEF76AF9029B022BCBD1FFF76DFEF9E7B8
:104A000003980222002834D106AB032143F8082D75
:104A100001220093434BFFF781FD022807D10122B9
:104A200011460320FEF750F9049B022BD1D0049AC3
:104A30008AB9B7421BD93E4B11460320FEF76CF9E9
:104A4000002849D0304B0193304B0093304A364B0D
:104A5000314938487CE7049B012B4AD1002211469A
:104A6000334B0320FEF758F902460028EAD1324BB7
:104A7000E2E7039D012D3CD106AB032143F8042D51
:104A8000002000934246274BFFF748FD022807D13C
:104A90002A4629460320FEF717F9059B022B98D0DA
:104AA000059B5BB1059B012B08D0174B0193174B5E
:104AB0000093174A1C4B1849204849E7E37B5BB138
:104AC0001F4B04229A60002211460320FEF724F9AE
:104AD0000028B7D1E37B4BB9A37B0BB90123029329
:104AE0000023A373029806B0BDE8F081FFF7F4FD40
:104AF000F0E7054B0193054B00930B4B3BE701207F
:104B0000F1E700BFA00A0020B8BA000000BB000017
:104B1000C5BA00002CC4000072BA000064CB0000CB
:104B20000ABA0000E146000018C400009CCB000057
:104B300010020020C9CB000090020020F2CB000040
:104B40003002002013B51F4B04461A7811B3002A17
:104B500035D101280FD01C4B01931C4B00931C4AEC
:104B60001C4B1D491D48FCF723FB404080F3118876
:104B70004FF0040002DF1870194B1146FEF7CCF815
:104B8000E8B1114B0193114B0093114A114B12499B
:104B90001448E8E79AB1197078B1012804D1124B92
:104BA000002211462046E9E7074B0193074B00938B
:104BB000074A084B08490D48D5E70D4BF0E702B00E
:104BC00010BD00BF840F0020B8BA000000BB000079
:104BD000C5BA0000DBC1000072BA0000CEC90000F7
:104BE00060020020C9CB0000800200200ABA000049
:104BF00070020020F8B590F8A430D0F8E8500446D0
:104C000018060E4605F104021ED4EDB119074CD565
:104C1000002A4AD06979002947D0297901F0030197
:104C2000032911D194F8341011F0010F03F0400161
:104C3000EB792CD131BB022B37D0112B04D82F4963
:104C400021FA03F3DB0730D494F8A43043F0800357
:104C500084F8A430FEF75CFB0378012262F30103C1
:104C600000224270D4F8E8200370DBB2D2B143F0E6
:104C70001003037003786FF34713037000238370EE
:104C80003060F8BD991E01290FD90B2BD4E729B943
:104C9000022B0AD0112BD7D81949D1E7022B04D007
:104CA000042BF6E762F30413E3E794F8F93094F881
:104CB000F810D01811B9417884F8F81023B1D15CFC
:104CC000012767F30101D15494F8F810C91AC9B249
:104CD0004170D45C1B296FF30414D45405D91B21F3
:104CE0004170D15C41F01001D15429680029C1D034
:104CF000D15C41F01001D154BCE700BF402002005C
:104D000060200200000000002DE9F04F8FB08146C6
:104D1000069303680991002B904638DA816842684F
:104D200023F0004391422CBF5B1A9B1A0024079387
:104D3000FF238DF82930ADF82A400B940C9405938D
:104D40009A46A3462546089402230D930DAB029381
:104D50007B4B01930CAB00930DF129020BAB0121AE
:104D60000020FFF711FC022817D00D9BCBB1754B2B
:104D70000193754B0093754A754B76497648FCF75D
:104D800017FA404080F311884FF0040002DF00233F
:104D9000CCE701210020FFF76BFC0D9B022BF8D024
:104DA000E3E79DF82920FF2A60D0BAF1FF0F0CD06D
:104DB0000B9B0899994208D0624B0193624B009378
:104DC000624A634B63496548D9E7042A49D9062AF0
:104DD00040F28C80059BFF2B48D1614B073A92B281
:104DE000FC21D3F81402FEF7CDF88145074638D0F0
:104DF000099B1BB990F83430DB0732D4079B0C9E1B
:104E00001E443B68002B08DABA68796823F0004337
:104E10008A422CBFB6187618F61AD8F800309E428F
:104E200017D99D4238BF1D460BF1640A189B1B78A9
:104E3000A34207D929463046FFF72EFCFB685344AE
:104E400098422ED2BDF82A30069AC8F800509342F4
:104E50000CD20B9B0893FB689DF829A003F1640B0F
:104E60003546189B1B78A3423FF66EAF9DF829305C
:104E7000FF2B11D1D8F80030DFF8E8902EA7D7E942
:104E800000679D4238BF1D464FF0070A189B1B78EC
:104E9000A3422DD8C8F80050189B1C700FB0BDE875
:104EA000F08F304A05EB0B03A3FB0201072202FB44
:104EB000031121A3D3E90023FBF7ACF940F2E2434D
:104EC000B0FBF3F0069B80B29842ADF82A000BD2FB
:104ED000199B022203EB44000DF12A010134FBF778
:104EE00077FFE4B22835A1E70025ABE70592B8E7E4
:104EF00005EB0B03A3FB09010AFB031132463B46FA
:104F0000FBF788F940F2E243B0FBF3F0069B80B276
:104F10008342ADF82A000BD9199B022203EB44000F
:104F20000DF12A010134FBF753FFE4B22835ADE758
:104F30000025AFE7AFF3008000CA9A3B00000000F5
:104F4000E1460000B8BA000000BB0000C5BA00008E
:104F500036C2000072BA000032CC00000ABA00006B
:104F6000A00A00208D49FD1A2DE9F041044688B0C1
:104F7000B0F8662034480623A2FB00018DF80D30FE
:104F800040F2231303FB02112DA3D3E90023FBF707
:104F900041F908AA0DF10D0105AE42F8100DB4F863
:104FA0005C300091019601212046FFF7ADFE04F12F
:104FB000660504F172074FF6FF78022229460DF1CB
:104FC0000E00FBF705FF9DF80D00BDF80E20002335
:104FD000D9B288421ED80235AF42EED194F858308B
:104FE00084F85930194B0022C3F88C22D4F8803051
:104FF00013F8052C42F0030203F8052C032203F8F2
:10500000042C112203F8022C0F2203F8012C202279
:105010001A7012E0424503D036F81310914201D0C5
:105020000133D5E740F2E2435343E36702220DF137
:105030000E01D4F88000FBF7CBFE08B0BDE8F0818C
:105040008D49FD1A070000000054CE09A00A002077
:105050001FB50023039306238DF80B3090F83430EE
:10506000DB0742BF0246436D42F8783FD0F880101C
:1050700001910DF10B01009158BF03AAB0F85C300B
:105080000021FFF741FE05B05DF804FB00000000C1
:105090002DE9F04F8BB00024FF25DFF834B18DF8F7
:1050A0001F508046894692461F461C60089426463B
:1050B0000AAB022243F8042D02933D4B019308AB47
:1050C00000930DF11F02534641460020FFF75CFAA2
:1050D000022815D0099BBBB1364B0193364B009388
:1050E000364A374B37493848FCF762F8404080F37E
:1050F00011884FF0040002DF41460020FFF7B8FAA4
:10510000099B022BF8D0E5E79DF81F20FF2A45D028
:10511000062ACDD9073A92B2FC21DBF81402FDF73A
:1051200031FF03460028C3D090F83420D207BFD403
:10513000D0F800E0089ABEF1000F09DA41688068F3
:105140002EF0004E88422CBF12185218A2EB0E020D
:10515000FF2D05D1DC689DF81F5027341646A7E7C0
:105160003146104605930492FFF796FA09F10201C1
:1051700021448842049A059BECD914483444A4FB8A
:105180000001072303FB041107A3D3E90023FBF766
:1051900041F8203038600BB0BDE8F08FFF2DECD126
:1051A000F9E700BFAFF3008000CA9A3B000000009F
:1051B000E1460000B8BA000000BB0000C5BA00001C
:1051C00017C2000072BA000032CC00008D49FD1AEF
:1051D000A00A00200000000073B5164602AA05468A
:1051E00042F8046D012027311C46FFF751FF01985A
:1051F000864211D03146FFF74FFA02461048072386
:10520000A2FB000103FB02110BA3D3E90023FBF770
:1052100001F82368184420602368002B05DB40F266
:10522000E24068432368984201D302B070BD1B1A64
:105230002360F7E7AFF3008000CA9A3B000000004C
:105240008D49FD1A13B500F17C030446426FC16815
:10525000808CFFF7C1FF02A9E36FD4F8800040F211
:10526000E242B3FBF2F3022221F8023DFBF7B0FD6C
:1052700002B010BD13B51F4A92F8453292F846129B
:1052800099420FD11C4B01931C4B00931C4A1D4BA0
:105290001D491E48FBF78CFF404080F311884FF0FA
:1052A000040002DF92F84512D2F8403253F8210090
:1052B00092F87C320168037092F8453292F84442C9
:1052C0000133DBB29C4208BF002382F8453202F56D
:1052D0001572FDF771FE40B9074B0193074B009320
:1052E000074A084B08490A48D4E702B0BDE8104015
:1052F00004F068B9A00A0020B8BA000000BB0000A2
:10530000C5BA000030C3000072BA00004CCA0000E9
:105310009FCA000037B541F2D6230021009308460A
:10532000254B0522FFF7FAF830F002010FD0234B8E
:105330000193234B0093234A234B24492448FBF732
:1053400037FF404080F311884FF0040002DF4FF434
:10535000975300930122184B0846FFF7DFF830F00F
:105360000202E4D141F2E52300931146124B1046AC
:10537000FFF7D4F830F00205D9D10120FFF7F4F996
:10538000044640B90D4B01930D4B00930D4A0E4B53
:105390000E491048D3E74FF6FF73C3800323037110
:1053A000182229460B30FBF73FFD3C23E37203B084
:1053B000BDE83040FFF75EBF49540000B8BA0000B6
:1053C00000BB0000C5BA000096C2000072BA00001F
:1053D0009EC40000ECC4000070B506460320FFF731
:1053E000C3F9A0B14FF6FF73447AC380022303715F
:1053F00000F108051C4446B1FDF7B4FF00F07F0042
:105400002855FFF737FF002070BD7F20F8E7012007
:1054100070BD00000B4A92F8843292F885129942CE
:105420000ED192F8843202EB4303A3F87E0292F885
:1054300084320133DBB2032B08BF002382F88432AD
:10544000704700BFA00A002007B578B1094B01934F
:10545000094B0093094A0A4B0A490B48FBF7A8FE7F
:10546000404080F311884FF0040002DF03B05DF884
:1054700004FB00BFB8BA000000BB0000C5BA0000C2
:1054800028C1000072BA0000CBCC0000012807B58B
:1054900005D10C4B9A7B052A04D100229A7303B0E4
:1054A0005DF804FB084B0193084B0093084A094B35
:1054B00009490A48FBF77CFE404080F311884FF011
:1054C000040002DFA00A0020B8BA000000BB000000
:1054D000C5BA00003EC1000072BA00000ABA00005E
:1054E000012807B505D10C4B9A7B062A04D100226E
:1054F0009A7303B05DF804FB084B0193084B0093CB
:10550000084A094B09490A48FBF752FE404080F31C
:1055100011884FF0040002DFA00A0020B8BA000092
:1055200000BB0000C5BA000055C1000072BA0000FF
:105530000ABA000007B598B10B4B9B7B052B0FD027
:105540000A4B01930A4B00930A4A0B4B0B490C4838
:10555000FBF72EFE404080F311884FF0040002DF7D
:1055600003B05DF804FB00BFA00A0020B8BA000039
:1055700000BB0000C5BA00006CC1000072BA000098
:10558000F8CC000007B5A0B10B4B9B7BC9B2994288
:105590000FD00A4B01930A4B00930A4A0A4B0B495E
:1055A0000B48FBF705FE404080F311884FF00400E4
:1055B00002DF03B05DF804FBA00A0020B8BA0000C7
:1055C00000BB0000C5BA000085C1000072BA00002F
:1055D00047CD0000044B1B7C23B10121002208466B
:1055E000FDF772BB704700BFA00A002007B50E4A46
:1055F00093601346002211461046FDF78DFB78B1EB
:105600000A4B01930A4B00930A4A0B4B0B490C4877
:10561000FBF7CEFD404080F311884FF0040002DF1D
:1056200003B05DF804FB00BF20020020B8BA000000
:1056300000BB0000C5BA000063C2000072BA0000DF
:10564000C9CB000007B500220C4B11461046FDF7F0
:1056500063FB78B10A4B01930A4B00930A4A0B4B48
:105660000B490C48FBF7A4FD404080F311884FF034
:10567000040002DF03B05DF804FB00BFF00100206E
:10568000B8BA000000BB0000C5BA0000B4C10000F9
:1056900072BA0000C9CB000007B500220C4B1146BE
:1056A0001046FDF739FB78B10A4B01930A4B009382
:1056B0000A4A0B4B0B490C48FBF77AFD404080F33C
:1056C00011884FF0040002DF03B05DF804FB00BF57
:1056D00050020020B8BA000000BB0000C5BA0000AC
:1056E000D0C1000072BA0000C9CB000007B5124A51
:1056F000137840B1591C1170DBB9012003B05DF87B
:1057000004EB03F05DBF7BB90C4B01930C4B009392
:105710000C4A0D4B0D490E48FBF74AFD404080F303
:1057200011884FF0040002DF013BDBB21370002B45
:10573000E4D003B05DF804FB200F0020B8BA0000ED
:1057400000BB0000C5BA0000A0C1000072BA000092
:1057500053C900000020FFF7C9BF000007B5C0B261
:10576000031F012B0FD9114B0193114B0093114AC9
:10577000114B12491248FBF71BFD404080F3118882
:105780004FF0040002DF0F4A137C43B1043B012BAE
:1057900005D9107403B05DF804EBFDF777BDFDF794
:1057A0009BFD0028F6D003B05DF804FBB8BA0000FA
:1057B00000BB0000C5BA000051C2000072BA000070
:1057C0007DC90000A00A002038B505460C4600211E
:1057D0000846FDF7EBFC95F8A430DB064FF001021C
:1057E0000CD51F210820FDF715FD214605F1A50068
:1057F000FDF7E0FEBDE83840FDF730BD08201B2175
:10580000FDF708FD2046F5E737B5184A92F87C32D7
:1058100092F878420133DBB29C4208BF002392F831
:105820007B429C420FD1124B0193124B0093124AC0
:10583000124B13491348FBF7BBFC404080F311881F
:105840004FF0040002DF92F87C52D2F8744224F840
:10585000350092F87C0204EBC004616082F87C326F
:1058600003B0BDE8304003F0ADBE00BFA00A002089
:10587000B8BA000000BB0000C5BA000042C3000077
:1058800072BA0000C5CA00002DE9F843244C064650
:1058900000272EB194F8793294F87A229A4201D1F5
:1058A000BDE8F88394F87982D4F87092D4F81402A1
:1058B00039F8382009EBC803FC215D682F60FDF73B
:1058C00061FB034639F838001A8C82421FD1D3F8A5
:1058D000F02042B9D3F8E820C3F8F0501AB9C3F861
:1058E000E850C3F8F420D3F8F42002B11560C3F8EF
:1058F000F45094F8793294F878220133DBB29A426A
:1059000008BF0023013E84F87932F6B2C1E72B7953
:1059100067F301032B712946FFF776FFE9E700BF24
:10592000A00A00202DE9F04F14681D688DB0002CEE
:1059300080460B9117469A469DF85C9003DA169CB8
:10594000AC4238BF2C46AC42584E25D941F2C70371
:105950000893574B05930021631B0093079643461A
:105960000691049103910291019101220846FEF7EC
:1059700047FD30F0020335D04E4B01934E4B009360
:105980004E4A4F4B4F495048FBF712FC404080F3C2
:1059900011884FF0040002DF1DD200231A46194679
:1059A0001846FFF74FFE41F2DC03002108932C1B41
:1059B000464B059307964346069104910391029145
:1059C0000191009401220846FEF71AFD30F002030F
:1059D000D2D12C460BE000231A4619461846FFF791
:1059E00031FE00231A4619461846FFF755FEDFF828
:1059F000E8B00B9BCBF8083041F2F4030893199BF5
:105A000006930022189B059304920392029201923E
:105A100011461046079600944346FEF7F1FC30F01D
:105A20000202A9D1052311461046FFF7DFFDDBF87E
:105A300088329D4222D03A68CAF8003022F00042F3
:105A40009A4238BF1A463B68002BB8BF23F0004388
:105A500041F22111B8BF3B6092B2A3B2069100217E
:105A60000293019200920596049103914A460846DA
:105A7000FEF70EFD30F002037FF47EAFFF20FFF74C
:105A800003FF134B012211460020C3F80890FDF7D5
:105A900043F940B1074B0193074B0093074A084B6A
:105AA00008490C4870E70DB0BDE8F08F495400007C
:105AB00045560000B8BA000000BB0000C5BA00009F
:105AC0006EC2000072BA00009EC400009956000029
:105AD000A0020020C9CB0000A00A00201FB5094A7F
:105AE0000523002413730394074C02940193D2F806
:105AF000CC30009302F1C803C432FFF713FF04B0A7
:105B000010BD00BFA00A00205161000073B5012242
:105B1000044611460020FDF7D7F894F82020002114
:105B200041F6E6330732009308463D4BD2B2FEF70A
:105B3000F5FC30F002010FD03A4B01933A4B009341
:105B40003A4A3B4B3B493C48FBF732FB404080F331
:105B500011884FF0040002DF384B1A7C052A1D46DD
:105B60001AD11A7B238C07339A4215D141F6F233AE
:105B7000009301222A4B0846FEF7D0FC30F00202C7
:105B8000DAD141F6F93300931146254B1046FEF762
:105B9000C5FC30F00203CFD1D4F8E810D4F8EC30D3
:105BA000994203D0D4F8F030994201D1244E12E04A
:105BB0000B796FF301030B710B68C4F8E830208C8C
:105BC000FFF722FEE8E70368C4F8E830C4F8EC30D9
:105BD0003146FDF7C2F9D4F8E80018B1D4F8F03036
:105BE0009842F0D10023C4F8EC30D4F8E81051B951
:105BF0004FF6FF732384D5F88C329C4208BFC5F85A
:105C00008C1202B070BD0B796FF301030B710B683E
:105C1000C4F8E830C4F8F030208CFFF7F5FDE4E775
:105C200049540000B8BA000000BB0000C5BA00002B
:105C300056C3000072BA00009EC40000A00A0020F3
:105C4000000D002038B505460C4600210846FDF73A
:105C5000ADFA95F8A4309B064FF001020CD51F2138
:105C60000820FDF7D7FA214605F1C600FDF7DAFC5A
:105C7000BDE83840FDF7F8BA08201B21FDF7CAFA45
:105C80002046F5E7262813B504460CD027280CD06B
:105C900025280CD10220FDF799FA204602B0BDE874
:105CA0001040FDF799BA1A20F5E75020F3E70A28CB
:105CB00002D802304000EEE7272801D80330F9E788
:105CC000074B0193074B0093074A084B08490948C3
:105CD000FBF76EFA404080F311884FF0040002DFBA
:105CE000B8BA000000BB0000C5BA000083C20000C3
:105CF00072BA00000ABA000038B51C4C94F855314D
:105D000094F856219A4206D00133DBB2022B08BF29
:105D1000002384F8553194F85501272303FB0040F4
:105D200000F20710FDF7A0FA9620FDF77DFBFDF7C6
:105D3000F7FA94F8D430C3F3C202D3B21946002064
:105D400011F0010F00F101050DD0013B134094F853
:105D5000D420C0B263F3C50284F8D4202530BDE856
:105D60003840FFF78FBF49082846E9E7A00A00201E
:105D700013B503460A46D3F89810983079B9184BF2
:105D80000193184B0093184A184B19491948FBF70F
:105D90000FFA404080F311884FF0040002DF1C8CA2
:105DA000A3F89E4083F8A0200424134A83F89C4063
:105DB00092F87C4283F8984002F51572FDF7FCF8E2
:105DC00040B9074B0193074B0093074A074B08491B
:105DD0000A48DCE702B0BDE8104003F0F3BB00BFA7
:105DE000B8BA000000BB0000C5BA000069C30000DB
:105DF00072BA000088CC0000A00A00209FCA0000F0
:105E000030B50468002C89B027DA436885680690AD
:105E10009D4224F0004434BFE41A641B104B0593E8
:105E2000A4B20023049303930293184601940094B0
:105E3000FEF72EFB30F002030FD00A4B01930A4B02
:105E400000930A4A0A4B0B490B48FBF7B1F9404053
:105E500080F311884FF0040002DF09B030BD00BFAD
:105E6000F1460000B8BA000000BB0000C5BA00004F
:105E7000EEC1000072BA00009EC4000000000000E5
:105E800030B58DB002230993FF238DF8233009AB81
:105E90000293814B01930AAB009305460BAB0020A4
:105EA0000DF1230201210A90FEF76EFB022815D0A6
:105EB000099CBCB1794B0193794B0093794A7A4B99
:105EC0007A497B48FBF774F9404080F311884FF022
:105ED000040002DF01210020FEF7CAFB099B022B10
:105EE000F8D0E5E79DF82330FF2B00F0AD800A9B4A
:105EF000A82B00F2A98001210846FEF723FE9DF899
:105F00002320042A65D9062AEDB264D9694B073AE1
:105F100092B2FC21D3F81402FDF734F804468368EA
:105F20004168994238BF19460368002B5ADA0A9A29
:105F300023F000431144CB1A0A93062D49D95D4B37
:105F4000EA1FD3F8140292B2FC21FDF71BF8036894
:105F5000002B05460ADA0A9A816823F000431344AD
:105F6000426891422CBF5B1A9B1A0A938CB3AB8C8C
:105F7000A28C9A422DD1504892B2A2FB000140F26D
:105F8000231303FB021142A3D3E90023FAF742F9DA
:105F90000A9B20F07F400022984241D302B10A932D
:105FA00095F8342012F0010F94F834203BD0D0073C
:105FB0000FD4EA683B329A420BD92846FEF7F4FB2D
:105FC000022806D194F88C30990702D52046FEF7B6
:105FD000EBFB0DB030BD394800F1E803052A18BFCE
:105FE00018469CE79942A8D25B1A9BB206903449A6
:105FF0000591002002939DF82320049003900190C6
:1060000000900121FEF744FA30F0020395D0234BB3
:106010000193234B0093234A234B2449294851E7FA
:106020001B1A0122B8E7D207D3D5EA683B329A425D
:10603000CFD92046FEF7B8FB0228CAD195F88C309C
:106040009B07C6D52846C2E700210120FEF77AFD4E
:106050009DF82320531FDBB2F92BBAD8062A0DD99D
:10606000144B073A92B2FC21D3F81402FCF78AFFD2
:106070009DF823200121FFF7C3FEAAE70F4800F196
:10608000E803052A18BF1846F2E700BFAFF3008007
:106090008D49FD1A07000000E1460000B8BA000073
:1060A00000BB0000C5BA000001C2000072BA0000C7
:1060B00032CC0000A00A00200054CE09640B00205E
:1060C000E5460000FEC9000070B514460E460546C0
:1060D000FEF7E0FA2146FEF7DFFAC41C092C0FD9BF
:1060E00000210846FEF72EFD324600212846FFF724
:1060F00087FEAB681C44262C00D8AC60012070BD24
:10610000002070BD13B502AC0E4B44F8043DFDF702
:106110003FF80020FDF754F80B48FDF725F8002163
:106120000846FDF743F82046FDF75CF800222521DC
:106130000820FDF76FF8054940F25B60FDF7D6F8DF
:1061400002B010BDD6BE898E1173000055555500A2
:10615000354B37B5DA7B054602F0FF011C467AB1B4
:10616000324B0193324B0093324A334B334934481C
:10617000FBF71EF8404080F311884FF0040002DF67
:106180001B7BDBB2052B08D0284B0193284B0093D7
:10619000284A294B29492B48EAE70122E2730222C7
:1061A0002173227463736060FFF7ACFF94F8D4200E
:1061B000134662F3C50384F8D430FFF79DFD94F8CD
:1061C000D43013F0C00F07D004F1D70294F8D610E2
:1061D00094F8D500FDF7DAF8A26805F1090101206D
:1061E000FDF728F9FDF7CEF92A4605211648FFF7F5
:1061F0006BFF034630B10423237403B0BDE8304085
:10620000FDF744B8114A0146FEF7FCF930F00203ED
:1062100008D0064B0193064B0093064A064B0749EC
:106220000B48A5E703B030BDA00A0020B8BA0000B3
:1062300000BB0000C5BA00008CC2000072BA0000AA
:106240006FC500005FC40000640B0020D55500003E
:106250009EC400002DE9F843214D95F8464295F87B
:10626000443295F858920134E4B2A34208BF0024A6
:1062700005F5137705F50D78B9F1000F03D095F802
:1062800045329C4201D1BDE8F8833846FCF74BFE0D
:1062900006460028F7D04046FCF745FE28B93046B0
:1062A0001049BDE8F843FCF758BE066095F8462251
:1062B000D5F8403243F8220085F8464295F844323A
:1062C0000134E4B2A34208BF002495F8583209F122
:1062D000FF39013B85F858325FFA89F9CCE700BFF6
:1062E000A00A0020EC0C002013B5334C94F81C22BB
:1062F000002A40D004F50673FC21D4F81402FCF700
:10630000EBFD2E4B94F83E22B4F83C12D4F8300248
:10631000FCF7E2FD94F8441294F81C22284BD4F8C0
:1063200048020A440821FCF7D7FD264BD4F85C024A
:1063300002222421FCF7D0FD94F87822D4F86402DC
:10634000214BB4F86C12013A92B2FCF7C5FD1C481F
:10635000FCF7E9FD90B91D4B01931D4B00931D4ABD
:106360001D4B1E491E48FAF723FF404080F3118859
:106370004FF0040002DFC4F81822C2E7194A111FC7
:10638000FCF717FE94F8D43043F0070384F8D430B8
:10639000FF2384F8263284F8273284F8283284F8E0
:1063A00029321F2384F82A32252384F82B3202B0A5
:1063B000BDE81040FFF74EBFA00A0020D40C00201B
:1063C000EC0C0020000D0020080D0020B8BA0000E1
:1063D00000BB0000C5BA000035C0000072BA000062
:1063E0009FCA0000F40C0020024B1868436800218B
:1063F0001B681847A00A0020024B18684368002158
:106400005B681847A00A002010B50446FCF7C0FEE0
:106410000020FCF7D5FE0A48FCF7A6FE04F11000A8
:10642000FCF7E0FE637DA17D1B0243EA0143217D71
:1064300040F25B601943BDE81040FCF757BF00BF56
:1064400011730000F0B54A4D1C46EB7B85B0064643
:1064500003F0FF027BB1474B0193474B0093474A40
:10646000474B48494848FAF7A3FE404080F311885B
:106470004FF0040002DF2B7B218CDBB207318B4213
:1064800008D03C4B01933C4B00933C4A3C4B3D496C
:106490003E48E8E785F8242285F82522DBB2042768
:1064A000EF732A736B73238DC5F820420220638536
:1064B000228528746E60FFF7E7F903A92046FEF7EE
:1064C00099FB039994F8A4200B7862F3C303C2F3F9
:1064D000400262F382030B702046FFF795FF039999
:1064E0002046FFF7AFFB9620FCF79EFFFCF718FF56
:1064F000237F5A0608D51F4B01931F4B00931F4A59
:106500001F4B20492248AEE703F03F03628DA17F75
:10651000009304F11F0004F11703FEF7EFF8FFF7F3
:10652000B1FBAA6806F109010120FCF783FFFDF722
:1065300029F894F8201007313246C9B22046FFF7F7
:10654000C3FD034620B12F74FCF7A0FE05B0F0BDDB
:10655000104A0146FEF756F830F00203F6D0054B1C
:106560000193054B0093054A054B06490A487AE713
:10657000A00A0020B8BA000000BB0000C5BA0000A5
:1065800023C3000072BA00006FC500001FC50000E1
:106590000ABA0000D55500009EC40000F7B5544D5E
:1065A0001C46EB7B064603F0FF022F467BB1514BA6
:1065B0000193514B0093514A514B52495248FAF7BB
:1065C000F7FD404080F311884FF0040002DF2B7B81
:1065D000218CDBB207318B4208D0464B0193464BEE
:1065E0000093464A464B47494848E8E785F8242245
:1065F00085F825220321DBB2E9732A736B73238D9F
:10660000C5F82042012168606385228520462974EF
:10661000FFF7FAFED5F8403295F8452253F82210DC
:1066200020460831FFF7D0F89620FCF7FDFEFCF776
:106630007FFE237F13F0400508D02E4B01932E4B95
:1066400000932E4A2E4B2F493148B8E703F03F0301
:10665000628DA17F009304F11F0004F11703FEF780
:106660004DF8FFF70FFB636C226C25641344E26B5B
:106670006364934288BF6264E36CA26C002013449D
:1066800006F10901BA68E364A064FCF7D3FE05468D
:10669000FCF752FFE36C606CF23303EB40002844DC
:1066A000FCF728FFFCF76EFF94F820100731324604
:1066B000C9B22046FFF708FD034648B104233B74E6
:1066C000FCF7E4FD022003B0BDE8F040FFF7DCB8C2
:1066D000104A0146FDF796FF30F00203F2D0054B59
:1066E0000193054B0093054A054B06490A4866E7A6
:1066F000A00A0020B8BA000000BB0000C5BA000024
:1067000017C3000072BA00006FC500001FC500006B
:106710000ABA0000D55500009EC4000010B590F8DC
:10672000A440D0F8EC3014F0800F22D1D0F8E8204B
:10673000FAB1240701D59A421BD1D0F8F040A24209
:1067400004BF1468C0F8F0404BB913680B601160C7
:10675000C0F8EC100B680BB9C0F8F41010BDD0F8FD
:10676000F0201C68944202D10A601960F2E72346C7
:10677000F7E72BB9D0F8E8300B60C0F8E810E7E78E
:10678000D0F8F0201C689442EED02346FAE70000CF
:1067900013B50B46044621BB1448FCF7C4FB014665
:1067A00078B9134B0193134B0093134A134B1449BD
:1067B0001448FAF7FDFC404080F311884FF00400C4
:1067C00002DF031D1A7842F003021A7001225A7088
:1067D0000622DA7039B1204602B0BDE81040FFF75A
:1067E0009DBF0021EEE702B010BD00BF000D0020EC
:1067F000B8BA000000BB0000C5BA0000ABC300007F
:1068000072BA00005FCC000013B504461148FCF7D3
:106810008AFB014678B9104B0193104B0093104A44
:10682000104B11491148FAF7C3FC404080F311881E
:106830004FF0040002DF037943F0030303710123E7
:1068400043710B23C371204602B0BDE81040FFF72F
:1068500065BF00BF000D0020B8BA000000BB0000FB
:10686000C5BA0000E0C3000072BA00005FCC0000AF
:106870002DE9F04F1C4693F82030AC4D0733DBB2C6
:106880008DB02B7394F834300A91D907804609D51E
:10689000A36B216C02FB03330B44E16B23648B423B
:1068A00088BF2164268D94F858303244668C92B2A9
:1068B0002285324496B294F859209A4200F03B83E4
:1068C0000022052311461046FEF790FE94F85A3038
:1068D000013B042B00F20A85DFE813F00500C50236
:1068E0006E036F049E04D5F88C220AB9C5F88C4259
:1068F00094F8853013F0070300F0368112B194420A
:1069000040F01983043B012B40F215838848FCF7C3
:106910000AFB0746002800F00E8394F8853003F048
:106920000703032B3DD194F83430DB0742D594F8AC
:10693000583084F859300023C5F88C323B7943F045
:1069400003033B7118237B711023FB71B4F85C3097
:106950003B817B81B4F85E30BB81B4F86030FB8151
:1069600094F862303B74B4F86430A7F81130B4F88E
:106970006630A7F81330B4F86830A7F81530B4F8CB
:106980006A30A7F81730B4F86C30A7F81930B4F8AB
:106990006E30A7F81B30B4F87030A7F81D303946B8
:1069A00086E2022B65D0032BC1D0012B40F0B480CE
:1069B000604900E0604994F8342012F0010258D197
:1069C00094F8853062F3020384F88530E38C063353
:1069D00033449BB2A4F864303879FA7140F0030074
:1069E00038710C20787194F884203A72E26F40F28A
:1069F000E240B2FBF0F2A7F80920B4F85C20A7F857
:106A00000B20B4F85E20A7F80D20B4F86020A7F89A
:106A10000F20A7F811302268C4F87480002A0ADA1F
:106A2000A368606822F0004283422CBF434408EB15
:106A300000039B1A636707F10903C4F880303F4BDA
:106A40000122D960002011469C60FCF765F90028FE
:106A5000A5D03B4B01933B4B00933B4B3B4A3C49FE
:106A60003C48FAF7A5FB404080F311884FF0040042
:106A700002DF94F88530052262F3020384F8853042
:106A80003B7943F003033B7118237B710F23FB71A8
:106A9000B4F85C303B817B81B4F85E30BB81B4F8E4
:106AA0006030FB8100233B74FB743B754FF0FF3378
:106AB000A7F811607B75BB75FB753B767B76BB7663
:106AC000FB763B777B77BB772268238E6386002A31
:106AD000C4F874800ADAA368616822F000428B422D
:106AE0002CBF434408EB01039B1A636707F11303B0
:106AF000C4F88030114B184ADA6001221146002098
:106B00009C60FCF709F900283FF449AF0C4B019356
:106B10000C4B0093114BA1E7094B0193094B0093D8
:106B20000F4B0A4A0A490F489BE700BFA00A002002
:106B3000000D002045520000694F00004002002077
:106B4000B8BA000000BB0000A5C20000C5BA000032
:106B500072BA0000C9CB000051500000BFC2000053
:106B6000D8C200000ABA0000B4F86470F71BBFB2C4
:106B7000380400F1E08194F8582084F85920D5F8C1
:106B80008C222B73944208BFC5F88C32E26D636A85
:106B90009A420CD1A38DA28CB4F860105A437D2385
:106BA00053434FF47A7293FBF2F399421DD00220C3
:106BB000FDF7DAFD40B9C24B0193C24B0093C24BC3
:106BC000C24AC349C3484CE7238CC38005230371E1
:106BD0000023C372B4F85C308381B4F85E30C381A3
:106BE000B4F860300382FEF745FB2368D4F804A0B4
:106BF000002B09DAA06823F0004350452CBF8044E5
:106C0000D0442360A8EB0308A38CB4F85C60B249BD
:106C100013FB07F39BB2B3FBF6F21FFA82F916FBE4
:106C200009F080B2834280F0B080C01A40F2231293
:106C30004243C31701FB0323A0FB010119449EA398
:106C4000D3E90023F9F7E6FA20F07F4000EB0803D0
:106C50000A93238DD4F87CB0DB1B4B442385236837
:106C60009A4538BF9A4694F83430CDF82CA040F2BB
:106C7000E24813F0010F08FB06F6DFF884A200F0EB
:106C80009580A26B216CC3F3420302FB171795F8A2
:106C90002C12924A32F8115032F813301D447543C9
:106CA00005F574258E4B05F23F25B5FBF3F594F8F9
:106CB0008430A56308FB03F305FB09F07208963ADC
:106CC000A36407440023974294BF27642264E263CD
:106CD0006365A0FB0A0178A3D3E90023F9F79AFAC8
:106CE0000A9B1B1ABBFBF8F008FB00F00A93A0FB01
:106CF0000A0171A3D3E90023F9F78CFA94F88530DF
:106D000003F01803102B20F07F48A6EB050502D1F5
:106D10002046FDF749FDB4F85C30B4F86020A38448
:106D2000B4F85E30E38442F210735343B3FBF6F3DE
:106D3000A3856C4BB3FBF6F694F88530268613F0EA
:106D4000180308BFE3850121002002F0D1FB0022D7
:106D5000012181461046FBF7B7FF94F8202041F24D
:106D60006553002107320093D2B25F4B0846FDF70E
:106D7000D5FB30F0020724D0514B0193514B0093C7
:106D8000524A514B524959486BE606FB123292B2B5
:106D9000A2FB010140F2231303FB021146A3D3E936
:106DA0000023F9F737FAA8EB000351E742A3D3E930
:106DB0000023ABFB0A01F9F72DFA354620F07F4896
:106DC000A9E7A5FB0AAB3CA3D3E9002350465946EB
:106DD000F9F720FA464A94F8206020F07F4507230F
:106DE00020F07F400021434302FB0133A0FB02015E
:106DF000BAEB000019444FF47A724FF000036BEBCA
:106E00000101F9F707FA0B9AE3683A490290134433
:106E10009AB294F83430049213F0010F06F1070689
:106E2000354B069408BF0B4641F275510891F6B2F6
:106E30002D490791059303970195CDF800800A9B92
:106E4000324639463846FDF7DBFA30F0020093D17E
:106E5000B9F1000F00F0AD80012211460DB0BDE880
:106E6000F04FFBF731BF94F85C30002B4AD0234839
:106E7000FCF759F8054600285DD0002384F85C3003
:106E8000E38C06333344A4F86230037943F0030300
:106E90000371082343710123C37104F15D010522CD
:106EA0000830F9F795FFB4F86230A5F80D3029469F
:106EB0002046FFF733FC3EE08D49FD1A0700000035
:106EC000B8BA000000BB0000D8C20000C5BA00007C
:106ED00072BA0000ECC400000054CE09E8C50000FE
:106EE00040420F00005A6202495400009EC4000054
:106EF0008D49FD1A097300000D730000000D00207C
:106F000000CA9A3BB4F86230F31A190413D494F807
:106F1000583084F8593004F11705052204F15D0159
:106F20002846F9F755FF05212846FCF762F8237F2C
:106F300060F30503237794F8952094F894309A42EF
:106F40001DD00022114610460523FEF74FFBCD4809
:106F5000FBF7E9FF014690B194F8943084F895303E
:106F6000037943F00303037102234371C37194F85F
:106F7000963003722046FFF7D1FB238E638694F888
:106F8000341094F82030C048A268039411F0010F27
:106F900003F10703BD49DBB208BF01468DE80C00D1
:106FA0000291231D22460A9940460136FEF7BAFC9B
:106FB00066840DB0BDE8F08FB248FBF7B4FF07461A
:106FC0000028B8D094F8349094F8583084F85930A8
:106FD00019F0010945D104F1A5052B464A4604F1F3
:106FE000770104F16700FCF795F82946102204F1B7
:106FF000C600F9F7EDFE04F1BE01082204F1DF003E
:10700000F9F7E6FE94F8BD3084F8B59069F3000313
:1070100084F8BD3094F8DE3084F8B69043F0010374
:1070200084F8DE3094F8A43084F8B79043F030034D
:1070300084F8B89084F8B99084F8BA9084F8BB903A
:1070400084F8BC90A4F8D690A4F8D890A4F8DA906C
:10705000A4F8DC9084F8A430391D2046FFF798FB93
:107060009DE494F8A43003F04803082B00F08E80D0
:10707000037943F00303037194F85C5045B1022394
:1070800043710D23C3710023057284F85C3086E4DC
:107090007C48FBF748FF814640B97D4B01937D4B0F
:1070A00000937D4A7D4B7E497E48DAE4037943F0C4
:1070B000030303710D2343714FF0040A00F1080329
:1070C00009F1100B80F807A008221846AA210B939B
:1070D000F9F7AAFE5246BB215846F9F7A5FE0B9BCD
:1070E0000822194604F17F00F9F772FE524659460C
:1070F00004F1C200F9F76CFE4946204604F1A509E7
:10710000FFF70CFB4B462A4604F1770104F16700B8
:10711000FCF700F81022494604F1C600F9F758FEC2
:10712000082204F1BE0104F1DF00F9F751FE94F8E2
:10713000BD3084F8B55043F0010384F8BD3094F8B5
:10714000DE3084F8B65065F3000384F8DE3094F83E
:10715000A43084F8B75043F0100384F8A43001231E
:1071600084F8B85084F8B95084F8BA5084F8BB5009
:1071700084F8BC50A4F8D650A4F8D850A4F8DA503B
:10718000A4F8DC507B710523FB7108E4D5F82002DC
:1071900090F8A43043F0200380F8A4300021FFF7DA
:1071A000F7FAD5F8202292F8A43003F0FB036FF32E
:1071B000C30382F8A430FFF7F2BB3248FBF7B3FEFB
:1071C000054600283FF4B7AE94F8583084F859309B
:1071D0000F23C4F88830037943F0030303710923B4
:1071E000437194F8343013F0010F0CBF08230E23C1
:1071F0000822C37100211044F9F716FED4F8883034
:107200002B721A0A1B0C6A72AB7229462046FFF7D2
:1072100085FA238E63868EE694F88C30DA0721D4C3
:107220001848FBF780FE014600283FF484AE94F82E
:10723000583084F8593094F88C3043F0010384F8C6
:107240008C30037943F003030371062343710C234D
:10725000C371092303724FF0FF3343728372C37209
:107260000373D3E79B073BD594F8583084F8593023
:107270000220FDF779FAC8B9054B0193054B00933D
:10728000094B9DE4000D0020456400009D65000051
:10729000B8BA000000BB0000C5BA00009EC30000E1
:1072A00072BA00005FCC0000EFC20000238CC380E4
:1072B00001230371037A43F003030372062343722D
:1072C0000C23C37294F88D300373B4F88E30A0F899
:1072D0000D30B4F89030A0F80F30FDF7CBFF2AE660
:1072E000054B0193054B0093054B1AE4024B0193A8
:1072F000024B0093034B14E4B8BA000000BB00003B
:10730000EFC20000FEC20000FFF7B2BAFFF7B0BA4A
:107310002DE9F04F91B0FBF7D9FFC5B245B3FBF7AC
:10732000F1FF5FFA80F9FCF75FF8C6B2FCF706FAE6
:10733000C4B2FCF7E9F9C3B20A93FCF721F8C7B26B
:10734000FBF7AEFFFCF762F8FCF744F8FCF7E2F954
:10735000FCF70EF86148037C8246052B01F2678436
:10736000DFE813F0540078000D008E0A8E0A8E0AB2
:10737000FF232F462C462E46A9460A93E0E7012319
:107380000374FCF711F904469620FCF74DF8FBF75F
:10739000CFFF9AF80F30013BCB34032B51D8DFE8F5
:1073A00003F002233838FBF7B7FFFBF757FFFBF773
:1073B00087FF40B14A4B01934A4B00934A4B4B4ADB
:1073C0004B494C480DE29AF8D43013F0C00F05D069
:1073D0009AF8430010B14849FCF770F92046FCF7D1
:1073E00089F8FCF7CFF811E09AF84522DAF8403234
:1073F00053F822000830FBF731FFFBF761FF00284C
:10740000D8D12046FCF776F8FBF7A2FF11B0BDE813
:10741000F08F9AF84522DAF84032DAF8200253F871
:1074200022100831FEF7D0F9FBF74AFF0028C1D13E
:107430002046FCF75FF8FCF7A5F80120FEF724FAD8
:10744000E4E7274B0193274B0093274B274A284912
:107450002A48C6E12DB903238AF81030FBF716FF3E
:10746000D4E7C37B013B032B01F20382DFE813F077
:107470000400C10157045704B9F1000FEBD0FBF72A
:107480004BFF037803F00F03032B054638D14378F5
:107490000C2BE0D19AF8D430580602D50EB9002C46
:1074A000D9D003238AF81030FBF74AFF9AF8A531A8
:1074B0009AF8A6219A4206D00133DBB2022B08BF0C
:1074C00000238AF8A5319AF8A501272303FB00A021
:1074D00000F25710FBF7C8FE98E700BFA00A002093
:1074E000B8BA000000BB000041C00000C5BA0000EF
:1074F00072BA0000F8C50000E40A00200ABA0000D1
:10750000052BA8D14378222BA5D19AF8D430DB09DA
:1075100002D00EB9002C9ED09AF886322BB19AF880
:1075200084329AF885229A4295D1DAF8A831002B54
:1075300091D00320FDF718F9064600288BD04FF0B4
:10754000040B8AF810B0FBF7A1FEDAF8A841DAF8CC
:1075500014120027FC222046CAF8A871FBF715FD7B
:107560000322208405F1120104F11400F9F730FC24
:1075700004F1100318465A4604F1170805F10E01EC
:107580000D93F9F725FC052205F11E014046F9F798
:107590001FFC05214046FBF72CFD227F0D9B60F36D
:1075A0000502227795F82320C2F30402A277B5F8EA
:1075B0001880A4F82480E97EAA7E42EA0122E284AF
:1075C00019465A4604F15000F9F702FCAA8B40F222
:1075D000E24942F2107309FB08F85343B3FBF8F396
:1075E000A385C94BB3FBF8F32386238CF38029468C
:1075F0000123F772337311F8023B4FF0030BC3F30F
:107600008013737386F804B0062206F10E00F9F7B2
:10761000DFFB2946062211F8083BC3F3C01333757C
:1076200006F11500F9F7D4FB9DF82830F3762B8B83
:10763000B3836B8BF383AB8B338495F82330C3F325
:10764000421386F82230208CFDF7E4FEFDF712FE8F
:1076500095F8232094F83430AC49520962F343037F
:1076600084F834309AF82C3231F8122031F8133083
:10767000134408FB03F303F57423A54A03F23F23E5
:10768000B3FBF2F34FEA5802963AA363E2636A7DD2
:10769000A76409FB02F2E264DAF8886266604FF0E0
:1076A00027092822A8EB030840F286334E45E26002
:1076B000C4F80090A7604FF0050200933946954B3F
:1076C000384638BF4E46FCF729FF40F28731FDF7B8
:1076D000DDFE9AF8553109FB03A999F8073103F04B
:1076E0000F03012B06D100973B465A4639463846D0
:1076F000FCF714FF94F82030874F0733DBB20D936B
:10770000DAF80430A3EB060BFBF74EFFA8FB078962
:1077100079A3D3E90023824649464046F8F77AFD2B
:1077200040F2A33308937D4B07937D4B069405935A
:10773000E3687C4ACDE90A011E4420F07F4007231C
:107740000021434302FB0133A0FB0201B8EB000020
:1077500019444FF00004B6B24FF47A724FF00003B0
:1077600069EB010104960394F8F754FD0A9B02901B
:1077700023F07F430193E88A80B2013040F2E24572
:107780004FF0000141F10001A0FB05230AF1FF3A8F
:1077900012EB0A0205FB013343F10003A2FB0701D0
:1077A00007FB031156A7D7E90067801952A3D3E955
:1077B00000237941F8F72EFD20F07F4000905B46D2
:1077C0000D9A21462046FCF71BFE30F002033FF4E1
:1077D0001DAE554B0193554B0093554B554A564999
:1077E0005648F9F7E5FC404080F311884FF004005B
:1077F00002DFB9F1000F00F0308290F8BC21C2F333
:1078000000121AB116B9002C00F02782DAF84032C3
:107810009AF8451253F82160DAF80C32FBB19AF865
:1078200086322BB19AF884329AF88512994216D191
:10783000337A190700F08680337A03F00F02012AA9
:107840000DD19AF8BC21DB09B3EBD21F00F02981DE
:107850009AF8BC31C3F301139D0700F12C81337AF0
:1078600013F00F0202D0062A40F004829AF8BC11ED
:10787000CC0740F1EE81DAF80C12002940F0E981E2
:107880003846FDF7A9FD002840F0E781FBF744FDED
:1078900003782B49032262F303039AF8BC21D2092F
:1078A00062F386130370337A0278C3F3801363F3B1
:1078B000C7120C2304464370027006220230F9F707
:1078C00087FA062206F10A0104F10800F9F780FAA6
:1078D0009AF8BC3143F002038AF8BC3120460223F7
:1078E0008AF81030FBF7C0FC9620FBF79DFDFBF7F4
:1078F00017FD76E5AFF300808D49FD1A0700000003
:1079000000DC356BD8FFFFFF005A6202E8C50000BB
:1079100040420F008D54000000CA9A3B49540000B9
:107920000D7300008D49FD1AB8BA000000BB0000BD
:1079300054C00000C5BA000072BA00009EC4000026
:10794000630C0020002A00F09980FBF72DFEDAF886
:10795000B83100F5FB74D4480722A3FB000102FBF9
:107960000311CDA3D3E90023F8F754FC84424FF070
:107970000005BFF474AF0320FCF7F6FE8146002833
:1079800000F06B814FF00408DAF80C428AF810809E
:10799000CAF80C52FBF7C0FC0278052161F3030220
:1079A0009AF8BC1102F0DF02C90961F38612027075
:1079B000327A0178C2F38012831C074662F3C71142
:1079C000222201704270B9490D931846062207F130
:1079D000080BF9F7FDF906F10A0106225846F9F7F6
:1079E000F7F9424604F1100107F10E00F9F7F0F93A
:1079F000032204F1140107F11200F9F7E9F9012358
:107A00007B75BAF80232DAF8106240F2E24202FB09
:107A100003F8002E5CD1FBF7C7FDBD7500F24B6685
:107A2000FD75BAF802323B83BAF804327B83BAF8A8
:107A30000632BB8304F11701052207F11E00F9F796
:107A4000C7F9A27F97F8233062F3040387F8233045
:107A50009AF82C2262F3471387F82330FBF770FC67
:107A60003846FBF701FCFBF72BFC0546002842D00B
:107A70008F4B01938F4B00938F4BA0E49AF8BC215E
:107A8000C3F38013C2F380129A427FF4D5AE06226C
:107A900006F10A018948F9F786F900283FF455AF45
:107AA000CAE6062206F110018048F9F77CF90028A1
:107AB0003FF44BAFCCE696F90830002BBFF6CFAEC3
:107AC000737D03F0C003402B7FF4C9AE3DE746440D
:107AD000002EFCDBFBF768FD00F24B608642F6D31C
:107AE000FBF762FDA6F24B63181A40F2E243B0FBCB
:107AF000F3F0F88295E7FBF745FDDAF81412FC2263
:107B00002046FBF742FA0323208489F80B5089F8BA
:107B10000C5089F804303B78A9F80600C3F3C01371
:107B200089F80D305946062209F10E00F9F750F98F
:107B30003B780D99DFF894B1C3F38013062289F8DE
:107B4000143009F11500F9F743F99DF8283089F848
:107B50001B30BAF80232A9F81C30BAF80432A9F87E
:107B60001E30BAF80632A9F8203097F82330C3F354
:107B7000421389F82230208CFDF74CFCFDF77AFB8C
:107B8000DAF88872DAF80832E36027239F426760E8
:107B9000236038BF1F464FF494630622A560294630
:107BA00000932846464BFCF7B9FC40F2A141FDF793
:107BB00097FC2B460422294600952846FCF7AEFC8C
:107BC000DAF80430A3EB070A94F820300694073360
:107BD000DBB20A934FF4976308933A4B07933A4BFF
:107BE0000593E3680395A8FB0B891F44BFB22CA340
:107BF000D3E90023404649460497F8F70BFB1046AB
:107C000019464FF47A720023F8F704FB24A3D3E952
:107C10000023029049464046F8F7FCFA20A3D3E936
:107C200000230190A6FB0B01F8F7F4FA20F07F4047
:107C3000009053460A9A29462846FCF7E1FB30F0AB
:107C400002033FF4E3AB1A4B01931A4B00931A4B18
:107C5000C4E57AB9737A002B59D103238AF810301E
:107C6000FBF714FB9AF8BC316FF341038AF8BC317F
:107C7000FFF7CCBB012A2BD0337A03F00B02022A88
:107C8000E8D003F00F03042BE7D19AF8BC31990731
:107C9000E0D4E2E7AFF3008000CA9A3B00000000A6
:107CA0008D49FD1A070000008D49FD1A630C002064
:107CB000B8BA000000BB00005FC000005D0C0020EF
:107CC000E1540000495400000973000000CA9A3BC7
:107CD0009AF8BC21DB09B3EBD21F0FD09AF8BC3164
:107CE000C3F301139807C7D596F90830002BC3DA00
:107CF000737D03F0C003402BBED1ABE7062206F133
:107D00001001C548F9F74FF80028A3D0E6E7DAF8E4
:107D10000C32002BA1D13846FDF75EFB9DE790F8B1
:107D2000243290F84522013380F82432D0F84032D2
:107D300053F8226001233371B9F1000F00F0688518
:107D40004FF00008D0F8204280F8258294F8A43043
:107D5000317A03F00102C1F38001914200F0FA8010
:107D600082F0010262F3000384F8A430DBB21A0649
:107D700000F1EC80D4F8E88094F8F92008F10400D0
:107D800087187D78002D7AD0815C9B0601F0030175
:107D90000AD5D4F8D620D4F8DA30013243F1000302
:107DA000C4F8D620C4F8DA30032968D1FB78023B46
:107DB0000B2B64D8DFE803F0064A9C6363636363BC
:107DC000656E63A303238AF81030FBF75FFAFBF7B5
:107DD00077FA30B1914B0193914B0093914BFFF7A0
:107DE000EEBA3979DAF82002132908BF1621FDF717
:107DF000BFFF0124DAF8203293F8F920154493F8F4
:107E0000F820EDB2AA4283F8F9501CD1D3F8E8204B
:107E1000D3F8EC1000208A4283F8F80083F8F900C8
:107E200077D1B8F1000F0ED01168D3F8F020C3F865
:107E3000EC109142C3F8E81008BFC3F8EC007A498F
:107E40004046FBF78AF84FF000086BE0082207F184
:107E50000E0104F17700F8F7BBFFDAF820020422E4
:107E600007F11601BE30F8F7B3FFDAF8203293F8C5
:107E7000A42042F0080283F8A4201A8E5A86002417
:107E8000B8E794F8A43043F0480384F8A430238E74
:107E90006386F4E79AF80F70FFB2042F28D198F8A0
:107EA000043043F0030388F80430172388F80530C2
:107EB000032388F80730082204F15D010430F8F745
:107EC00087FF94F8653088F8103094F8663088F8A9
:107ED00011300822CC2108F11200F8F7A5FF08F1B3
:107EE0001A003A46DD21F8F79FFF4FF00008C6E779
:107EF00094F8A43043F0080384F8A430BFE794F862
:107F0000A43003F0FB036FF3C30384F8A430002311
:107F1000BEE7D3F8F0108A42126808BFC3F8F02019
:107F2000C3F8E820B4B1DAF82002FDF7EFFD002332
:107F3000CAF82032B8F1000F3FF468AA0025DAF839
:107F400020324146188CFDF75FFC7BE168F3C713D4
:107F500084F8A430DAF82032327A93F8A430C2F3ED
:107F6000C002C3F340039A4240F064840320FCF74C
:107F7000FBFB002800F05E849AF88632A3B3DAF89F
:107F80005032DAF85422934205D19AF884229AF8B2
:107F90008512914228D0DAF85422934200F04A84A4
:107FA0009AF884329AF885229A4200F043849AF82B
:107FB000843233B9DAF82032BAF882221B8C9A4222
:107FC00012D09AF8843203F0FF05002B00F03384BE
:107FD0009AF88432DAF820120AEB4303B3F87C22D1
:107FE0000B8C9A4240F02684777A002F00F0B781FC
:107FF000DAF8203293F8A47017F010071FD0FBF7BF
:1080000039FBD8B9054B0193054B0093074A084B40
:1080100008490948FFF7E5BB630C0020B8BA000027
:1080200000BB00006AC00000000D0020C5BA0000BF
:10803000CEC0000072BA00002BC600000127DAF89B
:10804000203293F8A430DA0626D4DAF8204294F8E5
:10805000A43013F0040F337A32D113F0030300F08D
:10806000D083022B40F24B81F57A112D00F2B483BC
:10807000DFE815F03700F80028012C0147015F0107
:108080007701A803B601F3010A0216022E028D023F
:10809000B601960275016503FBF70AFB0028D4D1EF
:1080A00003238AF81030FBF7F1F8FBF709F90446CF
:1080B00058B1BF4B0193BF4B0093BF4BFFF77FB944
:1080C00003F00302032AEBD1C7E73D21DAF82002CF
:1080D000FDF74EFEDAF82002FDF718FDCAF820423F
:1080E00028E7B6F81510638CCB1A1B0400F1A6859F
:1080F00094F8593094F858209A4213D094F85A20A2
:10810000012A05D194F8852002F00702052A09D03A
:10811000A74B0193A74B0093A84AA94BA949AA488A
:10812000FFF75FBBDAF88C227AB994F83420D507D0
:1081300009D49F4B01939F4B0093A04AA04BA149A8
:10814000A248FFF74EBBCAF88C42327B84F88420E9
:10815000B6F80D0040F2E2424243E267307CF27B27
:1081600042EA0022A4F85C20B07C727C42EA002241
:10817000A4F85E20F27C307DA4F8641042EA00226C
:10818000A4F8602094F8852002F0F8026FF3C4028E
:1081900084F88520013B0122002584F85A2084F8C8
:1081A00059306586DAF8201291F8A43083F0020382
:1081B00081F8A4305FB1D1F8B520D1F8B9300132DF
:1081C00043F10003C1F8B520C1F8B9300027DAF84F
:1081D00020020FA990F8A440FCF70CFD9AF810308B
:1081E000032B4FEAD41415D0002F40F02683B9F1A9
:1081F000000F07D0337ADB0604D40F9B5B78002B8B
:1082000000F01B83DAF8203293F89730002B0CBF74
:1082100002230323032B8AF8103040F022839AF8BC
:108220000F30042B40F00B83DAF8203293F8A420AF
:1082300064F3C71283F8A420FBF728F8B8F1000F05
:108240007FF47DAE002D3FF4E1A8DAF82032188CDF
:10825000FDF7E0F8DAF820321B8CF380FDF70AF81E
:10826000FFF7D4B8B6F81130628C9B1A180400F1ED
:10827000E58494F8582094F859309A4209D04C4B30
:1082800001934C4B00934D4A514B4E495148FFF7D7
:10829000A8BA052206F10C0104F15D00F8F798FD7B
:1082A000737CB27C43EA0223A4F86230022384F890
:1082B0005A3094F859300025013B84F85C5084F81A
:1082C00059306FE7337B84F8973048E0082206F195
:1082D000160104F17700F8F77BFDDAF8200204229A
:1082E00006F11E01BE30F8F773FDDAF8203293F87C
:1082F000A42042F0040283F8A4201A8E5A86012595
:1083000050E7082206F10C0104F17F00F8F760FD48
:10831000DAF82002042206F11401C230F8F758FD01
:10832000DAF8202292F8A43043F0040382F8A43053
:1083300015E094F8582094F85930934209D01C4B1A
:1083400001931C4B00931D4A234B1E492348FFF702
:1083500048BA0322013B84F85A2084F8593000259A
:1083600020E79AF80F20D2B2032A17D194F85810B8
:1083700094F859308B42E2D1013B84F85A2084F8BA
:10838000593094F8A430590605D56FF3861384F854
:10839000A4300623337100236386B0E794F8A43039
:1083A00003F0FB036FF3C30384F8A430E9E700BFD5
:1083B000B8BA000000BB0000CEC00000C5BA000083
:1083C00082C3000072BA000051C60000F3C600006C
:1083D0008EC300002FC70000B9C0000071C70000A5
:1083E000337B727BC54843F07F4343F47E0343F401
:1083F000435343F0100343EA0223B27B43EA0243B0
:10840000D4F88820C2F310021340C4F88830FAF779
:108410008AFD054648B9BA4B0193BA4B0093BA4B53
:10842000BA4ABB49BB48FFF7DCB9037943F0030301
:108430000371082209234371C37100211044F8F726
:10844000F3FCD4F888302B721A0A1B0C6A72AB72D8
:1084500029462046FEF762F981E7337B727B43F0C1
:108460007F4343F47E0343F4435343F0100343EA52
:108470000223B27B43EA0243D4F88820C2F31002FD
:108480001340C4F8883086E72046FEF7BDF9DAF8D5
:10849000202292F8A43043F044036FF3041345E71D
:1084A0009AF80F30042B0AD12046FEF7ADF9DAF81E
:1084B000203293F8A4206FF3041283F8A420DAF892
:1084C000202292F8A43043F004036FF345132DE704
:1084D000337B84F88D30B27B737B94F88C5043EA05
:1084E0000223A4F88E30F37B327C43EA0223A4F803
:1084F000903094F88C3005F0030001284FF000050F
:1085000043F0020304BF6586054613F0010B84F8AF
:108510008C307FF447AE43F0010384F88C30774809
:10852000FAF701FD014628B9754B0193754B00938D
:10853000794B75E7037943F0030303710623437115
:108540000C23C371092303724FF0FF33437283720C
:10855000C37203732046FEF7E1F894F8A43043F0A9
:10856000800384F8A430FAF7D3FE037880F801B0D2
:10857000012262F30103D4F8E8200370DBB21AB1E0
:1085800043F0100303700DE662F30413FAE794F866
:10859000A43003F0FB036FF3C30384F8A430FAE6BE
:1085A00094F8592094F85830934268D1DAF88C3214
:1085B000002B40F09780DAF88C320BB9CAF88C4265
:1085C000717B337B43EA0123A4F85C30717C337CFC
:1085D00043EA0123A4F85E30708AA4F86000337D7A
:1085E00084F86230B17D737D43EA0123A4F86430DE
:1085F000317EF37D43EA0123A4F86630B17E737EB9
:1086000043EA0123A4F86830317FF37E43EA012373
:10861000A4F86A30B17F737F43EA0123A4F86C3079
:1086200096F82010F37F43EA0123A4F86E3096F801
:10863000221096F8213043EA0123A4F87030E16D4E
:10864000636A994202F1FF3294F885300AD1A18D14
:10865000A58C4D437D2169434FF47A7591FBF5F16B
:10866000884229D0042161F302036FF3C40301257A
:1086700084F8853084F85A5084F8592092E594F8AB
:108680003450DAF88C3215F0010524D09C420CD11C
:1086900094F85A30012B08D194F8853003F0070381
:1086A000591E012987D9052B85D0154B0193154BF0
:1086B00000931A4BFEF7CABE0320002560F30203A5
:1086C000012165F3C40384F88410E56784F88530DC
:1086D00084F85A10D0E79C42E7D194F85A30012B25
:1086E000E3D15FE50548FAF71EFC0146D0B9044B1B
:1086F0000193044B00930A4B92E600BF000D00204B
:10870000B8BA000000BB0000CFC30000C5BA00002B
:1087100072BA00005FCC0000F3C30000B9C00000D3
:1087200004C40000037943F003030371032343717E
:108730001123C3710F2303722023437289E694F837
:10874000583094F859209A423FF409AE84F85930D1
:1087500094F85A30012B2ED1DAF88C329C4209D091
:10876000A04B0193A04B0093A04AA14BA149A24862
:10877000FFF737B80023CAF88C3294F834206386A8
:10878000D20744BFA26F626594F8852012F0180FDB
:108790007FF4E5ADF37205223271E28CA38CF28195
:1087A000A28DB3815A437D2353434FF47A7293FBD6
:1087B000F2F33382A3E58B4B01938B4B00938F4BEA
:1087C000FEF744BE94F8583094F859209A423FF48A
:1087D000E2AD84F8593068E78948FAF7A4FB01460E
:1087E00028B9804B0193804B0093864B18E60379A0
:1087F000057243F003030371022343710723C3711E
:1088000027E6784B0193784B00937F4BFEF71EBE13
:1088100090F8253213B9022380F825329AF8257290
:10882000013FFFB28AF825720025B7FA87F77F0962
:10883000A846CCE400252F46C9E40323EAE4FAF76E
:108840007FFD0F99DAF820020B7890F8A42062F3EC
:10885000C303C2F3400262F382030B70FDF7F2F927
:10886000ECE49620FAF7E0FDFAF75AFDFAF78AFEF3
:10887000E7E75C4B01935C4B0093644BFEF7E6BD6E
:10888000C27B042A00F2BF81DFE812F0AC010500D0
:10889000480096009600032B0DD190F8D43013F0C9
:1088A000380F08D0FDF728FA02238AF81030FAF7BB
:1088B000E7FCFEF796BDFAF783FD9AF81030032B1C
:1088C0005DD19AF85531272202FB03A393F80731B3
:1088D00003F00F03012B52D040F6E1230021069351
:1088E0004B4B0593049140F2471303910291019180
:1088F000009105220846FBF7CBFD30F002033ED085
:108900009AF80E30052B3AD0364B0193364B009334
:10891000364A404B37494048FEF763BF032B21D10D
:10892000D0F8403290F8452253F822000830FAF788
:1089300095FC9620FAF778FDFAF7FAFCFAF708FDAD
:108940009AF8BC3113F0300F05D09AF8430010B1FB
:108950003249FAF7B3FE01238AF81030FAF78AFC9D
:10896000FEF73FBDFAF72CFD9AF81030052B06D123
:1089700000230093042219461846FBF7CFFD00247C
:108980008AF80F408AF810408AF80D40FAF7AAFDDD
:10899000224621462046224BFAF7BEF9044600281B
:1089A00000F038810F4B01930F4B00930F4A1D4B82
:1089B00010491D48FEF715BFD0F820020028DED070
:1089C0009AF80F30032B31D190F8971071B3FDF75F
:1089D000CFF9DAF82002FDF799F80023CAF820321F
:1089E000CDE700BFB8BA000000BB0000C5BA000068
:1089F0007EC0000072BA0000CBC70000A0C000001B
:108A0000000D0020BEC30000CEC00000DEC000008C
:108A100035550000F1C0000010C80000E40A002035
:108A200000020020C1C10000C9CB0000468D9AF8A9
:108A300024429AF80F30751CADB2002C5CD0032B89
:108A400055D1FAF795FDDAF82072DFF82C928346BB
:108A5000786C00F14808C34585A3D3E900233FD8CB
:108A6000A0FB0901F7F7D6FB84B2A8EB0B0080A3AB
:108A7000D3E90023A0FB0901F7F7CCFB82B2002366
:108A80007B64FB64FB8C7B85D7F8E83033B15B7982
:108A900013B997F8F9300BB100237B85DAF820324F
:108AA0000021D985DAF82002C38DBBB19D4280F048
:108AB00091805B1B9BB20021062BC385418540F250
:108AC0008B809AF80F30032B08D1002E40F0848061
:108AD000016D4B0811F0010134D10365002134E030
:108AE000ABFB0901F7F796FB022284B2C7E700222D
:108AF00080F835201446D1E7042B0BD190F897105D
:108B000041B1FDF735F9DAF82002FCF7FFFFCAF8AA
:108B1000204234E79AF80F30042B0CD190F835300E
:108B20004BB19D4205D25B1B80F8353000221446C4
:108B3000B8E73E214BE7C48D002CF7D1838DC38568
:108B40002246AFE743F000430365438E1BB19D42CD
:108B500044D25D1B458690F8595090F858309D429C
:108B600006D090F85A30013B012B9CBF002343856F
:108B700011B9438DB34233D0438D01339BB224B935
:108B80001AB913B900293FF4FAAE90F820502E48D4
:108B9000049107350021EDB205900393009223461E
:108BA0000695029101912A460846FBF771FC30F0C8
:108BB00002033FF4E4AE9AF80E309D423FF4DFAE7C
:108BC000224B0193224B0093224A234B23492448F2
:108BD000FEF707BE0821FAE60121B6E72221F6E6F4
:108BE0000B46CCE7043B012B09D9184B0193184BDA
:108BF0000093184A1B4B19491B48FEF7F2BD00238E
:108C00000374FEF703BC114B0193114B0093154BFA
:108C1000FEF71CBCDAF80000436821465B68984701
:108C2000012211462046FAF74FF8FEF7EFBB074B3B
:108C30000193074B00930D4BFEF708BC2823FFF769
:108C400042BB00BFAFF3008085550000B8BA0000FA
:108C500000BB0000C5BA0000FFC0000072BA0000EF
:108C60007EC800000EC10000F4C8000024C100004E
:108C70008D49FD1A0700000000CA9A3B2DE9F0411A
:108C8000394D9DF818C0099CBDF828602860C2EBDA
:108C9000821003F1030E85F82C12C5F81442A119B5
:108CA000043304EB80040CF10200BDF81C80C5F80D
:108CB0004042DBB2C0B204EB83040CF101074FEA7F
:108CC000C00C85F87802C5F8704204EB0C0008F17E
:108CD0000304282C5FFA8EFEA5F8388288BF08F1BD
:108CE0000E0885F858E28BBF28F003080EEB4E0EF5
:108CF00018FB0EFE4FEA0E1EA5F83AE2B5F83A420E
:108D0000C5F874024FF0300E6044A5F83CE2C5F897
:108D10003002B4FBFEFE20449C18C5F8480200EB6C
:108D2000C400BDF82040C5F85C020A3424F00304F6
:108D30004830A4B2FFB2A5F86C4207FB0404641AE1
:108D400085F81C2285F8443285F83EE2C5F86402B5
:108D500003D034442046BDE8F081012385F88632F3
:108D6000FDF7C2FAF6E700BFA00A002038B50321DC
:108D70000520FBF7C5FD04210620FBF7C1FD1A4CB9
:108D8000002594F81C22ABB29A4205F1010525D8C2
:108D90003021B4F83A22B2FBF1F284F83E2294F882
:108DA0004422A4F83C120023013A84F8453263744B
:108DB00084F8793284F84330C4F8A831C4F80C320E
:108DC00084F8463284F8582284F87A3284F87B3268
:108DD00084F87C32BDE83840FDF786BAA81DFF2133
:108DE000C0B2FBF78DFDCCE7A00A00200048704719
:108DF000A70B002000487047F70B0020024B002211
:108E00005A749A74704700BFA00A002070B5104BC6
:108E10005E7CFF2E1AD00022D5B246FA05F414F07B
:108E2000010402F10102F7D10122AA4032435A742F
:108E300000F00102987CAA4002439A74062202FBC9
:108E400005301330F7F7C4FF204670BD012070BD18
:108E5000A00A00202DE9F843174C637C06460F4614
:108E600043B108254FF006084FF013096B1EDDB221
:108E7000FF2D02D10120BDE8F883637CEB40DA07C7
:108E8000F4D5A37C2B417340DB07EFD418FB05908E
:108E9000062239462044F7F786FF0028E6D1012351
:108EA000AB40627CDB43DBB21A406274A27C1340AD
:108EB000A374BDE8F88300BFA00A002000000000F2
:108EC0002DE9F04FDFF878B28FB0022391469BF87E
:108ED00056210D934FF0270840F2071318FB023874
:108EE00007461BF8083003F00F03012B8A465E4645
:108EF00000F2D680DBF8A8510DB10120CDE00BF5D2
:108F00001370FAF710F80B900028F6D00BF50670E6
:108F1000FAF709F80B9A044628B90BF513711046B5
:108F2000FAF71BF8E9E74FF6FF7303840F23C0F845
:108F30008830037FC57765F38613037790F8343064
:108F4000458443F0010365F3041380F834300623AD
:108F5000C38590F88C30058565F3000365F3410304
:108F600080F88C3090F8A430458565F3000365F3F4
:108F7000410365F3820365F3C30365F3041365F3EB
:108F8000451365F3861365F3C713056445644565AA
:108F9000458680F8585080F8595080F8945080F8F1
:108FA000955080F89750C0F8982080F8A430C0F809
:108FB000E850C0F8EC50C0F8F050C0F8F45080F819
:108FC000F85080F8F950CBF8A80196F8D4306AF33D
:108FD000020369F3871386F8D430B9F1000F0BD080
:108FE0005149B37C86F8D630302201F1C400F7F73E
:108FF000EFFE737C86F8D530D6F88832C6F8C830D4
:10900000272B38BF272399461BF80830474DDFF838
:1090100034A12722C6F8C42003F00F030022C6F8AB
:10902000CC20012B4FF08202C6F8D0200DF1340B7A
:1090300049D1002F47D1FBF72DFBD6F8D030CDF822
:1090400020B04B449AB204920193804603460795A0
:109050000697CDF814A003970297009705220321E5
:109060003846FBF7CDF902281ED00D9800BB304BD7
:10907000059303224AF2FE330093CDF820B0079502
:109080000690049003900290019043461146FBF72E
:10909000B7F902283ED00D9850B90FB0BDE8F08F57
:1090A000002492E7FBF718FB0D9B022BFAD0DCE7BC
:1090B000002C3FF422AF1F49D4F89800F9F74DFF78
:1090C0001D4920462CE7FBF7E5FA07950025CDF86A
:1090D00020B00695CDF814A0D6F8D0300395804680
:1090E000994416480295BAB21FFA89F3A2FB00010F
:1090F0000493912303FB021109A3D3E90023F7F79B
:1091000089F8009501904346052203212846BEE7D1
:10911000FBF7E2FA0D9B022BFAD0BCE7AFF300801D
:109120008D49FD1A07000000B30A0020E146000047
:1091300015530000EC0C0020B80C0020002AE78436
:10914000A00A0020DD5A000070B503210520FBF7BE
:10915000D7FB054680B9094CD4F8A86166B1C4F8BC
:10916000A80104F51371D6F89800F9F7F6FE04F596
:1091700006713046F9F7F1FE284670BDA00A0020BE
:1091800008B5FBF7A7FB68B190F8582090F8593064
:10919000934207D10133052280F8583080F85A20D5
:1091A000002008BD012008BD10B50C46FBF792FB5E
:1091B00060B190F8952090F89430934206D1013335
:1091C00080F8964080F89430002010BD012010BD3A
:1091D0002DE9F341054608461849D1F85032D1F837
:1091E000542293420F461FD0D3F8048001F27B2112
:1091F00098F80020FBF724FB0446E0B902AE97F88C
:109200007B3206F8033D97F87C2231460DF10600CB
:10921000FBF716FB34B928B9C5F80080204602B028
:10922000BDE8F0810446EEE791F87C2201F27B2153
:10923000FBF706FB044600232B60EFE7A00A0020A3
:109240001FB5244C04AA002342F8043DD4F854026C
:1092500004F51471F9F7C0FE78B91F4B01931F4B49
:1092600000931F4A1F4B20492048F7F7A1FF4040B9
:1092700080F311884FF0040002DF04F51371F9F751
:109280006CFE039B1A79072A06D80123934013F03A
:10929000EE0F0AD1DB061BD40F4B01930F4B00934B
:1092A0000F4A104B10491248DFE794F8442294F813
:1092B0005832013A934208DB074B0193074B009366
:1092C000074A084B08490B48CFE7013384F8583266
:1092D00004B010BDA00A0020B8BA000000BB000016
:1092E000C5BA000039C4000072BA00009FCA00006D
:1092F0000ABA00000ACB00002DE9F3411B4C0546D9
:109300000068A4F50D76A4F11C0728B9286002B006
:10931000BDE8F041FCF79EBF0279D0F80080072A33
:1093200006D80123934013F0EE0F11D1DB0614D4BD
:109330000F4B01930F4B00930F4A104B10491148EC
:10934000F7F736FF404080F311884FF0040002DF4A
:109350002146F9F702FE4046D7E7C288D6F8140244
:10936000FC21F9F70FFE3946F3E700BFD40C0020CB
:10937000B8BA000000BB0000C5BA00004AC4000033
:1093800072BA00000ABA0000914210B5144B19D10C
:10939000D3F85422D3F85042944211D1002914BF7B
:1093A0000A460322013AD2B203EB420483F8852233
:1093B00093F88422A4F87E0291420FD083F885129C
:1093C000012010BD29B9B3F88232181A18BF012044
:1093D00010BD03EB4103B3F87C32F6E7002010BD6B
:1093E000A00A002030B4144B93F886220D4602B335
:1093F00093F88422D1B293F8852235B14FF6FF73EA
:10940000984216D030BCFFF7BFBFD3F85002D3F854
:109410005442A0420DD191420BD0D3F8544283F86C
:109420008512A04205D093F88402814208BF83F8D8
:109430008522002030BC7047A00A002038B50B4CB4
:10944000D4F84021D4F8445122B10020C4F840019E
:10945000FAF7C8FF2DB10023C4F844310120FAF710
:10946000C1FF0020BDE83840F9F7A4BC00B00040BF
:109470000120F9F79FBCFAF7DBB9684620F0070135
:109480008D4601B5F9F768FE00F0E2FD00F0DCFB67
:10949000BDE8014085467047012907B50FD00E4B46
:1094A00001930E4B00930E4A0E4B0F490F48F7F7EE
:1094B0007FFE404080F311884FF0040002DF182047
:1094C00022B103B05DF804EB00F07EBD03B05DF89F
:1094D00004EB00F087BD00BFB8BA000000BB00007D
:1094E000C5BA00009ECD000072BA00000ACE00008E
:1094F00007B529B90B2003B05DF804EB00F080BD7F
:10950000012901D11820F6E7074B0193074B00937F
:10951000074A084B08490948F7F74AFE404080F3DC
:1095200011884FF0040002DFB8BA000000BB000051
:10953000C5BA0000AFCD000072BA00000ABA000040
:1095400088420AD018B94B1E58425841704701282A
:1095500005D1B1FA81F04009704701207047002021
:109560007047000007B50F4B89B1012916D00E4B8B
:1095700001930E4B00930E4A0E4B0F490F48F7F71D
:1095800017FE404080F311884FF0040002DF4FF4D3
:109590000062C3F8002103B05DF804FB4FF0807255
:1095A000F7E700BF00E100E0B8BA000000BB000030
:1095B000C5BA0000C1CD000072BA00000ABA0000AE
:1095C00070470000014B186801F0F0BCF412002055
:1095D000F0B5384B87B0186008213748FAF7C0F863
:1095E000364800F0ABFE18B96FF0120007B0F0BDBE
:1095F000436801211B689847F9F70CFDF9F73AFB1E
:109600002F4B08221A7003221A7200242D4A1C7450
:1096100002270D251F76072102928DE828002A4A8D
:1096200004232046FAF78CFE284800F087FE002825
:10963000DAD0274B03934FF4F8761B230293019360
:1096400022460496009701230721FFF717FB0446E3
:1096500070B1204B0393204B0190009302961F4B57
:109660001F4A20492048F7F7A3FD6FF00B00BDE724
:1096700002460146012000F0D1FC224621460B2083
:1096800000F0CCFC22462146182000F0C7FC224600
:109690000121284600F0C2FC012000F095FC0B20BF
:1096A00000F092FC182000F08FFC284600F08CFCA3
:1096B00020469BE7F4120020940F0020B8B600006B
:1096C000D4120020981000209C0F0020C3B6000088
:1096D000300D0020B8BA000000BB0000CDCD000066
:1096E000C5BA000072BA0000D5CD000008B50B461F
:1096F00038B121B1062207491846F7F769FB05483A
:1097000008BD21B1062204491846F7F761FB02485B
:1097100008BD00BF8B0F0020850F0020062210B16E
:109720000248F7F755BB0248FBE700BF8B0F00204C
:10973000850F00202DE9F34106248DF80240022414
:109740008DF803400D463E4C01211F4600238D42FB
:109750008DF801108DF804108DF800309DF824105C
:1097600008BF2380E37818BF208061F30203E37011
:10977000A1789DF8283063F3871102AB1D4415F8DA
:10978000083C63F3030162F304110A466FF34512C8
:10979000A270FFF72BFB90F84F5005EB8503C5EB4C
:1097A000C305A378425D63F3030202F0CF02C3F363
:1097B000001363F386124255A27802F00F03012BC7
:1097C000064600EB050835D167F34512A2700899EB
:1097D0001C480622F7F7FCFA0622089908F108004F
:1097E000F7F7F6FA0C2388F80130A378725DC3F31B
:1097F000401363F3C7127255FFF7FCFA90F84F203D
:1098000002EB8203C2EBC3020421835C61F3030316
:10981000A17803F0CF03C1F3001161F386136FF356
:10982000C713851883546B780BB906236B7002B08D
:10983000BDE8F08198F80130002BD6D10623D2E79D
:10984000F8120020021300202DE9F843074688464D
:10985000FFF7CCFA90F84F4090F84E30A3420546FF
:1098600004D10134E4B2022C08BF002404EB8402CA
:10987000C4EBC202DFF86890AB5C99F8021061F3A8
:10988000030303F0CF03C1F3001161F3861399F8CA
:109890000210C1F3401161F3C713AE18AB5409F1C4
:1098A00004010622B01CF7F793FA99F8023003F08E
:1098B0000F03012B06F108000AD1062209F10A0163
:1098C000F7F786FA0C23737085F84F40BDE8F883EC
:1098D0003A4641460637F7F77BFA7770F4E700BF60
:1098E000F81200202DE9F04106460F46FFF782FAF4
:1098F00090F84F4090F84E30A342054604D1013411
:10990000E4B2022C08BF002404EB8402C4EBC202C0
:109910000421AB5C61F303030F49887803F0CF03A4
:10992000C0F3001060F3861305EB02086FF3C71352
:10993000AB54B31D88F801300622043108F102004F
:10994000F7F746FA3246394608F10800F7F740FAC9
:1099500085F84F40BDE8F081F812002070B518B9C5
:10996000BDE87040FFF7F0BBFFF740FA0646FFF78F
:1099700041FA96F84F20134C02EB8203C2EBC3026C
:1099800090F84F30164403EB8302C3EBC203C518B3
:10999000A078211DC0F30010FFF7A8FE211D0622AC
:1099A000B01CF7F715FA211D0622A81CF7F710FACC
:1099B000A278E1782088920901F00701BDE87040A3
:1099C000FFF77EBAF812002070B504464FF020036E
:1099D000EFF3118583F31188C38A4BB3828A9A42CD
:1099E0000FD9002101F0EEF858B185F31188012359
:1099F0000371002343710360038200F11403C36009
:109A00001CE0E68A731EE38285F31188218B608B4C
:109A1000A38A0330CA1C22F0030220F00300104482
:109A2000226A14309B1B03FB002084604182DEE726
:109A300085F3118801F0C6F80028D8D170BD70B543
:109A4000064601F0BFF8054628B10446637913F0D5
:109A5000010302D12360284670BD0021304601F089
:109A6000B1F86379206023F0010363710446EDE7E8
:109A700000F114031944C160704710B40A46146819
:109A800014B910BC01F058B8537943F00103537175
:109A90002246F4E710B5014601B910BD0B790C68F8
:109AA000013BDBB20B71002BF7D188680B60C369F7
:109AB0001BB1084698472146EEE701F039F8FAE76E
:109AC00003790133037170478388026819448180E8
:109AD000D018704730B4838804689D188580E018DA
:109AE00030BCF7F775B98388026810B55C1C8480B8
:109AF000D154D01810BD83885B1A83800368194441
:109B000001600846704708B5036801211A78FFF71D
:109B1000F2FF104608BD00F108030068C01A704744
:109B20000C4B1B78062B12D10B4B186810F00F0052
:109B30000DD104331B6803F0F003302B08D1074B21
:109B40001B6813F0F00F0CBF0120002070470020AD
:109B5000704700BFE00F00F0E40F00F0EC0F00F0E2
:109B600008B54FF02003EFF3118183F31188FFF75D
:109B7000D7FF20B12D4AD36823F08073D360FFF75D
:109B8000CFFF10B12A4B03221A60FFF7C9FF30B193
:109B90004FF080430022C3F80C21C3F810214FF08E
:109BA0001023D3F80022002A03DBD3F80032002B65
:109BB0002FDA204B0122C3F80425D3F80024002A11
:109BC000FBD04FF010221521C2F80012D3F8002468
:109BD000002AFBD04FF010231522C3F80422154BA6
:109BE0001A46D3F800140029FBD00021C3F804154D
:109BF000D2F80034002BFBD0BFF34F8F0E490F4B30
:109C0000CA6802F4E0621343CB60BFF34F8F00BF1A
:109C1000FDE7094B4FF0FF329A62DA62084B094ABE
:109C20001A6081F31188002008BD00BFF0ED00E04C
:109C3000A005004000E0014000ED00E00400FA054E
:109C4000B00200200090D00300B501F055F95DF896
:109C500004EB00BF064881684A897F2A06D88069DC
:109C6000884203D003494FF080520A6070470000D9
:109C7000DC13002004ED00E0044800232021C2187A
:109C80000133272B82F80013F9D1704700E100E07F
:109C90000E498A6828201044EFF3098C80E8F01FF1
:109CA0000B4F4FF00066202080F311888A698A608C
:109CB0003E60106E0023136680F3118802F12800C5
:109CC00090E8F01F8CF3098870470000DC13002037
:109CD00004ED00E01EF0040F0CBFEFF30880EFF37B
:109CE0000980816931F8021C11F0FF0101D00229BD
:109CF00007D0404080F3118804494FF080520A6039
:109D0000704700B500F030FA00BD000004ED00E03F
:109D100004498A68106604490968516600DF506E7C
:109D200070470000DC13002098D2000010B50446F4
:109D300001F0B8F822680146BDE810400148F7F785
:109D400037BA00BF9FCF000010B504461A48F7F796
:109D50002FFA04F11800194CFFF7E8FFA36A9A01E3
:109D600002D51748F7F724FAA36ADB0102D5154894
:109D7000F7F71EFAA36A180302D51348F7F718FA83
:109D80000E4CA36A590302D51048F7F711FAA36ADB
:109D90009A0302D50E48F7F70BFAA36ADB0302D544
:109DA0000C48F7F705FA054A936A6FEA03436FEA2E
:109DB0001343936210BD00BF70D0000000ED00E0BF
:109DC00089D000009DD00000B8D00000D7D000009E
:109DD000FDD0000018D1000038B5044617480D46E4
:109DE000F7F7E6F904F11800154CFFF79FFFA36A97
:109DF000DB0604D51348BDE83840F7F7D9B9A36AA4
:109E0000180701D51048F6E7A36A99070FD50F4840
:109E1000F7F7CEF9A36A1A060ED5616B0C48F7F76F
:109E2000C7F94DB1A36A23F08003A36238BDA36ACA
:109E3000DB0701D50748DEE738BD00BFE9CF0000EA
:109E400000ED00E000D0000012D0000026D000009D
:109E50003FD0000050D0000038B504461B480D46E6
:109E6000F7F7A6F904F11800194CFFF75FFFA36A92
:109E7000D90404D51748BDE83840F7F799B9A36A63
:109E80001A0501D51448F6E7A36A9B0514D51348B3
:109E9000F7F78EF9A36A180408D5A16B1048F7F7F5
:109EA00087F91DB1A36A23F40043A362084B9B6AA0
:109EB000590509D50B48DEE7A36A5A05FAD4A36A07
:109EC000DB0501D50848D6E738BD00BF66CE0000E7
:109ED00000ED00E000D0000012D000007DCE0000B8
:109EE0003FD0000097CE0000B3CE000038B5274D1C
:109EF0006B68C3F30803DA1E0446092A3AD8DFE880
:109F000002F00533352F3939393939372048F7F719
:109F10004FF9EB6A9A0703D51E48F7F749F90CE0A9
:109F2000EB6A5B0009D51C48F7F742F91B4B1B781D
:109F30004BB101212046FFF74FFF21460020BDE82D
:109F4000384000F015B9164B1B7823B1012120468B
:109F5000FFF782FFF1E7134B1B889BB2002BECD07D
:109F60002046FFF7F1FEE8E70021E3E70021EEE7F6
:109F70000D48D2E70D480E49A3F110020F2BD8BFB0
:109F800001460C48F7F714F9D7E700BF00ED00E0F1
:109F9000FACE000012CF000034CF000028ED00E020
:109FA00029ED00E02CED00E054CF0000CCCE000005
:109FB000E1CE00008BCF0000024A536943F010034A
:109FC0005361704700ED00E043B2012200F01F0032
:109FD00002FA00F05B09024A42F82300704700BF12
:109FE00000E100E043B201225B0900F01F0002FA29
:109FF00000F02033014A42F82300704700E100E0FE
:10A000004209054B00F01F0053F82220012303FAF8
:10A0100000F01040704700BF00E100E043B2002BA9
:10A02000A8BF03F1604301F101014FEA4111BBBF39
:10A0300000F00F00044B03F56143C9B2AABFC9B2D7
:10A04000195483F80013704714ED00E000F046B88F
:10A0500008B572B6044B586918B100225A6100F075
:10A0600087F962B608BD00BFDC1300202DE9F0417E
:10A070008D18884617461E4604220A9B09990446F5
:10A0800001F010FA0E48C4F8588025F00702A2F13A
:10A090002003002120F00100E1642165E76542F81A
:10A0A000080C42F8206C069A5A60079A9A60089A3F
:10A0B000DA604FF08072DA61A3642166BDE8F08156
:10A0C00061B30000014910220A60704710ED00E002
:10A0D000404080F3118830BF704700BF404080F39C
:10A0E0001188DFF81CC0DCF800C01CF4006C0CBF49
:10A0F000EFF30880EFF3098000B5FFF7F7FE00BD2E
:10A1000004ED00E038B5431E04460D46042B1AD872
:10A11000DFE803F00319131517000D48F7F748F8A7
:10A1200000F0C0FEAA6901460A48F7F741F829463F
:10A130002046BDE8384000F01BB80748EEE7074866
:10A14000ECE70748EAE701460648F7F731F8E7E7A2
:10A1500044D10000ECD100006ED1000094D1000089
:10A16000AED10000C9D1000001460068FFF7CABFA8
:10A17000052810B50CD001F0DBF860B101F0D8F87B
:10A180000C4B0D49002808BF19460C48F7F710F88A
:10A19000FFF79EFFFCE701F0DBF80028EED1084C4A
:10A1A0000848A168F7F704F8A068BDE8104000F07F
:10A1B0000BB800BF2CD2000028D200003DD2000016
:10A1C000DC1300205DD2000038B505464FF02003B7
:10A1D000EFF3118483F3118801F0F4F80B4B9B68C3
:10A1E0009D420DD10A4B5A68C2F3080222B900F011
:10A1F00083FE2046FFF78CFD5A6842F080525A6079
:10A200002046BDE8384000F0DDBD00BFDC13002073
:10A2100000ED00E000B572B60B4A506900281EBF81
:10A220000021516100F0A4F862B6EFF30580A0F1BF
:10A2300010004FEAC0000549014409C998475DF87C
:10A2400004EBFFF701BD0000DC130020DC00000080
:10A25000202080F3118805484FF40061401880F3F6
:10A260000988022080F3148800F006B864290020D1
:10A2700030BFFFF7FDBF00BF08B5074B074A23F00B
:10A280007F039360BFF34F8FBFF36F8F00F0A0F891
:10A2900000F0A8F800F0C6F80000000000ED00E0B3
:10A2A00008B5FFF7E5FFBDE80840FFF7D3BC0000A5
:10A2B000154B16491A6830B50D68C2F3072295424E
:10A2C0000FD8002248685A60954200F10C000AD16C
:10A2D00005225A600E4B01221A70BFF34F8FBFF355
:10A2E0006F8F002030BD50F80C1C50F8044C9A6061
:10A2F00021F01F0141F01001114344F00104D96025
:10A3000001321C61E0E700BF90ED00E0B4020020E4
:10A310000813002038B5084B53F82040013053F89B
:10A3200020502046A84204F10C0400D338BD54F854
:10A330000C3C5B689847F4E784D2000070B50A4C87
:10A340000A4D0646AC4201D100240AE063680BB90D
:10A350000C34F7E7236830461968F6F717FD002834
:10A36000F6D1204670BD00BF000300207803002016
:10A37000431C03D0034B1B68984201DBF6F71EBA5F
:10A38000704700BFF80200200F4D80B50F4F05F158
:10A390000C064FF02002EFF3118382F31188EB6873
:10A3A000B3420AD04BB11C69631C08D03B68A3427E
:10A3B00005DD6C61FFF78CFEEBE74FF0FF342046C4
:10A3C000F6F7E8F9F5E700BFDC130020F8020020FB
:10A3D0000248034A0021121AF6F726BDB8030020EE
:10A3E000641600200248034A0349121AF6F7F0BC2B
:10A3F00000000020B4030020A0D2000008B5022015
:10A40000FFF788FF0320FFF785FF01F001F8F6F75B
:10A41000CFF8034A137A23F00103137208BD00BF7B
:10A420007413002080B586B0324D06AFFFF724FCD0
:10A4300020235A195A510833B3F5907F5260F8D14E
:10A440002D4EDFF8DC80AE6100244FF00109434659
:10A450004FF480622949CDF810903046039402945D
:10A4600001940094FFF702FE737A304623F0040350
:10A47000737200F0F5FB0F2303932149CDF8109080
:10A480000294019400941F4B1F484FF4A072FFF7F1
:10A49000EDFD1D4B1C4A5B7A23F0040353721046FA
:10A4A00000F0DEFB194BEB602B61194B83F308883E
:10A4B000184BE02283F82220DC771C765C769C76B1
:10A4C0005A6A42F4E0225A62FFF776FDFFF7FAFD7E
:10A4D0002046FFF71FFF4846FFF71CFF0E4BAE60FC
:10A4E00023F007030D4A83F30988002181F31188C3
:10A4F00040461047DC130020741300202424002061
:10A500002428002089A300000C130020E813002059
:10A510006431002000ED00E02428002061B3000039
:10A52000FDA3000038B590F90A308B4204460D4671
:10A530000ED0437ADB060AD1036A013307D100F05B
:10A54000B5FBA5722046BDE8384000F089BBA57276
:10A5500038BD000070B5304A0D469168CB7A013B9A
:10A560000446CB72C36811464BB180689268904232
:10A5700011D095B900F040FC6FF00F0070BD9268EB
:10A5800092F90A2022610133E3608B68A36000F036
:10A5900033FC002070BD2269F4E792F90A1090F9AB
:10A5A0000A309942A8BF194621EAE1714FF0200311
:10A5B000EFF3118683F31188A06890F90A3099426D
:10A5C00001DAFFF7AFFF2046294600F0D5FB00F087
:10A5D00093FC3046FFF79CFB0028D8D02368216904
:10A5E0009C4208BF002333B193F90A309942A8BFB7
:10A5F000194621EAE1714FF02003EFF3118583F34F
:10A600001188A068FFF78EFF85F3118800F0F4FB36
:10A610006FF00A0070BD00BFDC130020F8B5344EA7
:10A62000B268D37A013B0546D372C368013BC3606D
:10A630001BB1BDE8F84000F0DFBB4FF02003EFF3A3
:10A64000118783F3118801698068FFF76BFF294B3D
:10A650002C681B6883B1A54208BF002424B987F386
:10A6600011880023AB60E4E7236A023308D16B68EA
:10A670009C42F4D02468F1E7A542F0D0002CEED043
:10A6800094E80C001A6022685360637A216A23F010
:10A69000020363724B1C04F110020ED033699A421C
:10A6A0001FBF226913695B181361636922691A600D
:10A6B000226953604FF0FF332362637A23F0040270
:10A6C00013F01B0F627202D1236A01330BD087F3A0
:10A6D000118800236366EB68AC600133EB6094F98A
:10A6E0000A302B61A5E7204600F0BAFAEFE700BF79
:10A6F000DC130020D81500200C2310B503FB01004B
:10A700000024002900DA10BD4379046003F00F0330
:10A71000022B06D0042B04D0012B04D183681C60CB
:10A7200001E083681C6182F311884FF02003EFF38E
:10A73000118283F3118801390C38E2E7F8B5002360
:10A740001360036807460E461546002B49D018686B
:10A75000437A23F0200242729A0742D5036A0233F9
:10A760004BD090E80C001A6002685360437A016A8B
:10A7700023F0020343724B1C00F110020FD0204B58
:10A780001B699A421FBF026913695B181361436911
:10A7900002691A60026953604FF0FF3303620023BD
:10A7A0004366437A13F01F041BD1036A013318D1A7
:10A7B00000F056FAEFF305830D2B1CD823B1114B93
:10A7C000586810F400600BD00D4B9B685B897F2BA1
:10A7D00001D9002004E000F0DFFA003018BF0120AA
:10A7E00028607B68C3F30432164366F310330020FD
:10A7F0007B603860F8BD2046F2E76FF00A00F8BDD4
:10A80000DC13002000ED00E02DE9F04F87B080461A
:10A8100001914FF02003EFF3118583F311885F4816
:10A820008468637A43F02003637285F3118806AF6E
:10A83000836847F80C3D002543462C464FF0FF3611
:10A840004FF0010A01998D4211DB4FF02003EFF325
:10A85000118583F3118881684B7A980667D42A465C
:10A8600031464046FFF748FF85F3118867E04FF017
:10A87000200EEFF311898EF3118893F805E00EF0A6
:10A880000F0EBEF1020F0ED0BEF1040F2BD0BEF1A1
:10A89000010F0ED19968D1F804C0BCF1000F08D0A7
:10A8A0004FF0020B64E09968D1F808C0BCF1000FCA
:10A8B0005CD1BAB3D0F808C09CF809B01BF0200FE7
:10A8C00030D07CBBBEF1020F16D0BEF1040F13D006
:10A8D000BEF1010F17D1D3F808E0DEF80010A9B9D6
:10A8E000CEF800300FE09968D1F808C0BCF1000F35
:10A8F000DFD04FF0080B3BE0D3F808E0DEF8101093
:10A9000021B9CEF810301F6001360BE05C686AF3A5
:10A9100010345C609CF8094024F020048CF8094055
:10A920006FF02F0489F3118801350C338AE723F087
:10A9300020034B723AB985F311886FF00A04204660
:10A9400007B0BDE8F08F04A811460490059000F010
:10A9500013FA00F0D1FA2846FFF7DAF904464FF06F
:10A960002003EFF3118583F3118878E74FF0040B90
:10A97000D3F804E0CEF3043C4BEA0C0C6CF3103E2D
:10A98000C3F804E0D0F808C0002119609CF809E081
:10A990002EF0200E8CF809E0C4E700BFDC13002085
:10A9A00007B50346002200681A6001AAFFF7C6FE39
:10A9B000019803B05DF804FB427A22F0040112F022
:10A9C0001B0F417204D1036A013301D100F048B971
:10A9D000704703691BB108211030FFF7E1BF18462B
:10A9E000704710B5044600F087FA2046BDE81040D5
:10A9F000FFF78EB908B5064B9B685B897F2B05D89E
:10AA000000F0CAF9003018BF012008BD002008BDC1
:10AA1000DC130020104A1268034600686AB18342C2
:10AA200008BF002008B900207047026A023207D12F
:10AA30005A689042F7D00068F4E783420AD050B1D8
:10AA400090E80C001A6002685360437A23F0020316
:10AA50004372704710467047D815002003695A1C8E
:10AA600011D00A4A126990421FBF01680A699B18F7
:10AA70000B6190E80C001A60026853604FF0FF33DE
:10AA80000361002070471846704700BFDC130020A8
:10AA900000238360C3600060406003617047000072
:10AAA000F8B5054614464FF02003EFF3118783F302
:10AAB0001188FFF7AFFF0646A0B11030FFF7CEFFB9
:10AAC0003046FFF779FF00237366F460EFF30583E8
:10AAD0000D2B23D81BB1134B5B681B051ED5FFF74D
:10AAE00089FF11E031B9AB682360EB68AC6043B912
:10AAF000EC6006E00B68236073B9EB6853B9EC6057
:10AB0000AC602846FFF765FF40B13846BDE8F84025
:10AB1000FFF767BF1C60EBE70C60F2E787F3118873
:10AB2000F8BD00BF00ED00E00A46C168FFF7B8BFFE
:10AB30000A460021FFF7B4BF2DE9F04704460D4651
:10AB400091464FF02003EFF3118883F311880768D3
:10AB50004FF0000AB84208BF00274DB12046FFF76A
:10AB600059FF064688B9E368DBB9A560C4F80C90C4
:10AB7000CFB1EFF305830D2B1ED81BB1104B5B68D3
:10AB80001B0519D5FFF736FF10E006F11000FFF79F
:10AB900065FF3046FFF710FFF560C6F864A02D682A
:10ABA000DBE71D60E2E72046FFF713FF20B14046D8
:10ABB000BDE8F047FFF715BF88F31188BDE8F087BF
:10ABC00000ED00E038B54FF02004EFF3118584F379
:10ABD000118884684CB1C168226882608C4208BFC9
:10ABE000C26085F31188204638BD19B985F31188F4
:10ABF000084638BD00F0C0F82846FFF7F2FE0028EE
:10AC0000F1D1024B9B68D86838BD00BFDC1300202F
:10AC100030B5CA60114A886010460B6150F80C3F8D
:10AC200083420CD1086013694B601369196011618C
:10AC300030BD641B0C611469A342F3D01B68002B68
:10AC4000F0D00C691D69AC42F3DC5A682C1B1C6106
:10AC50004A600B605A681160596030BDDC130020F7
:10AC600030B590F90A30104C03F110014A11063248
:10AC700004EB820201F01F050121A940556814333D
:10AC800004EBC3032943516003605A6842605A6869
:10AC900010605860A36990F90A1093F90A20914254
:10ACA000A8BF1846A06130BDDC13002090E80A0060
:10ACB00010B590F90A201960016814324B60144BEA
:10ACC00003EBC20153F832208A420FD190F90A10E7
:10ACD00010314A11063203EB8202012401F01F01F8
:10ACE00004FA01F1546824EA010454609A6990421C
:10ACF0000BD1D96991FAA1F20029B2FA82F208BF08
:10AD00004FF0FF32043253F832209A6110BD00BF79
:10AD1000DC13002030B40C68A14208BF002434B911
:10AD200001604B6843604B68186048600BE090F925
:10AD30000A5094F90A309D4216DA63684360046051
:10AD4000636818606060437A43F002034372531CE7
:10AD50000FD009320A2330BCB2FBF3F30A460133A9
:10AD600000F11001FFF754BF4B689C42D8D0246813
:10AD7000D5E730BC7047000070B5064C0E4605465E
:10AD8000A068FFF793FF32462946A068BDE87040EF
:10AD9000FFF7C0BFDC130020094AD169926800297F
:10ADA00091FAA1F392F90A00B3FA83F308BF4FF0C6
:10ADB000FF33103B9842D4BF00200120704700BFF2
:10ADC000DC13002010B50A4B9B685B897F2B04467F
:10ADD00002D8FFF7E1FF10B984F3118810BD054BCD
:10ADE00000222046BDE810401A60FEF791BF00BF68
:10ADF000DC130020DC1500204FF02003EFF311805E
:10AE000083F31188034B9A68D37A0133D372FFF727
:10AE1000D9BF00BFDC13002010B590F90A30114AE9
:10AE2000143302EBC303596888421AD0416804689E
:10AE30000C6004686160036059684160596808608B
:10AE40005860936998420BD1D16991FAA1F3002916
:10AE5000B3FA83F308BF4FF0FF33043352F83330B3
:10AE6000936110BDDC13002038B54FF02003EFF3E1
:10AE7000118583F31188094CA068FFF7CDFFA26804
:10AE8000A3699A4202D185F3118838BD044B002290
:10AE90001A602846BDE83840FEF73ABFDC130020B0
:10AEA000DC150020014B9868704700BFDC130020C0
:10AEB0000D4B1B68002B14DD0C4B1B68984210D007
:10AEC0000B4A90F90A30126893420ADB094A14339C
:10AED00002EBC30152F833004B68C01A18BF0120BF
:10AEE00070470020704700BFFC1400209CD2000077
:10AEF00000150020DC130020014B00221A6070476F
:10AF0000DC150020427A22F0040112F01B0F41727E
:10AF100004D1036A013301D1FFF7A2BE70470000DC
:10AF2000104A1268034600686AB1834208BF0020D5
:10AF300008B900207047026A023207D15A6890426D
:10AF4000F7D00068F4E783420AD050B190E80C00D3
:10AF50001A6002685360437A23F002034372704719
:10AF600010467047D815002003695A1C11D00A4AB0
:10AF7000126990421FBF01680A699B180B6190E833
:10AF80000C001A60026853604FF0FF330361002029
:10AF900070471846704700BFDC1300200023816013
:10AFA000C2600060406003617047000070B50446F5
:10AFB0004FF02003EFF3118683F31188FFF7B0FF02
:10AFC0000546A0B9A368E2689A4218BF0133A3609E
:10AFD000236943B3042104F11000FFF7E1FC10B32F
:10AFE000FFF78AFF3046BDE87040FEF791BE103093
:10AFF000FFF7BAFF2846FFF785FF00236B66EFF3E4
:10B0000005830D2B0FD81BB1084B5B681B050AD5B8
:10B01000074B9B685B897F2B05D8FFF7BDFE00308F
:10B0200018BF0120DBE786F3118870BD00ED00E05A
:10B03000DC13002038B54FF02003EFF3118483F3C5
:10B04000118883682BB1013B836084F31188002051
:10B0500038BD21B984F311886FF00F0038BDFFF7B8
:10B060008BFEFFF749FF2046BDE83840FEF750BE93
:10B070002DE9F34706464FF02003EFF3118083F3E9
:10B0800011885A49D1E90045A21945EBE673C1E997
:10B09000002380F311886846CDF800D0CDF804D0A5
:10B0A0004FF02003EFF3118483F31188504D2A46AB
:10B0B000214652F80C3F9342944600D0FBB984F3EA
:10B0C0001188A868FFF7F4FEB0B14A4B1A680A204D
:10B0D00006FB0020484A1860126890420CDB0022F0
:10B0E0001A604FF02003EFF3118483F31188A868EE
:10B0F000FFF792FE84F3118802B0BDE8F0871C6967
:10B100003E4FA41B1C6101243C606FF001041A69CE
:10B11000D2B993E80440CEF800201A68C2F804E0DF
:10B12000009A1A60009A5860009353601C6181F382
:10B1300011884FF02003EFF3118183F31188EB683E
:10B14000634501D0002BE2D181F31188009B83423B
:10B1500002D100233B60B4E7002BFAD0019A93425E
:10B1600014BF1C6800244FF0FF384FF0000993E82B
:10B170000600116019684A6098684FF02002EFF3EA
:10B18000118A82F31188C3F8108008B3DB6853B1C9
:10B1900042680368136003685A60437AC0F81C90E1
:10B1A00023F002034372437A23F0040213F01B0FCF
:10B1B000427202D1036A013312D08AF31188002C43
:10B1C000C7D0019BA3420ED0226823461446CEE787
:10B1D0008AF311885A69002AF1D018469047EEE7A1
:10B1E000FFF73EFDE9E70022EFE700BFE015002092
:10B1F000DC130020DC150020FC140020D8150020F2
:10B2000008B54FF480624FF0FF330349034800F064
:10B2100073F9002008BD00BF64310020E81500204C
:10B22000437ADA0604D1006A431C584258417047F9
:10B230000020704710B501464FF02003EFF3118452
:10B2400083F31188437A23F004034372FFF7E8FF86
:10B2500010B984F3118810BD0846FFF701FD084BB3
:10B260009B685B897F2BF4D8FFF796FD0028F0D010
:10B27000FFF742FE2046BDE81040FEF749BD00BF83
:10B28000DC13002003695A1C11D00A4A126990424B
:10B290001FBF01680A699B180B6190E80C001A60D7
:10B2A000026853604FF0FF33036100207047184677
:10B2B000704700BFDC130020F0B54FF02003EFF320
:10B2C000118683F31188194A80610A230931B1FB81
:10B2D000F3F10131016211460023C36151F80C3FC3
:10B2E0008B4200F1100507D10161136943611D60B4
:10B2F000156186F31188F0BD002BF5D0D2F810E06F
:10B30000046A1F69BC4208DC5A683C1B1C6142612C
:10B3100003615A6815605D60EBE7E41B73450462E6
:10B32000E2D01B68002BEBD1DEE700BFDC1300206E
:10B33000EFF305800D2807D838B1044B586880F426
:10B340000060C0F3C02070470120704700ED00E0AE
:10B35000024B9B68187A00F001007047DC13002054
:10B3600008B50446084611461A46A047FFF7F0FF05
:10B3700028B1404080F311884FF0010002DF024BFA
:10B380009868FEF721FF00BFDC13002070B586B07F
:10B3900004460E9E04960D9E03960C9E02960B9EEE
:10B3A0000F9D01960A9E0096FEF760FE2DB920467D
:10B3B000FFF740FF204606B070BD29462046FFF744
:10B3C0007BFFF7E7036D10B5044603B198472046AD
:10B3D000FFF726FF38B12046FFF768FC637A43F099
:10B3E0000803637210BD637A9B0708D594E80C00CC
:10B3F0001A6022685360637A23F002036372236A3F
:10B400000133EBD004F11000FFF73CFFE6E700004A
:10B41000F0B5214F214D87B03E46BD4205F13004C5
:10B4200014D31F4B9A68D37A013BD3724FF0200399
:10B43000EFF3118583F31188184CB4421FD385F3C1
:10B44000118807B0BDE8F040FFF7D6BC54F8103CB7
:10B45000049354F8143C039354F8183C029354F8A2
:10B460001C3C019354F8203C0093A4F130000FC819
:10B47000FEF7FCFD54F8303CDD642546CDE7616AFB
:10B480004B1C03D0206819B9FFF7D4FE3034D4E741
:10B49000FFF712FFFAE700BF7803002078030020CF
:10B4A000DC1300200372427200234FF0FF328172DE
:10B4B000C3720262C36183614362704710B5044680
:10B4C0004FF0FF312046FFF77DFB0346083342680B
:10B4D000BFF35B8F53E8001F21F0010E43E800EC3F
:10B4E000BCF1000FF6D1BFF35B8FCB0700D59047BF
:10B4F000FFF7BAFCE4E70000F0B587B004461F464A
:10B500000D461646FFF7C4FA0020059004900290FD
:10B51000019003970094044B3246294604F114002D
:0EB52000FFF734FF07B0F0BDBDB40000704768
:08B530003C4DFF7F010000000B
:10B5380027B600001106000000000000A0B60000B9
:10B5480085060000D0B60000A7B60000E907000095
:10B5580000000000B1B600009309000024B7000005
:10B56800B8B60000650B000000000000C3B600007C
:10B57800650B00000000000027B60000692A0000E3
:10B588000000000027B60000619B000000000000DA
:10B5980027B60000B1A200000000000027B6000096
:08B5A80001B2000000000000E8
:10B5B00069BD00006EBD000072BD000076BD0000D8
:10B5C0007ABD00007EBD000082BD000086BD000087
:10B5D0008ABD00008EBD000000FFFFFFFFFFFF00DF
:10B5E000112233445566778899001122334455005F
:10B5F0000101000000000020030200000100002003
:10B600001613000003000020426C7565746F6F74A0
:10B610006820696E6974206661696C6564202865BC
:10B620007272202564290A00426C7565746F6F740C
:10B630006820696E697469616C697A65640A0041A1
:10B6400064766572746973696E67206661696C659A
:10B650006420746F20737461727420286572722084
:10B660002564290A00426561636F6E2073746172FC
:10B670007465640A005374617274696E6720426570
:10B6800061636F6E2044656D6F0A0000090B000056
:10B6900094B600005465737420626561636F6E0038
:10B6A000554152545F30007379735F636C6F636B05
:10B6B000004750494F5F3000636C6B5F6B333273F0
:10B6C000726300636C6B5F6D3136737263000000F0
:10B6D000002000400024F4002D0600004D0600006C
:10B6E00069060000000000000002000000000000E9
:10B6F0000006000000010000000300000000000040
:10B700000007000000000000000000000000000032
:10B710000000000000040000000500000000000020
:10B7200000000000000000500000005000600040D9
:10B730000D0A0000B308000093080000D5080000BF
:10B74000190900005909000000000000C90C0000A0
:10B7500000000000000000007D0B0000090B00004D
:10B760000000000030313233343536373839616209
:10B7700063646566006863695F636D645F646F6ED0
:10B7800065006863695F6C655F6D6574615F6576B0
:10B79000656E74006863695F6576656E74007365D5
:10B7A0006E645F636D640070726F636573735F6571
:10B7B00076656E7473006863695F74785F7468722D
:10B7C000656164006C655F696E6974007365745FC0
:10B7D0007374617469635F616464720073686F7726
:10B7E0005F6465765F696E666F006863695F696E46
:10B7F00069740062745F726563760062745F72657B
:10B8000063765F7072696F0062745F656E61626C0F
:10B8100065005B25735D25732025733A2025734EE3
:10B820006F204843492064726976657220726567AB
:10B830006973746572656425730A005B25735D2501
:10B84000732025733A202573484349206472697632
:10B850006572206F70656E206661696C6564202872
:10B8600025642925730A005B25735D2573202573E4
:10B870003A202573556E61626C6520746F20736584
:10B880006E6420746F206472697665722028657218
:10B89000722025642925730A005B25735D257320BA
:10B8A00025733A202573546F6F20736D616C6C2083
:10B8B0007573657220646174612073697A6525739C
:10B8C0000A005B25735D25732025733A2025735587
:10B8D0006E68616E646C6564204C45206576656EAB
:10B8E0007420307825303278206C656E2025753ACA
:10B8F00020257325730A005B25735D25732025734E
:10B900003A202573556E68616E646C6564206576B7
:10B91000656E7420307825303278206C656E202575
:10B92000753A20257325730A005B25735D25732006
:10B9300025733A202573496E76616C6964206275BF
:10B9400066207479706520257525730A005B257360
:10B950005D25732025733A202573617373657274B6
:10B960003A20272162745F6863695F6576745F6956
:10B97000735F7072696F286864722D3E65767429F2
:10B9800027206661696C656425730A005B25735D19
:10B9900025732025733A2025736173736572743A99
:10B9A000202762745F6275665F6765745F74797083
:10B9B000652862756629203D3D2042545F42554608
:10B9C0005F45565427206661696C656425730A00DB
:10B9D0005B25735D25732025733A2025736173738E
:10B9E0006572743A20276275662D3E6C656E203E46
:10B9F0003D2073697A656F66282A6864722927205A
:10BA00006661696C656425730A005B25735D257347
:10BA10002025733A2025736173736572743A202769
:10BA20003027206661696C656425730A005B2573A5
:10BA30005D25732025733A202573617373657274D5
:10BA40003A202762745F6863695F6576745F697323
:10BA50005F7072696F286864722D3E65767429275D
:10BA6000206661696C656425730A00205B57524E3D
:10BA70005D006274005B25735D25732025733A2099
:10BA800025734F70436F64652030782530347820FB
:10BA9000636F6D706C6574656420696E7374656145
:10BAA00064206F6620657870656374656420307803
:10BAB0002530347825730A001B5B306D001B5B302A
:10BAC0003B33336D00205B4552525D005B25735D57
:10BAD00025732025733A2025734E6F6E2D4C45201B
:10BAE00063617061626C6520636F6E74726F6C6C01
:10BAF00065722064657465637465642125730A004A
:10BB00001B5B303B33316D005B25735D2573202556
:10BB1000733A202573556E61626C6520746F2073D3
:10BB2000746F7265207374617469632061646472F8
:10BB300065737325730A005B25735D257320257378
:10BB40003A2025735573696E672074656D706F7246
:10BB5000617279207374617469632072616E646FBD
:10BB60006D206164647265737325730A005B2573CD
:10BB70005D25732025733A2025734F6E6C792073F1
:10BB800074617469632072616E646F6D20616464B6
:10BB90007265737320737570706F72746564206161
:10BBA00073206964656E7469747925730A00707511
:10BBB000626C69630072616E646F6D00307825306D
:10BBC000327800253032583A253032583A25303212
:10BBD000583A253032583A253032583A25303258C2
:10BBE000202825732900205B494E465D005B2573A4
:10BBF0005D25732025733A2025734964656E746949
:10BC000074793A20257325730A005B25735D2573CB
:10BC10002025733A2025734843493A20766572738C
:10BC2000696F6E20257320283078253032782920DE
:10BC30007265766973696F6E203078253034782CA0
:10BC4000206D616E756661637475726572203078FF
:10BC50002530347825730A005B25735D2573202514
:10BC6000733A2025734C4D503A2076657273696F94
:10BC70006E2025732028307825303278292073757E
:10BC8000627665722030782530347825730A005B3F
:10BC900025735D25732025733A202573556E6162E7
:10BCA0006C6520746F20736574206964656E7469B7
:10BCB0007479206164647265737325730A005B256F
:10BCC000735D25732025733A202573556E65787052
:10BCD0006563746564206B5F706F6C6C206576655E
:10BCE0006E7420737461746520257525730A005B7A
:10BCF00025735D25732025733A202573556E636C7B
:10BD000065617265642070656E64696E6720736535
:10BD10006E745F636D6425730A005B25735D257324
:10BD20002025733A2025736173736572743A202756
:10BD3000657272203D3D203027206661696C656424
:10BD400025730A005B25735D25732025733A202532
:10BD5000736173736572743A202762756627206673
:10BD600061696C656425730A00312E306200312EE2
:10BD70003100312E3200322E3000322E3100332E7F
:10BD80003000342E3000342E3100342E3200352E67
:10BD90003000436F6E74726F6C6C657200756E6B01
:10BDA0006E6F776E0001000202026863695F636D67
:10BDB000645F68616E646C6500656E636F64655F87
:10BDC000636F6E74726F6C006C655F756E6B6E6F17
:10BDD000776E5F72737000656E636F64655F646138
:10BDE00074615F6374726C005B25735D257320253D
:10BDF000733A2025734E6F2048434920436F6D6D81
:10BE0000616E642068656164657225730A005B2554
:10BE1000735D25732025733A202573496E76616C16
:10BE200069642048434920434D44207061636B6539
:10BE300074206C656E67746825730A005B25735DFA
:10BE400025732025733A202573747970653A203064
:10BE5000782530327825730A00656E636F64655FFC
:10BE60006E6F6465006863695F6472697665725FAE
:10BE700073656E64006863695F6472697665725F9A
:10BE80006F70656E0000000092BD000000000000B1
:10BE9000D52B0000592B00005B25735D25732025F1
:10BEA000733A2025734C4C20696E697469616C6922
:10BEB0007A6174696F6E206661696C65643A2025E9
:10BEC0007525730A005B25735D25732025733A2061
:10BED0002573456D70747920484349207061636B08
:10BEE000657425730A005B25735D25732025733AFD
:10BEF000202573556E6B6E6F776E20484349207412
:10BF000079706520257525730A00636E74725F73FE
:10BF1000746F70005B25735D25732025733A2025AF
:10BF2000736173736572743A20275F726566636F1D
:10BF3000756E7427206661696C656425730A0072EA
:10BF4000616E645F696E6974005B25735D257320A3
:10BF500025733A2025736173736572743A202763E1
:10BF60006F6E746578745F6C656E203E2073697ABD
:10BF7000656F66287374727563742072616E6429CC
:10BF800027206661696C656425730A007469636BB8
:10BF900065725F6A6F625F636F6D706172655F7516
:10BFA0007064617465007469636B65725F696E7358
:10BFB00074616E6365305F63616C6C65725F696448
:10BFC0005F676574007469636B65725F696E737433
:10BFD000616E6365315F63616C6C65725F69645F3C
:10BFE000676574007469636B65725F696E73746111
:10BFF0006E6365305F7363686564007469636B6565
:10C00000725F696E7374616E6365315F73636865D7
:10C0100064005B25735D25732025733A20257361C9
:10C0200073736572743A20276927206661696C65AD
:10C030006425730A00636F6D6D6F6E5F696E69745E
:10C04000006973725F726164696F5F7374617465B4
:10C050005F7478006973725F72785F6164760069FB
:10C0600073725F72785F6F6273006973725F727868
:10C070005F636F6E6E5F706B745F61636B0069739B
:10C08000725F72785F636F6E6E5F706B745F637404
:10C09000726C5F72656A5F636F6E6E5F757064006D
:10C0A0006973725F72785F636F6E6E5F706B745FDF
:10C0B0006374726C5F72656A006973725F72785F35
:10C0C000636F6E6E5F706B745F6374726C00697324
:10C0D000725F72785F636F6E6E5F706B740069730E
:10C0E000725F726164696F5F73746174655F7278A7
:10C0F000006973725F636C6F73655F61647600697A
:10C1000073725F636C6F73655F636F6E6E006973EC
:10C11000725F726164696F5F73746174655F636C91
:10C120006F736500697372007469636B65725F7326
:10C130007563636573735F617373657274007469AB
:10C14000636B65725F73746F705F6164765F617358
:10C1500073657274007469636B65725F73746F707A
:10C160005F6F62735F617373657274007469636B90
:10C1700065725F7570646174655F6164765F617339
:10C1800073657274007469636B65725F7570646166
:10C1900074655F736C6176655F617373657274005B
:10C1A0006D6179666C795F726164696F5F616374F8
:10C1B000697665006576656E745F6163746976653E
:10C1C000006576656E745F696E616374697665009B
:10C1D0006576656E745F7874616C006D6179666C0C
:10C1E000795F7874616C5F72657461696E007072FA
:10C1F00065706172655F6E6F726D616C5F7365749F
:10C20000006D6179666C795F7874616C5F73746FCF
:10C21000705F63616C630073636865645F6166741B
:10C2200065725F6D7374725F667265655F736C6F64
:10C23000745F6765740073636865645F66726565E3
:10C240005F77696E5F6F66667365745F63616C6369
:10C25000006D6179666C795F726164696F5F737498
:10C260006F70006576656E745F73746F70006576CD
:10C27000656E745F636F6D6D6F6E5F707265706118
:10C280007265006368616E5F736574006576656EE4
:10C29000745F616476006576656E745F6164765F75
:10C2A00073746F70006576656E745F636F6E6E5F3A
:10C2B0007570646174655F73745F696E697400653D
:10C2C00076656E745F636F6E6E5F757064617465C2
:10C2D0005F73745F726571006576656E745F636F1E
:10C2E0006E6E5F7570646174655F70726570006515
:10C2F00076656E745F7665785F70726570006576DE
:10C30000656E745F636F6E6E656374696F6E5F7088
:10C31000726570617265006576656E745F736C61DD
:10C320007665006576656E745F6D61737465720025
:10C330007061636B65745F72785F656E717565754A
:10C3400065007064755F6E6F64655F74785F7265B9
:10C350006C6561736500636F6E6E656374696F6EA3
:10C360005F72656C65617365007465726D696E619D
:10C3700074655F696E645F72785F656E717565750F
:10C380006500636F6E6E5F757064617465006368ED
:10C39000616E5F6D61705F75706461746500656E7C
:10C3A000635F7273705F73656E640073746172743F
:10C3B0005F656E635F7273705F73656E6400756E48
:10C3C0006B6E6F776E5F7273705F73656E6400661D
:10C3D0006561747572655F7273705F73656E64001A
:10C3E00070617573655F656E635F7273705F7365AF
:10C3F0006E640076657273696F6E5F696E645F73F9
:10C40000656E640072656A6563745F696E645F651A
:10C4100078745F73656E6400726F6C655F616374DE
:10C420006976655F64697361626C6500726F6C65E3
:10C430005F64697361626C6500726164696F5F72E9
:10C44000785F6465717565756500726164696F5FB9
:10C4500072785F6D656D5F72656C65617365005BB9
:10C4600025735D25732025733A20257361737365E9
:10C4700072743A20275F726164696F2E7469636B0E
:10C4800065725F69645F70726570617265203D3DC1
:10C49000203527206661696C656425730A005B2579
:10C4A000735D25732025733A20257361737365725C
:10C4B000743A2027287469636B65725F73746174C2
:10C4C0007573203D3D203029207C7C2028746963D1
:10C4D0006B65725F737461747573203D3D20322902
:10C4E00027206661696C656425730A005B25735DAE
:10C4F00025732025733A2025736173736572743A2E
:10C500002027726164696F5F7064755F6E6F646528
:10C510005F727827206661696C656425730A005B29
:10C5200025735D25732025733A2025736173736528
:10C5300072743A20275F726164696F2E7469636B4D
:10C5400065725F69645F70726570617265203D3D00
:10C55000202837202B20636F6E6E2D3E68616E643D
:10C560006C652927206661696C656425730A005B28
:10C5700025735D25732025733A20257361737365D8
:10C5800072743A20275F726164696F2E726F6C65F6
:10C59000203D3D20524F4C455F4E4F4E4527206673
:10C5A00061696C656425730A005B25735D257320E2
:10C5B00025733A2025736173736572743A20275F7F
:10C5C000726164696F2E7469636B65725F69645F21
:10C5D00070726570617265203D3D2036272066616E
:10C5E000696C656425730A00F401FA009600640022
:10C5F0004B0032001E0014005B25735D257320255F
:10C60000733A2025736173736572743A202721721F
:10C610006164696F5F69735F726561647928292756
:10C62000206661696C656425730A005B25735D256E
:10C63000732025733A2025736173736572743A20F1
:10C6400027646F6E6527206661696C656425730ACF
:10C65000005B25735D25732025733A202573617374
:10C66000736572743A202728636F6E6E2D3E6C6C72
:10C6700063705F726571203D3D20636F6E6E2D3E6D
:10C680006C6C63705F61636B29207C7C202828635D
:10C690006F6E6E2D3E6C6C63705F74797065203DBB
:10C6A0003D204C4C43505F434F4E4E454354494F01
:10C6B0004E5F555044415445292026262028636F5B
:10C6C0006E6E2D3E6C6C63702E636F6E6E65637460
:10C6D000696F6E5F7570646174652E7374617465E3
:10C6E000203D3D2035292927206661696C65642538
:10C6F000730A005B25735D25732025733A2025732B
:10C700006173736572743A2027636F6E6E2D3E728B
:10C710006F6C652E736C6176652E726F6C6520216F
:10C720003D203027206661696C656425730A005BD3
:10C7300025735D25732025733A2025736173736516
:10C7400072743A2027636F6E6E2D3E6C6C63705F5F
:10C75000726571203D3D20636F6E6E2D3E6C6C6383
:10C76000705F61636B27206661696C656425730A7D
:10C77000005B25735D25732025733A202573617353
:10C78000736572743A20275F726164696F2E636FFC
:10C790006E6E5F637572722D3E6C6C63705F726556
:10C7A00071203D3D205F726164696F2E636F6E6E14
:10C7B0005F637572722D3E6C6C63705F61636B2793
:10C7C000206661696C656425730A005B25735D25CD
:10C7D000732025733A2025736173736572743A2050
:10C7E000275F726164696F2E636F6E6E5F75706430
:10C7F000203D3D205F726164696F2E636F6E6E5FD6
:10C800006375727227206661696C656425730A001E
:10C810005B25735D25732025733A2025736173733F
:10C820006572743A2027287469636B65725F73744C
:10C8300061747573203D3D203029207C7C20287454
:10C8400069636B65725F737461747573203D3D201D
:10C850003229207C7C20285F726164696F2E7469A4
:10C86000636B65725F69645F73746F70203D3D2018
:10C87000352927206661696C656425730A005B258C
:10C88000735D25732025733A202573617373657278
:10C89000743A2027287469636B65725F73746174DE
:10C8A0007573203D3D203029207C7C2028746963ED
:10C8B0006B65725F737461747573203D3D2032291E
:10C8C000207C7C20285F726164696F2E7469636BC1
:10C8D00065725F69645F73746F70203D3D20746999
:10C8E000636B65725F69642927206661696C6564A2
:10C8F00025730A005B25735D25732025733A202577
:10C90000736173736572743A2027285F726164697A
:10C910006F2E7374617465203D3D2053544154451E
:10C920005F53544F5029207C7C20285F72616469DA
:10C930006F2E7374617465203D3D205354415445FE
:10C940005F41424F52542927206661696C65642516
:10C95000730A005B25735D25732025733A202573C8
:10C960006173736572743A2027735F6163746976CB
:10C970006527206661696C656425730A005B257311
:10C980005D25732025733A20257361737365727476
:10C990003A2027287374617465203D3D205354412B
:10C9A00054455F53544F5029207C7C202873746178
:10C9B0007465203D3D2053544154455F41424F52E0
:10C9C000542927206661696C656425730A005B251C
:10C9D000735D25732025733A202573617373657227
:10C9E000743A202763616C6C65725F6964203D3D19
:10C9F000203127206661696C656425730A005B2518
:10CA0000735D25732025733A2025736173736572F6
:10CA1000743A20272830203D3D207469636B65728D
:10CA20005F73746174757329207C7C202832203DEB
:10CA30003D207469636B65725F73746174757329EB
:10CA400027206661696C656425730A005B25735D48
:10CA500025732025733A2025736173736572743AC8
:10CA600020275F726164696F2E7061636B65745F0C
:10CA700072785F6C61737420213D205F726164691C
:10CA80006F2E7061636B65745F72785F616371753F
:10CA900069726527206661696C656425730A005BAD
:10CAA00025735D25732025733A20257361737365A3
:10CAB00072743A20276C696E6B27206661696C6519
:10CAC0006425730A005B25735D25732025733A2066
:10CAD00025736173736572743A20276C61737420D7
:10CAE000213D205F726164696F2E7061636B6574B4
:10CAF0005F72656C656173655F6669727374272028
:10CB00006661696C656425730A005B25735D257336
:10CB10002025733A2025736173736572743A202758
:10CB20005F726164696F2E6C696E6B5F72785F64AF
:10CB30006174615F71756F7461203C20285F726160
:10CB400064696F2E7061636B65745F72785F636F89
:10CB5000756E74202D20312927206661696C65640B
:10CB600025730A005B25735D25732025733A202504
:10CB7000736173736572743A2027215F726164690F
:10CB80006F2E7469636B65725F69645F73746F7035
:10CB900027206661696C656425730A005B25735DF7
:10CBA00025732025733A2025736173736572743A77
:10CBB00020277265745F636220213D203227206642
:10CBC00061696C656425730A005B25735D257320BC
:10CBD00025733A2025736173736572743A20272197
:10CBE00072657476616C27206661696C6564257373
:10CBF0000A005B25735D25732025733A2025736138
:10CC000073736572743A2027287265745F636220BB
:10CC10003D3D203029207C7C20287265745F636252
:10CC2000203D3D20312927206661696C65642573AC
:10CC30000A005B25735D25732025733A20257361F7
:10CC400073736572743A20277265745F6362203D66
:10CC50003D203027206661696C656425730A005B9E
:10CC600025735D25732025733A20257361737365E1
:10CC700072743A20276E6F64655F7478272066614E
:10CC8000696C656425730A005B25735D2573202537
:10CC9000733A2025736173736572743A2027726149
:10CCA00064696F5F7064755F6E6F64655F72782D25
:10CCB0003E6864722E6F6E696F6E2E6C696E6B27A4
:10CCC000206661696C656425730A005B25735D25C8
:10CCD000732025733A2025736173736572743A204B
:10CCE00027737461747573203D3D20302720666181
:10CCF000696C656425730A005B25735D25732025C7
:10CD0000733A2025736173736572743A2027287310
:10CD10007461747573203D3D203029207C7C20286F
:10CD20005F726164696F2E7469636B65725F6964B9
:10CD30005F73746F70203D3D20352927206661693F
:10CD40006C656425730A005B25735D25732025736C
:10CD50003A2025736173736572743A2027287374BF
:10CD600061747573203D3D203029207C7C20285F34
:10CD7000726164696F2E7469636B65725F69645F69
:10CD800073746F70203D3D207469636B65725F69D9
:10CD9000642927206661696C656425730A006D61EA
:10CDA00079666C795F656E61626C655F6362006D68
:10CDB0006179666C795F69735F656E61626C6564E9
:10CDC000006D6179666C795F70656E64006C6C5F94
:10CDD000696E6974005B25735D25732025733A20A5
:10CDE000257352657175697265642052414D2073D7
:10CDF000697A653A2025642C20737570706C6965BA
:10CE0000643A2025752E25730A005B25735D257312
:10CE10002025733A2025736173736572743A202755
:10CE200063616C6C65655F6964203D3D203127203E
:10CE30006661696C656425730A00464C4153485F1E
:10CE400030005352414D5F300046414354555345E5
:10CE5000524346475F30005045524950485F3000CA
:10CE60005050425F30002A2A2A2A2A204255532055
:10CE70004641554C54202A2A2A2A2A0A00202050AA
:10CE800072656369736520646174612062757320E3
:10CE90006572726F720A002020496D707265636955
:10CEA0007365206461746120627573206572726FAE
:10CEB000720A002020496E737472756374696F6E14
:10CEC00020627573206572726F720A005265736515
:10CED0007276656420457863657074696F6E20288A
:10CEE0000053707572696F757320696E7465727224
:10CEF000757074202849525120002A2A2A2A2A2093
:10CF000048415244204641554C54202A2A2A2A2A74
:10CF10000A002020427573206661756C74206F6E64
:10CF200020766563746F72207461626C652072652F
:10CF300061640A0020204661756C7420657363612A
:10CF40006C6174696F6E20287365652062656C6F13
:10CF500077290A002A2A2A2A2A204465627567202E
:10CF60006D6F6E69746F7220657863657074696F38
:10CF70006E20286E6F7420696D706C656D656E74BF
:10CF8000656429202A2A2A2A2A0A002A2A2A2A2AE1
:10CF900020257320256429202A2A2A2A2A0A0020EB
:10CFA00020457865637574696E6720746872656181
:10CFB000642049442028746872656164293A2025F8
:10CFC000700A20204661756C74696E6720696E7303
:10CFD0007472756374696F6E2061646472657373D3
:10CFE0003A2020307825780A002A2A2A2A2A204D39
:10CFF0005055204641554C54202A2A2A2A2A0A00F4
:10D000002020537461636B696E67206572726F7262
:10D010000A002020556E737461636B696E6720652A
:10D0200072726F720A002020446174612041636350
:10D030006573732056696F6C6174696F6E0A0020A6
:10D0400020416464726573733A20307825780A0051
:10D050002020496E737472756374696F6E2041632A
:10D06000636573732056696F6C6174696F6E0A0033
:10D070002A2A2A2A2A205553414745204641554C01
:10D0800054202A2A2A2A2A0A002020446976697311
:10D09000696F6E206279207A65726F0A00202055D0
:10D0A0006E616C69676E6564206D656D6F72792065
:10D0B0006163636573730A0020204E6F20636F7095
:10D0C000726F636573736F7220696E7374727563C8
:10D0D00074696F6E730A002020496C6C6567616C1F
:10D0E000206C6F6164206F66204558435F52455441
:10D0F00055524E20696E746F2050430A002020491B
:10D100006C6C6567616C20757365206F6620746850
:10D110006520455053520A002020417474656D709B
:10D120007420746F206578656375746520756E640E
:10D130006566696E656420696E737472756374697F
:10D140006F6E0A002A2A2A2A2A20496E76616C69A3
:10D1500064204578697420536F6674776172652026
:10D160004572726F7221202A2A2A2A2A0A002A2A44
:10D170002A2A204B65726E656C20416C6C6F63616E
:10D1800074696F6E204661696C75726521202A2A68
:10D190002A2A0A002A2A2A2A2A204B65726E656CDE
:10D1A000204F4F505321202A2A2A2A2A0A002A2AAD
:10D1B0002A2A2A204B65726E656C2050616E696365
:10D1C00021202A2A2A2A2A0A002A2A2A2A20556EB7
:10D1D0006B6E6F776E20466174616C204572726F62
:10D1E0007220256421202A2A2A2A0A004375727295
:10D1F000656E7420746872656164204944203D2026
:10D2000025700A4661756C74696E6720696E737467
:10D2100072756374696F6E206164647265737320E4
:10D220003D20307825780A004953520065737365B4
:10D230006E7469616C207468726561640046617423
:10D24000616C206661756C7420696E2025732120E5
:10D250005370696E6E696E672E2E2E0A00466174D9
:10D26000616C206661756C7420696E2074687265EB
:10D270006164202570212041626F7274696E672E8F
:10D280000A000000000300203C0300203C030020B3
:10D290007803002078030020F5FFFFFF0C13002027
:10D2A00004AAFEAAFE1000007A6570687972707296
:10D2B0006F6A65637408000000C201006F0E000011
:10D2C000000000000000000000000000000000005E
:10D2D000000000000000000000000000000000004E
:10D2E000000000000000000000000000000000003E
:10D2F000000000000000000000000000000000002E
:10D30000000000000000000000000000000000001D
:10D31000000000000000000000000000000000000D
:10D3200000000000F51A00000000000000000000EE
:10D3300000000000000000000000000000000000ED
:10D34000A0000020A000002001000000010000005B
:10D3500000000000000000000000000000000000CD
:10D36000000000000000000000000000CC000020D1
:10D37000CC000020000000000000000000000000C1
:10D380000000000000000000000000000004000099
:10D39000CC000020F4000020F40000200000000079
:10D3A0000000000000000000020002004C00080025
:10D3B00000000000FC1C00201801002018010020C3
:10D3C0000000000000000000000000000300030057
:10D3D0004C00040000000000F822002000000000C3
:10D3E000FFFFFFFFFF1F00001F0000000000000004
:10D3F00000000000500A0020F8090020053B000052
:10D4000000000000580A0020F8090020B13B00008D
:10D4100000000000600A0020F8090020053B000021
:10D4200000000000680A0020F8090020B13B00005D
:10D4300000000000700A0020F8090020B13B000045
:10D4400000000000780A0020240A0020053B0000AC
:10D4500000000000800A0020240A0020B13B0000E8
:10D4600000000000880A0020240A0020053B00007C
:10D4700000000000900A0020240A0020B13B0000B8
:10D4800000000000980A0020240A0020B13B0000A0
:10D4900000000000240F002001000000ED560000F5
:10D4A000000000002C0F0020000000005557000075
:10D4B000000000006C0F0020000000005557000025
:10D4C00000000000540F0020000000005D57000025
:10D4D000000000007C0F0020000000005D570000ED
:10D4E00000000000640F00200000000000000000A9
:10D4F00000000000340F002000000000E96300007D
:10D50000000000003C0F002000000000E963000064
:10D5100000000000440F002000000000F96300003C
:10D52000000000004C0F002000000000F963000024
:10D5300000000000740F002000000000F9630000EC
:10D54000000000005C0F002000000000815E000071
:10D550000090D00305000000BC0200200000000085
:10D560003ACE0000240008070000002042CE000050
:10D570001E0008130000001049CE00001800100320
:10D580000000004057CE000038001003000000E00B
:10D5900060CE00001E000403030000000100000034
:10D5A0008CB50000000000000000000098B50000ED
:10D5B000000000000000000044B500000000000072
:10D5C0001800002068B500004CB700000000000003
:10D5D00074B5000058B700000000000050B500000E
:10D5E00000000000000000005CB5000030B7000043
:10D5F000C4030020A4B500000000000000000000EB
:10D6000080B50000000000000000000038B50000F8
:08D61000000000000000000012
:10D61800780300207803002000000000FFFFFFFFD0
:04D6280000000000FE
:10D62C008C0300208C030020000000000000000090
:04D63C000F000000DB
:10D64000A0030020A0030020000000000000000054
:04D6500000000000D6
:040000030000A25106
:00000001FF
